:1000000000000320D501000051020000AFE5000010
:1000100055020000570200005902000000000000D5
:100020000000000000000000000000005B02000073
:100030005D020000000000005F020000610200009D
:100040002DDD000035DD00003DDD000045DD000058
:100050004DDD000055DD00005DDD000065DD0000C8
:100060006DDD000075DD00007DDD000085DD000038
:100070008DDD000095DD00009DDD0000A5DD0000A8
:10008000ADDD0000B5DD0000BDDD0000C5DD000018
:10009000CDDD0000D5DD0000DDDD0000E5DD000088
:1000A000ED240000EDDD0000F5DD0000FDDD0000C9
:1000B00005DE00000DDE000015DE00001DDE000084
:1000C00025DE00002DDE000035DE00003DDE0000F4
:1000D00045DE00004DDE000055DE00001D6B000017
:1000E0005DDE000065DE00006DDE000075DE0000F4
:1000F0007DDE000085DE00008DDE000095DE000064
:10010000416A00009DDE0000A5DE0000ADDE0000BB
:10011000B5DE0000BDDE0000C5DE0000CDDE000063
:10012000D5DE0000DDDE0000E5DE0000EDDE0000D3
:1001300069780000C97800009978000081D100003A
:10014000F5DE0000FDDE000005DF00000DDF000031
:1001500015DF00001DDF000025DF00002DDF00009F
:1001600035DF0000D91300003DDF000045DF00004F
:100170004DDF000055DF00005DDF000065DF00009F
:100180006DDF000075DF00007DDF000085DF00000F
:100190008DDF000095DF00008810010000000020C6
:1001A000C0580000881001000000FF1F0000000080
:1001B000881001000000001400000000C05800205A
:1001C000587801000000FF1F00000000000000142C
:1001D0000000000010B572B60CF0E0F80D4B07E01F
:1001E00003F10C049A685968186800F019F823465E
:1001F000094A9342F4D306E01C46596854F8080BA8
:1002000000F01DF82346054A9342F5D362B60FF07D
:10021000B5FAFEE798010000BC010000D40100001F
:10022000002393420AD210B450F8044B41F8044B17
:1002300004339342F8D35DF8044B704770470023B2
:100240008B4204D2002240F8042B0433F8E77047B5
:10025000FEE7FEE7FEE7FEE7FEE7FEE7FEE7FEE776
:10026000FEE7FEE7FFFFFFFFFFFFFFFFFFFFFFFFD0
:10027000FFFFFFFFFFFFFFFFFFFFFFFFFFFFFFFF8E
:10028000FFFFFFFFFFFFFFFFFFFFFFFFFFFFFFFF7E
:10029000FFFFFFFFFFFFFFFFFFFFFFFFFFFFFFFF6E
:1002A000FFFFFFFFFFFFFFFFFFFFFFFFFFFFFFFF5E
:1002B000FFFFFFFFFFFFFFFFFFFFFFFFFFFFFFFF4E
:1002C000FFFFFFFFFFFFFFFFFFFFFFFFFFFFFFFF3E
:1002D000FFFFFFFFFFFFFFFFFFFFFFFFFFFFFFFF2E
:1002E000FFFFFFFFFFFFFFFFFFFFFFFFFFFFFFFF1E
:1002F000FFFFFFFFFFFFFFFFFFFFFFFFFFFFFFFF0E
:10030000FFFFFFFFFFFFFFFFFFFFFFFFFFFFFFFFFD
:10031000FFFFFFFFFFFFFFFFFFFFFFFFFFFFFFFFED
:10032000FFFFFFFFFFFFFFFFFFFFFFFFFFFFFFFFDD
:10033000FFFFFFFFFFFFFFFFFFFFFFFFFFFFFFFFCD
:10034000FFFFFFFFFFFFFFFFFFFFFFFFFFFFFFFFBD
:10035000FFFFFFFFFFFFFFFFFFFFFFFFFFFFFFFFAD
:10036000FFFFFFFFFFFFFFFFFFFFFFFFFFFFFFFF9D
:10037000FFFFFFFFFFFFFFFFFFFFFFFFFFFFFFFF8D
:10038000FFFFFFFFFFFFFFFFFFFFFFFFFFFFFFFF7D
:10039000FFFFFFFFFFFFFFFFFFFFFFFFFFFFFFFF6D
:1003A000FFFFFFFFFFFFFFFFFFFFFFFFFFFFFFFF5D
:1003B000FFFFFFFFFFFFFFFFFFFFFFFFFFFFFFFF4D
:1003C000FFFFFFFFFFFFFFFFFFFFFFFFFFFFFFFF3D
:1003D000FFFFFFFFFFFFFFFFFFFFFFFFFFFFFFFF2D
:1003E000FFFFFFFFFFFFFFFFFFFFFFFFFFFFFFFF1D
:1003F000FFFFFFFFFFFFFFFFFFFFFFFFFFFFFFFF0D
:10040000FFFFFFFFFFFFFFFFFFFFFFFFFEFFFFFFFD
:1004100080B596B000AF78607B689B10FB64934B0F
:100420001A68FB6C1B0113441B68BB647B685A424F
:1004300003F0030302F0030258BF53427B648B4B6B
:100440001A68FB6C1B0113445B6807EE903AB8EE28
:10045000677ADFED876AC7EE267AB1EE007A67EE3B
:10046000877AC7ED157A814B1A68FB6C1B01134420
:100470009B6807EE903AB8EE677ADFED7D6AC7EECB
:10048000267AB1EE007A67EE877AC7ED147A794B57
:100490009B68002B48D0784AFB6C063352F8233017
:1004A000002B26D0754B1A68FB6C1B0113449B680C
:1004B00040F6DB72934237D86F4AFB6C063300215B
:1004C00042F82310FB6C9B0003331B016C4A1A4457
:1004D000FB6C9B0003336B492C2000FB03F30B44A4
:1004E0001433D3ED007AB0EE670A10460DF0ECFF3E
:1004F0001AE0624B1A68FB6C1B0113449B6840F6C0
:10050000FA72934210D95C4AFB6C0633012142F81F
:100510002310FB6C9B0003331B01594A1344B6EEB6
:10052000000A18460DF0D0FF534AFB6C063352F810
:100530002330002B0DD0D7ED147A67EEA77AC7EDE4
:10054000147A97ED147AF3EE006AC7EE267AC7EDB7
:10055000147AD7ED157AB6EE007A77EEC77AC7ED42
:10056000157AD7ED157AF5EEC07AF1EE10FA06D5C8
:10057000D7ED157AB1EE007A77EE877A01E0D7ED04
:10058000157AC7ED157A3C4AFB6C063352F82330D6
:10059000002B12D03C49FA6C13465B0013449B00BD
:1005A0000B4404331B683B65D7ED147AB1EE007A37
:1005B00067EE877AC7ED157A1CE03349FA6C13466B
:1005C0005B0013449B000B44083393ED007AD7ED96
:1005D000147A67EE277A97ED157A77EE277AC7EDCA
:1005E000157A07E0D7ED157AB1EE007A77EE877AC3
:1005F000C7ED157AD7ED157AF5EEC07AF1EE10FA5F
:10060000F0D407E0D7ED157AB1EE007A77EEC77A2D
:10061000C7ED157AD7ED157AB1EE007AF4EEC77A08
:10062000F1EE10FAEEDCB1EE001ADFED180A97EDEC
:10063000150A0DF0CEFD87ED150AD7ED157AB0EE4F
:10064000007A77EE877AC7ED107AD7ED107AB1EE9F
:10065000007AF4EEC77AF1EE10FA19DDD7ED107AD0
:10066000B1EE007A77EEC77A14E000BF04000020F4
:1006700000F07F4508000020505A002000000020B4
:10068000E86E0020C86A0020746A002000000000A4
:10069000D7ED107AC7ED107AA34B1A68FB6C1B01DB
:1006A00013445B6807EE903AB8EE677ADFED9F6A15
:1006B000C7EE267AC7ED0F7AB7EE007AD7ED0F7A3C
:1006C00077EE677AC7ED0F7AD7ED0F7A67EEA77AE4
:1006D000C7ED0E7AD7ED0F7A9FED957A67EE877AA0
:1006E000C7ED0D7A934AFB6C063352F82330002B8A
:1006F00040F04482D7ED157AB7EE007AF4EEC77A6F
:10070000F1EE10FA7BD58C4BD3ED037A8B4B93ED46
:10071000007AB0EE471ADFED8A0AB0EE670A0DF0F4
:100720001EFDF0EE407A844BC3ED037A824BD3ED8D
:10073000027A824B93ED007AB0EE471ADFED800A21
:10074000B0EE670A0DF00BFDF0EE407A7A4BC3ED88
:10075000027A786D0DF0CEFA71A3D3E900230DF083
:100760000FF802460B46104619464FF000024FF0B4
:1007700080430DF08FF802460B46104619460DF0E7
:100780008DFA034600EE103A0FF007F8F0EE407ACB
:10079000DFED6C0AB0EE670A00F092FFF0EE407AEF
:1007A000654BC3ED017A786D0DF0A4FA5CA3D3E933
:1007B00000230CF0E5FF02460B46104619464FF0A9
:1007C00000024FF080430DF065F802460B461046DC
:1007D00019460DF063FA034600EE103A0CF09AFD4C
:1007E000F0EE407ADFED570AB0EE670A00F068FFDE
:1007F000F0EE407A504BC3ED007A00F001BDD7ED2A
:10080000157AB0EE007AF4EEC77AF1EE10FA40F104
:100810009B80D7ED157AB7EE007A77EEC77AC7EDF1
:10082000157A454BD3ED037A444B93ED007AB0EE45
:10083000471ADFED430AB0EE670A0DF090FCF0EEC8
:10084000407A3D4BC3ED037A786D0DF053FA34A333
:10085000D3E900230CF094FF02460B4610461946DC
:100860004FF000024FF080430DF014F802460B46A3
:10087000104619460DF012FA034600EE103A0EF03B
:100880008CFFF0EE407ADFED2F0AB0EE670A00F041
:1008900017FFF0EE407A284BC3ED027A786D0DF029
:1008A00029FA1FA3D3E900230CF06AFF02460B4686
:1008B000104619464FF000024FF080430CF0EAFF5B
:1008C00002460B46104619460DF0E8F9034600EEC5
:1008D000103A0CF01FFDF0EE407ADFED1A0AB0EE90
:1008E000670A00F0EDFEF0EE407A134BC3ED017A9B
:1008F000114BD3ED007A114B93ED007AB0EE471A0D
:10090000DFED0F0AB0EE670A0DF029FCF0EE407A39
:10091000094BC3ED007A00F073BC00BFAFF3008059
:10092000182D4454FB2109400400002000F07F45AD
:1009300052B85E3F505A0020405A002030580020E4
:10094000000000009A99193FD7ED157AB0EE087AA9
:10095000F4EEC77AF1EE10FA40F18380D7ED157A04
:10096000B0EE007A77EEC77AC7ED157A786D0DF0A4
:10097000C1F9E7A3D3E900230CF002FF02460B46BE
:10098000104619464FF000024FF080430CF082FFF2
:1009900002460B46104619460DF080F9034600EE5C
:1009A000103A0EF0FAFEF0EE407ADFEDDB0AB0EE20
:1009B000670A00F085FEF0EE407AD84BC3ED037A6B
:1009C000786D0DF097F9D2A3D3E900230CF0D8FE8F
:1009D00002460B46104619464FF000024FF0804386
:1009E0000CF058FF02460B46104619460DF056F91A
:1009F000034600EE103A0CF08DFCF0EE407ADFED8D
:100A0000C60AB0EE670A00F05BFEF0EE407AC34B18
:100A1000C3ED027AC14BD3ED017AC14B93ED007A5D
:100A2000B0EE471ADFEDBF0AB0EE670A0DF097FB94
:100A3000F0EE407AB94BC3ED017AB84BD3ED007AB2
:100A4000B74B93ED007AB0EE471ADFEDB60AB0EE81
:100A5000670A0DF084FBF0EE407AB04BC3ED007AEC
:100A6000CEE3D7ED157AB1EE007AF4EEC77AF1EE67
:100A700010FA00F2C583D7ED157AB0EE087A77EE5A
:100A8000C77AC7ED157A786D0DF034F9A0A3D3E9D4
:100A900000230CF075FE02460B46104619464FF037
:100AA00000024FF080430CF0F5FE02460B46104664
:100AB00019460DF0F3F8034600EE103A0EF06DFE05
:100AC000F0EE407ADFED940AB0EE670A00F0F8FD30
:100AD000F0EE407A914BC3ED007A786D0DF00AF993
:100AE0008BA3D3E900230CF04BFE02460B461046C5
:100AF00019464FF000024FF080430CF0CBFE024647
:100B00000B46104619460DF0C9F8034600EE103AA0
:100B10000CF000FCF0EE407ADFED7F0AB0EE670AE1
:100B200000F0CEFDF0EE407A7C4BC3ED037A7B4BB8
:100B3000D3ED027A7A4B93ED007AB0EE471ADFEDEF
:100B4000790AB0EE670A0DF00AFBF0EE407A734BBB
:100B5000C3ED027A714BD3ED017A714B93ED007ABC
:100B6000B0EE471ADFED6F0AB0EE670A0DF0F7FA44
:100B7000F0EE407A694BC3ED017A41E3D7ED157A87
:100B8000B7EE007AF4EEC77AF1EE10FA40F1CC80BD
:100B9000786D0DF0AFF85EA3D3E900230CF0F0FD03
:100BA00002460B46104619464FF000024FF08043B4
:100BB0000CF070FE02460B46104619460DF06EF81A
:100BC000034600EE103A0EF0E8FD87ED060A786D58
:100BD0000DF090F84EA3D3E900230CF0D1FD0246AE
:100BE0000B46104619464FF000024FF080430CF0C0
:100BF00051FE02460B46104619460DF04FF80346CB
:100C000000EE103A0CF086FB87ED050AD7ED067A68
:100C100027EEA77AD7ED067A67EE277A97ED0E1AB8
:100C2000F0EE670A97ED060A0DF04BFAF0EE407A07
:100C30003A4BC3ED017AD7ED057A27EEA77AD7EDC7
:100C4000057A67EE277A97ED0E1AF0EE670A97EDB0
:100C5000050A0DF036FAF0EE407A304BC3ED007A1B
:100C6000D7ED107AB0EE007A77EEC77AC7ED107A3A
:100C7000386C0DF03FF826A3D3E900230CF080FD7B
:100C800002460B46104619464FF000024FF08043D3
:100C90000CF000FE02460B46104619460CF0FEFF13
:100CA000034600EE103A0EF078FDB0EE407AD7ED34
:100CB0000D7A67EE277A194BC3ED037A386C0DF085
:100CC00019F813A3D3E900230CF05AFD02460B4692
:100CD000104619464FF000024FF080430CF0DAFD49
:100CE00002460B46104619460CF0D8FF034600EEAC
:100CF000103A0CF00FFBB0EE407AD7ED0D7A67EEAC
:100D0000277A064BC3ED027A7AE200BFAFF3008088
:100D1000182D4454FB2109409A99193F405A00204C
:100D20003058002000000000D7ED157AB0EE007AB0
:100D3000F4EEC77AF1EE10FA40F1C580D7ED157ADE
:100D4000B7EE007A77EEC77AC7ED157A786D0CF0BA
:100D5000D1FFC1A3D3E900230CF012FD02460B46DC
:100D6000104619464FF000024FF080430CF092FD00
:100D700002460B46104619460CF090FF034600EE63
:100D8000103A0EF00AFD87ED080A786D0CF0B2FFFC
:100D9000B1A3D3E900230CF0F3FC02460B46104646
:100DA00019464FF000024FF080430CF073FD0246ED
:100DB0000B46104619460CF071FF034600EE103A40
:100DC0000CF0A8FA87ED070AD7ED087A27EEA77A84
:100DD000D7ED087A67EE277A97ED0E1AF0EE670ADC
:100DE00097ED080A0DF06DF9F0EE407A9C4BC3EDDB
:100DF000027AD7ED077A27EEA77AD7ED077A67EE62
:100E0000277A97ED0E1AF0EE670A97ED070A0DF0B4
:100E100058F9F0EE407A924BC3ED017AD7ED107A93
:100E2000B0EE087A77EEC77AC7ED107A386C0CF01E
:100E300061FF89A3D3E900230CF0A2FC02460B4614
:100E4000104619464FF000024FF080430CF022FD8F
:100E500002460B46104619460CF020FF034600EEF2
:100E6000103A0EF09AFCB0EE407AD7ED0D7A67EEAC
:100E7000277A7B4BC3ED007A386C0CF03BFF76A3EE
:100E8000D3E900230CF07CFC02460B4610461946C1
:100E90004FF000024FF080430CF0FCFC02460B4682
:100EA000104619460CF0FAFE034600EE103A0CF01C
:100EB00031FAB0EE407AD7ED0D7A67EE277A684BBB
:100EC000C3ED037A9CE1D7ED157AB0EE087AF4EE23
:100ED000C77AF1EE10FA40F1C580D7ED157AB0EE81
:100EE000007A77EEC77AC7ED157A786D0CF002FFBD
:100EF00059A3D3E900230CF043FC02460B461046ED
:100F000019464FF000024FF080430CF0C3FC02463C
:100F10000B46104619460CF0C1FE034600EE103A8F
:100F20000EF03BFC87ED0A0A786D0CF0E3FE4AA355
:100F3000D3E900230CF024FC02460B461046194668
:100F40004FF000024FF080430CF0A4FC02460B4629
:100F5000104619460CF0A2FE034600EE103A0CF0C3
:100F6000D9F987ED090AD7ED0A7A27EEA77AD7EDE6
:100F70000A7A67EE277A97ED0E1AF0EE670A97ED78
:100F80000A0A0DF09EF8F0EE407A354BC3ED037A75
:100F9000D7ED097A27EEA77AD7ED097A67EE277A97
:100FA00097ED0E1AF0EE670A97ED090A0DF089F831
:100FB000F0EE407A2A4BC3ED027A386C0CF09AFEC0
:100FC00025A3D3E900230CF0DBFB02460B461046B9
:100FD00019464FF000024FF080430CF05BFC0246D4
:100FE0000B46104619460CF059FE034600EE103A27
:100FF0000EF0D3FBB0EE407AD7ED0D7A67EE277A8C
:10100000174BC3ED017A386C0CF074FE12A3D3E9D0
:1010100000230CF0B5FB02460B46104619464FF074
:1010200000024FF080430CF035FC02460B461046A0
:1010300019460CF033FE034600EE103A0CF06AF944
:10104000B0EE407AD7ED0D7A67EE277A044BC3ED08
:10105000007AD5E0AFF30080182D4454FB210940FD
:10106000405A0020D7ED157AB1EE007AF4EEC77A37
:10107000F1EE10FA00F2C480D7ED157AB0EE087ADE
:1010800077EEC77AC7ED157A786D0CF033FEC8A3FA
:10109000D3E900230CF074FB02460B4610461946B8
:1010A0004FF000024FF080430CF0F4FB02460B4679
:1010B000104619460CF0F2FD034600EE103A0EF011
:1010C0006CFB87ED0C0A786D0CF014FEB8A3D3E925
:1010D00000230CF055FB02460B46104619464FF014
:1010E00000024FF080430CF0D5FB02460B46104641
:1010F00019460CF0D3FD034600EE103A0CF00AF945
:1011000087ED0B0AD7ED0C7A27EEA77AD7ED0C7A8C
:1011100067EE277A97ED0E1AF0EE670A97ED0C0A44
:101120000CF0CFFFF0EE407AA34BC3ED007AD7ED81
:101130000B7A27EEA77AD7ED0B7A67EE277A97ED31
:101140000E1AF0EE670A97ED0B0A0CF0BAFFF0EEFC
:10115000407A994BC3ED037AD7ED107AB7EE007A57
:1011600077EEC77AC7ED107A386C0CF0C3FD90A308
:10117000D3E900230CF004FB02460B461046194647
:101180004FF000024FF080430CF084FB02460B4608
:10119000104619460CF082FD034600EE103A0EF0A0
:1011A000FCFAB0EE407AD7ED0D7A67EE277A824BE3
:1011B000C3ED027A386C0CF09DFD7DA3D3E90023CA
:1011C0000CF0DEFA02460B46104619464FF00002BC
:1011D0004FF080430CF05EFB02460B46104619466A
:1011E0000CF05CFD034600EE103A0CF093F8B0EE04
:1011F000407AD7ED0D7A67EE277A6F4BC3ED017A0F
:101200006E4AFB6C063352F82330002B24D06C4B13
:101210001A68FB6C1B011344DB6807EE903AB8EECA
:10122000677ADFED686AC7EE267A77EEA77AB7EEBF
:10123000007A77EEC77AF0EE000AB0EE670A00F0A7
:101240003FFAF0EE407AB1EE007A67EE877AB7EEB9
:10125000007A77EE877A2DE0594B1A68FB6C1B01F8
:101260001344DB6807EE903AF8EE677ADFED556AD3
:1012700087EEA67AF0EE000AB0EE470A00F020FAF8
:10128000F0EE406A4E4B1A68FB6C1B0113449B68DE
:1012900007EE903AB8EE677A9FED4A6AC7EE067A93
:1012A00066EEA77AB0EE087A67EE877AB7EE007A34
:1012B00077EE877AC7ED047ABB6C07EE903AB8EE0A
:1012C000E77AD7ED047A27EE277A3B4A7B6C9B00BE
:1012D0001344D3ED007A67EE277AFDEEE77A17EE36
:1012E000903ABB64BB6C07EE903AF8EEE77A9FED5C
:1012F000351ADFED350AB0EE670A0CF06AFFF0EE42
:10130000407AB7EE002ADFED301A9FED301ADFED9C
:101310002E0AB0EE670A00F07DFC87ED030AD7EDD8
:10132000037A9FED2B7AF4EEC77AF1EE10FA10D51E
:101330009FED282ADFED241A9FED251ADFED220A02
:1013400097ED030A00F066FCF0EE407AFDEEE77AD6
:101350001FE0B7EE002ADFED1C1AB7EE001ADFED32
:101360001C0A97ED030A00F055FCF0EE407AB0EE4F
:10137000670A0CF0E4FEF0EE407AB0EE671ADFED9B
:10138000110A9FED140A0CF0EAFEF0EE407AFDEE31
:10139000E77AC7ED127ABB6C07EE903AF8EEE77A7F
:1013A000B0EE670A5837BD4680BD00BFAFF300807E
:1013B000182D4454FB210940405A0020505A002067
:1013C0000400002000F07F450000000000007A4586
:1013D0000AD7233C00400345B0B584B000AFAC4B06
:1013E0007B600021AB4800F0FFFBAB4B1B685A1C35
:1013F000A9490A609B007A68134402461A60A64B0A
:101400001968A64B83FB01235A10CB17D21A134637
:10141000DB001344CA1AA04B1A609F4B1B68DB0009
:101420009F4A13441A4600219A4809F01DF90023E7
:10143000FB601AE19B4B1A68FB681B011344DB68D5
:1014400007EE903AF8EE677AC7ED027A964AFB68A3
:10145000063352F82330002B36D0D7ED027A9FEDB9
:10146000937A77EEC77AC7ED027A97ED027ADFEDCD
:10147000906AC7EE267AC7ED027AB8680CF03AFC9B
:1014800002460B4643EC102B0EF09FFA55EC104B26
:10149000B8680CF02FFC02460B46204629460CF09B
:1014A0006FF902460B46104619460CF0F7FB03464F
:1014B000BB60B7EE001AFFEE000A97ED020A0CF0CF
:1014C00088FE87ED020A1BE097ED027ADFED796A6C
:1014D000C7EE267AC7ED027AD7ED027A9FED767ACB
:1014E000F4EEC77AF1EE10FA0AD57449FA68134699
:1014F0005B0013449B000B4404334FF07C521A6092
:10150000B8680CF0F7FB5EA3D3E900230CF038F9C0
:1015100002460B46104619460CF0C0FB01466748D0
:10152000FA6813465B0013449B0003441960634947
:10153000FA6813465B0013449B000B44043393ED9D
:10154000007A5E49FA6813465B0013449B000B4423
:10155000D3ED007A77EE277A5849FA6813465B0094
:1015600013449B000B440433C3ED007A5349FA68DB
:1015700013465B0013449B000B440433D3ED007A05
:10158000B7EE007AF4EEC77AF1EE10FA17DD4B49A8
:10159000FA6813465B0013449B000B440433D3EDFD
:1015A000007AB7EE007A77EEC77A4449FA681346B4
:1015B0005B0013449B000B440433C3ED007A3F49A6
:1015C000FA6813465B0013449B000B440433D3EDCD
:1015D000007AF5EEC07AF1EE10FA17D53749FA68BD
:1015E00013465B0013449B000B440433D3ED007A95
:1015F000B7EE007A77EE877A3049FA6813465B00D7
:1016000013449B000B440433C3ED007A2B49FA6862
:1016100013465B0013449B000B440433D3ED007A64
:1016200077EEA77A17EE900A0CF064FB16A3D3E9C5
:1016300000230CF0A5F802460B46104619460CF0A4
:101640002DFB034600EE103A0EF0A7F8F0EE407ABC
:101650001A49FA6813465B0013449B000B44083395
:10166000C3ED007AFB680133FB60FB68052B7FF755
:10167000E1AEBFF34F8F00BF00BF1037BD46B0BD16
:10168000FCA9F1D24D62503F182D4454FB21094072
:10169000506A002000B00B40A8CD0120398EE338FD
:1016A0007458002000000020505A0020000000451F
:1016B00000E0FF4400F07F45BD378635746A0020A6
:1016C0002DE9F047F7EE007A2DED048BF4EE670A72
:1016D000F1EE10FA82B0F0EE608A1AD0B5EEC00AD0
:1016E000F1EE10FA33D8B5EE400AF1EE10FA15D14A
:1016F000F5EEC00AF1EE10FA00F2BD80944BF5EE63
:10170000400A2122F1EE10FA1A6000F01A819FEDD2
:10171000910A02B0BDEC048BBDE8F087FDEEE07AE3
:10172000B1EE400A17EE90AA0AF0010AF0EE007A34
:10173000F4EE678AF1EE10FA0CD1DFED877AB4EEA1
:10174000E70AF1EE10FA05D520EE000AE1E74FF0C6
:10175000000AEBE701A80BF07DFF10EE100A0CF079
:10176000C9FA79A3D3E900230F4606460EF04FFBD2
:10177000002814BF08240024784D04F1040805EB68
:10178000C80132463B46D1E900010EF06BFB002850
:1017900018BF444604F1020805EBC80132463B4637
:1017A000D1E900010EF05EFB002818BF444605EBAE
:1017B000C403D3E90289304642464B4639460CF011
:1017C0000BF90CF06BFA07EE900A32463B464046A6
:1017D000494637EEA78A0CF0D7F90CF05FFA07EE0E
:1017E000900A88EE279A0198C4EB00100138DFEDCB
:1017F0005C6ADFED5C7A29EE097AE7EE267A67EE1D
:10180000877A9FED597A67EE897AE7EE877AE9EE73
:10181000077AB0EE678A07EE900AFAEECE7A17EEF4
:10182000900A0CF067FA78EE097A064617EE900AED
:101830000F460CF05FFA02460B46304639460CF074
:10184000A3F9064618EE900A0F460CF053FA02462A
:101850000B46304639460BF093FF444B00220646B8
:101860000F460BF08DFF0EF087FA10F5006F05DACA
:10187000374B22221A609FED3E0A4AE707EE900A94
:101880000028B4BF00F10F040411F8EEE77AB4BFEA
:1018900024110134C0EB041817EE900A0CF02AFA58
:1018A000344B00220BF06CFF02460B4630463946A3
:1018B0000CF092F80CF0F2F99FED2F7ADFED2F6A21
:1018C00007EE900AE7EE876A05EBC8059FED2C7AD4
:1018D000A6EEA77ADFED2B6AE7EE276A9FED2A7A5C
:1018E000A6EEA77A67EE277A17EE900A0CF002FAB6
:1018F000264B00220CF048F9D5E900230BF040FFFD
:101900000CF0CCF900EE100A01A80BF0A3FE019830
:101910002044802809DD0E4B22221A60BAF1000F04
:101920007FF4F5AE9FED1A0AF3E610F17D0F9FDB11
:101930000BF0BAFEBAF1000F3FF4EBAEB1EE400A85
:10194000E7E6B0EE670AE4E6CD3B7F669EA0E63FA1
:10195000FCD00120000080FFA95F635880FF0000D9
:1019600000E84C3CAAAAAA3DEDA8E23E00003040A7
:10197000000000000000B03F1815AB3A4B8D1D3C35
:101980003758633DF0FD753E1872313F0000F03F5F
:101990000000807FFFFFFFFF2DE9F84355EC104B5F
:1019A00010EE100A0022002329460EF030FA78B11A
:1019B00000220023204629460EF0FEF920B1384BC4
:1019C000384D21221A60002445EC104BBDE8F88305
:1019D00040F2FE33C5F30A5763F31E5520462AA38F
:1019E000D3E9002329460BF0CBFE29A3D3E900233A
:1019F0000CF0CAF88046894602460B462046294626
:101A00000BF048FF42464B460CF0BEF8264B002236
:101A10000BF0B6FE8046894602460B462046294614
:101A20000BF038FF42464B460CF0AEF81E4B00223E
:101A30000BF0A6FE02460B46804689462046294604
:101A40000BF028FF42464B460CF09EF80022164B46
:101A50000BF096FEA7F2FE36F20704460D4609D5B6
:101A60000DA3D3E900230BF08BFE6FF47F730446C4
:101A70000D46FE18C5F30A5306EBD67603EB660651
:101A800066F31E55A0E700BF18096D3997E2E23FE3
:101A9000F7CC920035B5DA3FCD3B7F669EA0E63F9E
:101AA000FCD001200000F0FF0000E03FFFFFFFFF3F
:101AB000D0B5DFED3F7AF4EEE70AF1EE10FA2DED46
:101AC000028B10EE103A044609DB3A4B9FED3A8A3E
:101AD00021221A60B0EE480ABDEC028BD0BDDFEDCA
:101AE000377A9FED377A70EEA70AC0EE877AFDEE5F
:101AF000E77A17EE902AD207B8EEE78A48BF444249
:101B000019B1F6EE007A38EE678A18460CF0F2F852
:101B1000064618EE100A0F460CF0ECF822A3D3E9A3
:101B200000230BF02DFE02460B46304639460BF0E3
:101B300053FF0CF0B3F800EE100A08EE100A0DF097
:101B400024FEDFED207AB4EEE70AF1EE10FA23DB93
:101B500068EE087ADFED1C6A9FED1C7AA7EEA67A84
:101B6000DFED1B6AE7EE276A9FED1A7AA6EEA77AE9
:101B7000DFED196AE7EE276A9FED187AA6EEA77ADD
:101B8000DFED176AE7EE276A9FED167AA6EEA77AD1
:101B900067EE277AA8EE278A002CB8BFB1EE488AF4
:101BA00098E700BFAFF30080182D4454FB21094093
:101BB0000050C347FCD00120000080FFDB0FC93F6D
:101BC000DB0F4940FFE6DB2EFB074427072157AB1D
:101BD000E391302F2A32D7B21DEF3836010D50B9BC
:101BE0008988083CABAA2ABE80B582B000AF786075
:101BF00039603B68012B02D905480BF05FFB7B681D
:101C00003A68043253F8223018460837BD4680BD82
:101C10000800010080B52DED028B86B000AF87ED86
:101C2000050AC7ED040A87ED031AC7ED021A87ED0E
:101C3000012A97ED047AD7ED037AB4EEE77AF1EE54
:101C400010FA2AD597ED057AD7ED047A37EE678A30
:101C500097ED037AD7ED047A77EE677ADFED270AFE
:101C6000B0EE670A0CF099FAB0EE407AC8EE077A47
:101C7000B7EE001ADFED220AB0EE670A0CF0A9FAFF
:101C8000F0EE407AB0EE671AD7ED010A97ED020A3E
:101C90000CF065FAF0EE407A29E097ED057AD7ED81
:101CA000037A37EE678A97ED047AD7ED037A77EEF9
:101CB000677ADFED120AB0EE670A0CF06EFAB0EE4A
:101CC000407AC8EE077AB7EE001ADFED0D0AB0EEE3
:101CD000670A0CF07EFAF0EE407AB0EE671AD7EDA4
:101CE000020A97ED010A0CF03AFAF0EE407AB0EEF3
:101CF000670A1837BD46BDEC028B80BDBD378635FF
:101D00000000000080B52DED028B84B000AF78603C
:101D100087ED000A7B68D3ED037A97ED007A77EEC2
:101D2000677AC7ED037AD7ED037AF5EEC07AF1EE64
:101D300010FA26D57B6893ED027A7B68D3ED007AA2
:101D400037EE677AD7ED037A27EE278A7B6893ED23
:101D5000037A7B68D3ED007A77EE677ADFED310A9C
:101D6000B0EE670A0CF019FAF0EE407A88EE277AA6
:101D70007B68D3ED027A77EE277A7B68C3ED027A2F
:101D80002CE0D7ED037AF5EEC07AF1EE10FA25DDFE
:101D90007B6893ED017A7B68D3ED027A37EE677A40
:101DA000D7ED037A27EE278A7B6893ED017A7B686B
:101DB000D3ED037A77EE677ADFED1A0AB0EE670AA1
:101DC0000CF0EBF9F0EE407A88EE277A7B68D3EDE1
:101DD000027A77EE277A7B68C3ED027A7B68D3EDCF
:101DE000027A7B6893ED007A7B68D3ED016AB0EEEE
:101DF000661AF0EE470AB0EE670A0CF0EAF9F0EE68
:101E0000407A7B68C3ED027A7B683A68DA607B6867
:101E10009B6807EE903AB0EE670A1037BD46BDECFE
:101E2000028B80BDBD37863580B582B000AF1822E9
:101E300012493C2000F0AAFC72B600BF104805F021
:101E4000AFFE03F0B5F900237B6002E07B6801334D
:101E50007B607B680B4A9342F8DDFF2005F00EFFA4
:101E600003F0A6F900233B6002E03B6801333B60CE
:101E70003B68044A9342F8DDE0E700BF14580020B5
:101E80001C480020BFC62D0080B400AF034B0122C8
:101E90001A7000BFBD465DF8047B70470CD101206D
:101EA00080B400AF034B01221A7000BFBD465DF83D
:101EB000047B70470BD1012080B400AF034B01229B
:101EC0001A7000BFBD465DF8047B704708D1012041
:101ED00080B500AF094B186801230122084907F0BB
:101EE000A5FF0346002B01D0FFF79EFF0C220449FB
:101EF00004480DF065FC00BF80BD00BF2C580020D9
:101F000084790020BC6A002080B584B000AF78607E
:101F1000474B186801230022464907F087FF034614
:101F2000002B01D0FFF780FF424B1B68424A9342CF
:101F300002D17B68002B53D00C2200213F480DF0CA
:101F400041FC4FF4805200213D480DF03BFC3B4BDF
:101F500001221A60394B08225A60384B08229A60D5
:101F6000334B186801230122344908F003F8034673
:101F7000002B01D0FFF758FF0023BB6011E02C4B72
:101F80001868BB68DB0002331A4608232C4907F0A7
:101F9000F1FF0346002B01D0FFF746FFBB6801337A
:101FA000BB60BB681E2BEADD4FF4007200212148A4
:101FB0000DF008FC1F4B204A1A601E4B42F28E2285
:101FC0009A601C4B06225A60194B186801230022A4
:101FD000184907F0CFFF0346002B01D0FFF724FF7D
:101FE000144B1B68144A93421BD1124B9B6842F25C
:101FF0008E22934211D00F4B9B68FB600D4B9B6868
:1020000003F00F030E2B02D1FB681B1100E0FB68ED
:10201000FB60F8680CF083FA03E0064B1B68064A85
:102020009342FFF755FF00BF1037BD4680BD00BF8C
:102030002C580020847500204B45454EBC6A00207A
:10204000505A002080B582B000AF4C4B1B78DBB2F9
:10205000002B40D04A4B18684A4B1B69DB00023307
:102060001A460823484907F0E1FE0346002B01D039
:10207000FFF7DAFE72B600BF4FF480524249434880
:102080000DF09EFB4FF4F072414942480DF098FB71
:1020900000237B6012E07B681B013F4A1A443B49E6
:1020A0007B68FC339B000B44D3ED007AB0EE670AEB
:1020B00010460CF009FA7B6801337B607B68172BB4
:1020C000E9DD304B00229A602C4B00221A7004F09C
:1020D000AFFB62B600BF314B1B78DBB2002B2AD0BE
:1020E00000233B600EE02C4A3B681B01134408337D
:1020F0001A6826493B68FC339B000B441A603B6816
:1021000001333B603B68172BEDDD1D4B18681D4B01
:102110001B69DB0002331A4608231C4907F02AFF1B
:102120000346002B01D0FFF77FFE164B00229A607A
:102130001A4B00221A701A4B1B78DBB2002B19D0F5
:102140004FF40072002117480DF03CFB0C22164999
:1021500014480DF035FB0A4B186801230122114980
:1021600007F008FF0346002B01D0FFF75DFE0C4B84
:1021700000221A7000BF0837BD4680BD0CD1012077
:102180002C58002008000020847B0020505A00209A
:10219000605C00207C700020E86E00200BD10120E4
:1021A00008D1012084770020BC6A002080B500AFF0
:1021B0001C4B00221A701C4B00221A701B4B002271
:1021C0001A701B4B00221A701A4B00221A70002141
:1021D00019480CF088F9194B1868002305220021D2
:1021E0000BF02CF8154B1B68184608F05BF80346FB
:1021F000002B01D0FFF718FE104B1B68184607F0A4
:10220000ADFF0346002B01D0FFF70EFE0B4B1B6802
:10221000184607F0E7FD0346002B01D0FFF704FE48
:1022200000BF80BD08D1012009D101200AD10120C1
:102230000BD101200CD1012000D000402C580020EF
:1022400080B483B000AF0346FB71044AFB79D370BE
:1022500000BF0C37BD465DF8047B70470060064048
:1022600080B483B000AF0346FB71074B9B79DAB2B1
:102270000549FB791343DBB28B7100BF0C37BD46B8
:102280005DF8047B704700BF0060064080B400AF7B
:10229000064B9B79DBB2054A43F02003DBB2937116
:1022A00000BFBD465DF8047B704700BF006006407C
:1022B00080B400AF064B9B79DBB2054A23F02003C4
:1022C000DBB2937100BFBD465DF8047B704700BF71
:1022D0000060064080B500AF044B01221A70002256
:1022E000002103480CF0E6FC00BF80BD0FD10120A7
:1022F0000060064080B500AF02480CF00CFD00BF46
:1023000080BD00BF0060064080B500AF4AF2040205
:10231000002112480DF056FA4AF20402002110483A
:102320000DF050FA0F4B00221A700F4B00221A705A
:102330000E4B00221A700D4B00229A700B4B9B78AB
:10234000DBB20A4A63F03F03DBB29370FFF7B0FFE2
:10235000074B02221A7000BF80BD00BFA48B002073
:10236000A82B01200DD101200ED1012000600640D4
:102370000FD1012080B584B000AF584B03F5204346
:102380001A88564B03F5204302331B889A4205D026
:10239000534B1B78022B01D1FFF79CFF514B03F5E8
:1023A00020431A884F4B03F5204302331B889A427F
:1023B00000F090804B4B03F5204302331A88531CE6
:1023C00099B2484B03F52043023319801146454A20
:1023D0000B469B000B445B001A443B1D1068516880
:1023E00003C312891A803F4B03F5204302331B8835
:1023F000C3F30B039AB23B4B03F5204302331A801D
:102400007B79042B5FD13B7A013B162B5DD801A26F
:1024100052F823F0712400008D240000CB2400002A
:10242000CB240000CB240000CB240000CB240000F0
:10243000CB240000CB240000CB240000CB240000E0
:10244000CB240000CB240000CB240000CB240000D0
:10245000CB240000CB240000CB240000CB240000C0
:10246000B7240000CB240000A9240000BF240000F2
:102470001D4B5B68002B2AD07B7A1E2B27D87B7ADA
:102480001A46194B1A61FFF7FFFC20E0164B5B68F8
:10249000002B1ED07B7A1E2B1BD87B7A1A46124B40
:1024A0001A61FFF7FDFC14E00F4B01221A600E4B7E
:1024B00001225A600EE00C4B01221A600AE00A4B1E
:1024C00000225A6006E000BF04E000BF02E000BF47
:1024D00000E000BF00BF1037BD4680BDA82B012023
:1024E0000FD10120A48B00200800002080B582B00D
:1024F00000AF6E4B1B78012B49D16D4B0222DA7075
:102500006C4B1B78DBB2062B23D1FFF7F3FE6A4B33
:1025100003F5204302331B8801339AB2664B03F55F
:10252000204302331A80644B03F5204302331B8897
:10253000C3F30B039AB2604B03F5204302331A80B6
:102540005A4B02221A705B4B00221A70584B002221
:102550001A71584B1B78DBB2052B00F2A080564B4A
:1025600003F5204302331B881A4613469B0013448D
:102570005B00514A1A444F4B1B78DBB2591CC8B25E
:102580004C49087013444A4A1B78137187E0484B42
:10259000DB78DBB23B603B6803F01003002B0ED00E
:1025A0001020FFF74DFE3B6803F04003002B06D1DF
:1025B0005020FFF755FE0220FFF742FE72E03C4B31
:1025C0009B79FB713B6803F04003002B1BD03B4B16
:1025D00000221A70FFF75AFE354BC0229A70344B16
:1025E000364A1278D2B21B79D9B2354B99542F4B57
:1025F00003221A705020FFF733FE4220FFF720FE1F
:102600002B4B9B79FB71FB7903F05003002B34D0EB
:102610005020FFF725FEFFF74BFE254BC8229A708E
:102620000220FFF70DFE274B03F520431B885A1CA1
:1026300091B2244A02F5204211801A4613469B00AB
:1026400013445B001F4A13440A221D4918460DF02B
:10265000B7F81C4B03F520431B88C3F30B039AB256
:10266000184B03F520431A802022002114480DF056
:10267000A9F80E4B02221A7014E00D4A0F4B1B787A
:10268000DBB2591CC8B20D49087019461379DAB289
:102690000B4B5A5445F2020105480BF0DBFCBFF32B
:1026A0004F8F00BF0837BD4680BD00BF0FD101204E
:1026B000006006400DD10120A82B01200ED1012081
:1026C000848B0020A48B002080B400AF0B4B9B6850
:1026D000002B0ED1094B1B68002B07D0074B5B6802
:1026E000002B06D0054B01229A6002E0034B012229
:1026F0009A6000BFBD465DF8047B7047080000206B
:1027000080B5ADF5047D00AF3B1D18603B461960F8
:1027100007F1100340221A6004334FF4FE720021C7
:1027200018460DF04FF83A463B1D07F11001481CC2
:10273000126819680DF044F800223C2112480CF090
:10274000B9FA07F10F0301221A7000E000BF07F188
:102750000F031B78DBB25A1CD1B207F10F021170C4
:10276000002BF3D13B461B685A1C07F110010023D4
:1027700005480CF021FB04480CF0CDFA00BF07F52A
:102780000477BD4680BD00BF00600E4080B586B0B6
:1027900000AF0346B9607A60FB73FB7B00221946E9
:1027A0000D480CF087FA0123FB7500E000BFFB7DAC
:1027B000DBB25A1CD2B2FA75002BF7D100237A682B
:1027C000B96805480CF0F8FA03480CF0A4FA00BF09
:1027D0001837BD4680BD00BF00600E4080B582B096
:1027E00000AF0022032112480BF0D8FB0122122176
:1027F0000F480BF0D3FB012213210D480BF0CEFB49
:1028000000237B6008E07B680022194608480BF033
:10281000C5FB7B6801337B607B68022BF3D9054ADB
:102820000021054807F020FF00BF0837BD4680BDE6
:1028300040F00F406C58002000B00340B0B582B0AB
:1028400000AF994B5B68984A1360974B9B68002BCD
:1028500005DD954B9B68013B934A93601DE01A216F
:1028600092480BF0B8FB0346002B0CBF012300235A
:10287000DBB21A468C4B5A608B4B1A688A4B5B68EA
:102880009A420AD0884B5B68002B03D0884B1B68A8
:10289000854AD360844B04229A60834B5B69824AE9
:1028A0001361814B9B69002B05DD7F4B9B69013BCD
:1028B0007D4A93611FE005217E480BF08CFB0346A7
:1028C000002B0CBF01230023DBB21A46764B5A6162
:1028D000754B1A69744B5B699A420CD005F0ECF9A0
:1028E000714B5B69002B03D0714B1B686E4AD3613F
:1028F0006D4B04229A616C4B5B6A6B4A13626A4BA4
:102900009B6A002B05DD684B9B6A013B664A93621C
:102910001FE00E2167480BF05EFB0346002B0CBF47
:1029200001230023DBB21A465F4B5A625E4B1A6AE0
:102930005D4B5B6A9A420CD005F0BEF95A4B5B6A5C
:10294000002B03D05A4B1B68574AD362564B0422C4
:102950009A62554B5B6B544A1363534B9B6B002B32
:1029600005DD514B9B6B013B4F4A93631FE00121F7
:1029700051480BF030FB0346002B0CBF0123002312
:10298000DBB21A46484B5A63474B1A6B464B5B6B9C
:102990009A420CD005F090F9434B5B6B002B03D0AF
:1029A000434B1B68404AD3633F4B04229A633E4B20
:1029B0005B68012B1BD13E4B1A683B4BDB68D31A7B
:1029C000B3F5FA7F13D93D4B1B68002B0FD03C4B5E
:1029D0001B68002B06D03A4B5B68C3F10103384AF1
:1029E000536001E0FFF75CFA344B00221A602E4B73
:1029F0001B68012B0CD12C4B5B68002B08D12F4B93
:102A00001B68002B01D005F057F92C4B01221A60EE
:102A10002C4B1B78DBB2032B00F2768201A252F81A
:102A200023F000BFC92A0000352A0000EB2E000069
:102A30008D2A00001C4B1B6B002B09D11A4B5B6BC2
:102A4000012B05D1FFF738FA1E4B00221A705BE20A
:102A5000154B1B69002B0AD1134B5B69012B06D167
:102A6000174BDB68C3F10103154AD3604CE20E4BF0
:102A70005B68002B40F04182104B1B68002B01D09B
:102A800005F01AF90D4B01221A6036E2064B1B6B5A
:102A9000002B40F03482044B5B6B012B40F02F8203
:102AA000084B00221A702FE2BCCB012000F10F402E
:102AB0007470002000F00F40C0F00F403458002028
:102AC0000800002010D10120A04B5B6B012B4BD1E3
:102AD0009E4B1B69002B07D19C4B5B69012B03D1DB
:102AE0009B4B01221A700FE2984B1B6A002B07D1F7
:102AF000964B5B6A012B03D1954B03221A7003E2BC
:102B0000924B1B68002B40F08480904B5B68012B3C
:102B10007FD105F0D1F88F4B00221A6000237B6033
:102B20001EE0FFF7D1FD8C4B1A688C4913465B0001
:102B30001344DB007A6813440C33002241F823204D
:102B4000854B1A68854913465B001344DB007A689D
:102B500013448433002241F823207B6801337B60D7
:102B60007B68172BDDDD54E0784B5B6A012B50D17D
:102B70007B4B1A68754BDB6AD31AB3F5FA7F48D3DF
:102B8000784B1B68002B44D0774B1B68002B00DA76
:102B900003339B101A46714B53F82230002B0CBFA5
:102BA00001230023D9B2704B1B68002B00DA0333DA
:102BB0009B101A46694B43F822106B4B1B68002B85
:102BC00000DA03339B103B6016E0FFF77DFD3B68A6
:102BD0001B01664A1A4466493B682C2000FB03F33C
:102BE0000B441433D3ED007AB0EE670A10460BF0B5
:102BF0006BFC3B6801333B605B4B1B68002B00DACE
:102C000003339B1003333A689A42DEDD554B0022B2
:102C10001A604E4B1B69012B40F00E814B4B5B69D8
:102C2000002B40F009814C4B1A684F4B19684B48F8
:102C300013465B001344DB000B440C3350F8233085
:102C4000002B00F0F980FFF73FFD434B1A68464B1D
:102C50001968424813465B001344DB000B4484337D
:102C600050F82330632B0FD13B4B1A683E4B196849
:102C70003A4813465B001344DB000B4484336FF087
:102C8000620240F82320D7E0334B1A68364B1968AC
:102C9000324813465B001344DB000B44843350F886
:102CA0002330002B68DA2C4B1A682F4B19683148F7
:102CB00013465B001344DB000B4450F82330002B19
:102CC00034DA254B1A68284B19682A4813465B00EA
:102CD0001344DB000B4450F823101F4B1A68224B9F
:102CE00018681E4C13465B001344DB000344843316
:102CF00054F82330994219DD174B19681A4B1C6898
:102D0000154B1A68184B18681A4D0B465B000B449C
:102D1000DB00234455F82310104C13465B0013448A
:102D2000DB000344843344F8231085E00A4B1A681F
:102D30000D4B1968094813465B001344DB000B4434
:102D40008433002240F8232076E000BFBCCB012072
:102D500010D101203458002068700020505A002003
:102D600074700020385800206C700020E86E00203D
:102D7000C86A00207C700020654B1A68654B196892
:102D8000654813465B001344DB000B44843350F862
:102D90002330002B50DB5E4B1A685E4B19685F488E
:102DA00013465B001344DB000B4450F82330002B28
:102DB00034DD574B1A68574B1968584813465B0067
:102DC0001344DB000B4450F82310514B1A68514B4D
:102DD0001868514C13465B001344DB0003448433F2
:102DE00054F82330994219DD494B1968494B1C6846
:102DF000474B1A68474B1868484D0B465B000B441D
:102E0000DB00234455F82310434C13465B00134466
:102E1000DB000344843344F823100DE03C4B1A6874
:102E20003C4B19683C4813465B001344DB000B44E1
:102E30008433632240F82320394B1B6A012B60D175
:102E4000374B5B6A002B5CD1364B1A68344BDB6A1C
:102E5000D31AB3F5FA7F44D2334B1B68002B04D14D
:102E6000314B40F2DC521A603BE0FFF72DFC284B5F
:102E70001A68284B1968284813465B001344DB0086
:102E80000B440C3350F82330002B1CD0204B1A6815
:102E9000204B1968204813465B001344DB000B44A9
:102EA0000C33002240F82320194B1A68194B19687B
:102EB000194813465B001344DB000B4484330022A3
:102EC00040F823200DE0124B1A68124B1968124883
:102ED00013465B001344DB000B440C33012240F823
:102EE0002320124B01221A600EE00D4B5B69002B70
:102EF00009D10F4B00221A7005E000BF04E000BFAB
:102F000002E000BF00E000BF0837BD46B0BD00BF13
:102F1000687000206C700020505A00207C700020E7
:102F2000BCCB012074700020FCCB0120385800205D
:102F300010D1012080B582B000AF0023BB80284AA9
:102F40003B461268114619800233120C1A70254B49
:102F50005A68254B1B689A4225D0224B5B68002B90
:102F60000BDD204B5B68013BDBB21A4692001A4432
:102F7000520013445B00DBB20AE01A4B5B68DB4390
:102F8000DBB21A4692001A44520013445B00DBB2D3
:102F9000BB703B46032219463C20FFF7F7FB114B61
:102FA0005B68114A13600F4B5B68002B07DAA7239D
:102FB0007B713B1D022219463C20FFF7E7FB094BC2
:102FC0005B68002B07DDA6237B713B1D022219469F
:102FD0003C20FFF7DBFB00BF0837BD4680BD00BFCC
:102FE00020010100BC6A002070CC012080B584B0B3
:102FF00000AFC54B1B78DBB2002B41F04781C34BC0
:103000001B68042B00F2908001A252F823F000BF4D
:1030100025300000593000008D300000C130000024
:10302000F530000001220021B9480AF0B7FF002264
:103030000F21B8480AF0B2FF00221021B5480AF06B
:10304000ADFF00220521B2480AF0A8FF00220621A8
:10305000AF480AF0A3FF67E000220021AC480AF065
:103060009DFF01220F21AB480AF098FF002210219A
:10307000A8480AF093FF00220521A5480AF08EFF18
:1030800000220621A2480AF089FF4DE0002200211B
:103090009F480AF083FF00220F219E480AF07EFF1E
:1030A000012210219B480AF079FF0022052198484F
:1030B0000AF074FF0022062195480AF06FFF33E002
:1030C0000022002192480AF069FF00220F21914856
:1030D0000AF064FF002210218E480AF05FFF0122EF
:1030E00005218B480AF05AFF0022062188480AF081
:1030F00055FF19E00022002185480AF04FFF002209
:103100000F2184480AF04AFF0022102181480AF06A
:1031100045FF002205217E480AF040FF01220621DA
:103120007B480AF03BFF00BF0822FF217A480CF0E1
:1031300049FB0023FB6001F0A5B8FB68172B01F2E7
:103140009E8001A252F823F0A931000059320000FC
:103150002D330000DD3300008D3400003D350000CC
:1031600005360000B5360000653700001538000050
:10317000DD3800008D3900003D3A0000E53A0000DE
:10318000A53B00004D3C0000F53C00009D3D0000CB
:103190005D3E0000053F0000AD3F000055400000CF
:1031A00015410000BD410000584B1A685B491346A9
:1031B0005B001344DB00FA6813440C3351F82330EE
:1031C000002B28D0564B1B68FA689A4217D1554BF2
:1031D0001B6803F00103D9B24F4A937961F3C3032B
:1031E0009371504B1B68002B0CBF01230023D9B2F5
:1031F000494A937961F38203937101F040B8464ADA
:10320000937943F008039371434A93796FF38203F0
:10321000937101F034B8424B1B68FA689A420FD19F
:10322000414B1B68002B0BD03B4A93796FF3C303D0
:103230009371394A937943F00403937101F01FB8F5
:10324000354A937943F008039371334A937943F0F5
:103250000403937101F013B82C4B1A682F491346DD
:103260005B001344DB00FA6813440C3351F823303D
:10327000002B28D02A4B1B68FA689A4217D1294B99
:103280001B6803F00103D9B2234A537961F3C713D2
:103290005371244B1B68002B0CBF01230023D9B2B0
:1032A0001D4A537961F38613537100F0E8BF1A4A3F
:1032B000537943F080035371174A53796FF38613A0
:1032C000537100F0DCBF164B1B68FA689A420FD1AD
:1032D000154B1B68002B0BD00F4A53796FF3C713A4
:1032E00053710D4A537943F04003537100F0C7BF47
:1032F000094A537943F080035371074A537943F0E5
:103300004003537100F0BBBF10D101206870002052
:10331000C0F00F4000F00F40E8720020505A00202B
:103320006C70002078700020FCCB0120AF4B1A6835
:10333000AF4913465B001344DB00FA6813440C33B7
:1033400051F82330002B28D0AA4B1B68FA689A4208
:1033500017D1A94B1B6803F00103D9B2A74A5379CF
:1033600061F341035371A44B1B68002B0CBF012375
:103370000023D9B2A14A537961F30003537100F0DD
:103380007EBF9E4A537943F0020353719B4A53799F
:103390006FF30003537100F072BF964B1B68FA681D
:1033A0009A420FD1964B1B68002B0BD0934A53794E
:1033B0006FF341035371914A537943F00103537101
:1033C00000F05DBF8D4A537943F0020353718B4A7D
:1033D000537943F00103537100F051BF834B1A68D6
:1033E000834913465B001344DB00FA6813440C3333
:1033F00051F82330002B28D07E4B1B68FA689A4284
:1034000017D17D4B1B6803F00103D9B27B4A937936
:1034100061F3C7139371784B1B68002B0CBF01231A
:103420000023D9B2754A937961F38613937100F042
:1034300026BF724A937943F0800393716F4A937960
:103440006FF38613937100F01ABF6A4B1B68FA681A
:103450009A420FD16A4B1B68002B0BD0674A9379B5
:103460006FF3C7139371654A937943F040039371E7
:1034700000F005BF614A937943F0800393715F4A7E
:10348000937943F04003937100F0F9BE574B1A68EB
:10349000574913465B001344DB00FA6813440C33AE
:1034A00051F82330002B28D0524B1B68FA689A42FF
:1034B00017D1514B1B6803F00103D9B24F4A9379DE
:1034C00061F3410393714C4B1B68002B0CBF01232C
:1034D0000023D9B2494A937961F30003937100F054
:1034E000CEBE464A937943F002039371434A9379DF
:1034F0006FF30003937100F0C2BE3E4B1B68FA6885
:103500009A420FD13E4B1B68002B0BD03B4A93795C
:103510006FF341039371394A937943F00103937137
:1035200000F0ADBE354A937943F002039371334AFC
:10353000937943F00103937100F0A1BE2B4B1A68FD
:103540002B4913465B001344DB00FA6813440C3329
:1035500051F82330002B28D0264B1B68FA689A427A
:1035600017D1254B1B6803F00103D9B2234A5379C5
:1035700061F345135371204B1B68002B0CBF0123D3
:103580000023D9B21D4A537961F30413537100F03B
:1035900076BE1A4A537943F020035371174A537980
:1035A0006FF30413537100F06ABE124B1B68FA6884
:1035B0009A420FD1124B1B68002B0BD00F4A537944
:1035C0006FF3451353710D4A537943F01003537150
:1035D00000F055BE094A537943F020035371074A5E
:1035E000537943F01003537100F049BE6870002016
:1035F000505A00206C70002078700020E872002083
:10360000FCCB0120AF4B1A68AF4913465B00134453
:10361000DB00FA6813440C3351F82330002B28D018
:10362000AA4B1B68FA689A4217D1A94B1B6803F092
:103630000103D9B2A74A537961F3C3035371A44B71
:103640001B68002B0CBF01230023D9B2A14A537978
:1036500061F38203537100F012BE9E4A537943F026
:10366000080353719B4A53796FF38203537100F03F
:1036700006BE964B1B68FA689A420FD1964B1B68A0
:10368000002B0BD0934A53796FF3C3035371914AC4
:10369000537943F00403537100F0F1BD8D4A53791F
:1036A00043F0080353718B4A537943F00403537179
:1036B00000F0E5BD834B1A68834913465B00134451
:1036C000DB00FA6813440C3351F82330002B28D068
:1036D0007E4B1B68FA689A4217D17D4B1B6803F03A
:1036E0000103D9B27B4A937961F345139371784B07
:1036F0001B68002B0CBF01230023D9B2754A9379B4
:1037000061F30413937100F0BABD724A937943F0E8
:10371000200393716F4A93796FF30413937100F050
:10372000AEBD6A4B1B68FA689A420FD16A4B1B68A0
:10373000002B0BD0674A93796FF345139371654A59
:10374000937943F01003937100F099BD614A937926
:1037500043F0200393715F4A937943F01003937110
:1037600000F08DBD574B1A68574913465B00134450
:10377000DB00FA6813440C3351F82330002B28D0B7
:10378000524B1B68FA689A4217D1514B1B6803F0E1
:103790000103D9B24F4AD37861F3C713D3704C4BAE
:1037A0001B68002B0CBF01230023D9B2494AD378F0
:1037B00061F38613D37000F062BD464AD37843F0BC
:1037C0008003D370434AD3786FF38613D37000F02D
:1037D00056BD3E4B1B68FA689A420FD13E4B1B68A0
:1037E000002B0BD03B4AD3786FF3C713D370394A01
:1037F000D37843F04003D37000F041BD354AD3780D
:1038000043F08003D370334AD37843F04003D3703E
:1038100000F035BD2B4B1A682B4913465B0013444F
:10382000DB00FA6813440C3351F82330002B28D006
:10383000264B1B68FA689A4217D1254B1B6803F088
:103840000103D9B2234AD37961F30003D371204B2A
:103850001B68002B0CBF01230023D9B21D4AD3796A
:1038600061F34103D37100F00ABD1A4AD37943F0E2
:103870000103D371174AD3796FF34103D37100F079
:10388000FEBC124B1B68FA689A420FD1124B1B68A0
:10389000002B0BD00F4AD3796FF30003D3710D4A7D
:1038A000D37943F00203D37100F0E9BC094AD3791C
:1038B00043F00103D371074AD37943F00203D37174
:1038C00000F0DDBC68700020505A00206C700020B1
:1038D00078700020E8720020FCCB0120AB4B1A6806
:1038E000AB4913465B001344DB00FA6813440C3306
:1038F00051F82330002B28D0A64B1B68FA689A4257
:1039000017D1A54B1B6803F00103D9B2A34A137961
:1039100061F304131371A04B1B68002B0CBF012330
:103920000023D9B29D4A137961F34513137100F056
:10393000A6BC9A4A137943F010031371974A13797E
:103940006FF34513137100F09ABC924B1B68FA6831
:103950009A420FD1924B1B68002B0BD08F4A1379E0
:103960006FF3041313718D4A137943F0200313711D
:1039700000F085BC894A137943F010031371874A1C
:10398000137943F02003137100F079BC7F4B1A6860
:103990007F4913465B001344DB00FA6813440C3381
:1039A00051F82330002B28D07A4B1B68FA689A42D2
:1039B00017D1794B1B6803F00103D9B2774A93788A
:1039C00061F3C7139370744B1B68002B0CBF01236A
:1039D0000023D9B2714A937861F38613937000F093
:1039E0004EBC6E4A937843F0800393706B4A937891
:1039F0006FF38613937000F042BC664B1B68FA6845
:103A00009A420FD1664B1B68002B0BD0634A937808
:103A10006FF3C7139370614A937843F04003937038
:103A200000F02DBC5D4A937843F0800393705B4AAD
:103A3000937843F04003937000F021BC534B1A6815
:103A4000534913465B001344DB00FA6813440C33FC
:103A500051F82330002B26D04E4B1B68FA689A424F
:103A600016D14D4B1B6803F00103D9B24B4AD378F2
:103A700061F34513D370484B1B68002B0CBF012327
:103A80000023D9B2454AD37861F30413D370F6E327
:103A9000424AD37843F02003D370404AD3786FF37F
:103AA0000413D370EBE33B4B1B68FA689A420ED1C8
:103AB0003B4B1B68002B0AD0384AD3786FF3451371
:103AC000D370364AD37843F01003D370D7E3334A28
:103AD000D37843F02003D370304AD37843F01003F7
:103AE000D370CCE3294B1A68294913465B00134471
:103AF000DB00FA6813440C3351F82330002B26D036
:103B0000244B1B68FA689A4216D1234B1B6803F0BA
:103B10000103D9B2214AD37961F38203D3711E4BD9
:103B20001B68002B0CBF01230023D9B21B4AD37999
:103B300061F3C303D371A2E3184AD37943F00403BA
:103B4000D371164AD3796FF3C303D37197E3114B43
:103B50001B68FA689A420ED1114B1B68002B0AD0E1
:103B60000E4AD3796FF38203D3710C4AD37943F0B1
:103B70000803D37183E3094AD37943F00403D37173
:103B8000064AD37943F00803D37178E368700020C4
:103B9000505A00206C70002078700020E8720020DD
:103BA000FCCB0120A74B1A68A74913465B001344BE
:103BB000DB00FA6813440C3351F82330002B26D075
:103BC000A24B1B68FA689A4216D1A14B1B6803F0FE
:103BD0000103D9B29F4A137961F3861313719C4B89
:103BE0001B68002B0CBF01230023D9B2994A13791B
:103BF00061F3C713137142E3964A137943F040030C
:103C00001371944A13796FF3C713137137E38F4B12
:103C10001B68FA689A420ED18F4B1B68002B0AD0A2
:103C20008C4A13796FF3861313718A4A137943F020
:103C30008003137123E3874A137943F04003137120
:103C4000844A137943F08003137118E37D4B1A689B
:103C50007D4913465B001344DB00FA6813440C33C0
:103C600051F82330002B26D0784B1B68FA689A4213
:103C700016D1774B1B6803F00103D9B2754A9378CC
:103C800061F345139370724B1B68002B0CBF01232B
:103C90000023D9B26F4A937861F304139370EEE274
:103CA0006C4A937843F0200393706A4A93786FF3D9
:103CB00004139370E3E2654B1B68FA689A420ED1D5
:103CC000654B1B68002B0AD0624A93786FF345134B
:103CD0009370604A937843F010039370CFE25D4A8B
:103CE000937843F0200393705A4A937843F010037B
:103CF0009370C4E2534B1A68534913465B00134454
:103D0000DB00FA6813440C3351F82330002B26D023
:103D10004E4B1B68FA689A4216D14D4B1B6803F054
:103D20000103D9B24B4AD37861F3C303D370484B34
:103D30001B68002B0CBF01230023D9B2454AD3785E
:103D400061F38203D3709AE2424AD37843F00803C6
:103D5000D370404AD3786FF38203D3708FE23B4B2A
:103D60001B68FA689A420ED13B4B1B68002B0AD0A5
:103D7000384AD3786FF3C303D370364AD37843F00D
:103D80000403D3707BE2334AD37843F00803D37043
:103D9000304AD37843F00403D37070E2294B1A6899
:103DA000294913465B001344DB00FA6813440C33C3
:103DB00051F82330002B26D0244B1B68FA689A4216
:103DC00016D1234B1B6803F00103D9B2214AD379E2
:103DD00061F30413D3711E4B1B68002B0CBF01232E
:103DE0000023D9B21B4AD37961F34513D37146E25C
:103DF000184AD37943F01003D371164AD3796FF37D
:103E00004513D3713BE2114B1B68FA689A420ED1FD
:103E1000114B1B68002B0AD00E4AD3796FF30413A1
:103E2000D3710C4AD37943F02003D37127E2094AB6
:103E3000D37943F01003D371064AD37943F02003BA
:103E4000D3711CE268700020505A00206C70002072
:103E500078700020E8720020FCCB0120A74B1A6884
:103E6000A74913465B001344DB00FA6813440C3384
:103E700051F82330002B26D0A24B1B68FA689A42D7
:103E800016D1A14B1B6803F00103D9B29F4A1379E5
:103E900061F3C30313719C4B1B68002B0CBF012300
:103EA0000023D9B2994A137961F382031371E6E1D1
:103EB000964A137943F008031371944A13796FF308
:103EC00082031371DBE18F4B1B68FA689A420ED1B3
:103ED0008F4B1B68002B0AD08C4A13796FF3C303F6
:103EE00013718A4A137943F004031371C7E1874AB7
:103EF000137943F008031371844A137943F00403E0
:103F00001371BCE17D4B1A687D4913465B00134475
:103F1000DB00FA6813440C3351F82330002B26D011
:103F2000784B1B68FA689A4216D1774B1B6803F0EE
:103F30000103D9B2754A937861F300039370724B11
:103F40001B68002B0CBF01230023D9B26F4A937862
:103F500061F34103937092E16C4A937843F001035B
:103F600093706A4A93786FF34103937087E1654BCE
:103F70001B68FA689A420ED1654B1B68002B0AD069
:103F8000624A93786FF300039370604A937843F02A
:103F90000203937073E15D4A937843F001039370D9
:103FA0005A4A937843F00203937068E1534B1A68BE
:103FB000534913465B001344DB00FA6813440C3387
:103FC00051F82330002B26D04E4B1B68FA689A42DA
:103FD00016D14D4B1B6803F00103D9B24B4AD3787D
:103FE00061F34103D370484B1B68002B0CBF0123C6
:103FF0000023D9B2454AD37861F30003D3703EE180
:10400000424AD37843F00203D370404AD3786FF327
:104010000003D37033E13B4B1B68FA689A420ED120
:104020003B4B1B68002B0AD0384AD3786FF341030F
:10403000D370364AD37843F00103D3701FE1334A7B
:10404000D37843F00203D370304AD37843F00103AE
:10405000D37014E1294B1A68294913465B001344B5
:10406000DB00FA6813440C3351F82330002B26D0C0
:10407000244B1B68FA689A4216D1234B1B6803F045
:104080000103D9B2214AD37961F38613D3711E4B50
:104090001B68002B0CBF01230023D9B21B4AD37924
:1040A00061F3C713D371EAE0184AD37943F04003B0
:1040B000D371164AD3796FF3C713D371DFE0114B75
:1040C0001B68FA689A420ED1114B1B68002B0AD06C
:1040D0000E4AD3796FF38613D3710C4AD37943F028
:1040E0008003D371CBE0094AD37943F04003D37105
:1040F000064AD37943F08003D371C0E06870002092
:10410000505A00206C70002078700020E872002067
:10411000FCCB01204E4B1A684E4913465B001344FA
:10412000DB00FA6813440C3351F82330002B26D0FF
:10413000494B1B68FA689A4216D1484B1B6803F03A
:104140000103D9B2464A137961F300031371434B5B
:104150001B68002B0CBF01230023D9B2404A1379FE
:1041600061F3410313718AE03D4A137943F001037F
:1041700013713B4A13796FF3410313717FE0364BA0
:104180001B68FA689A420ED1364B1B68002B0AD086
:10419000334A13796FF300031371314A137943F0F3
:1041A000020313716BE02E4A137943F0010313717C
:1041B0002B4A137943F00203137160E0244B1A6811
:1041C000244913465B001344DB00FA6813440C33A4
:1041D00051F82330002B26D01F4B1B68FA689A42F7
:1041E00016D11E4B1B6803F00103D9B21C4A937809
:1041F00061F382039370194B1B68002B0CBF0123E2
:104200000023D9B2164A937861F3C303937035E063
:10421000134A937843F004039370114A93786FF331
:10422000C30393702AE00C4B1B68FA689A421BD1B7
:104230000C4B1B68002B17D0094A93786FF382034D
:104240009370074A937843F00803937016E000BF19
:1042500068700020505A00206C7000207870002098
:10426000E8720020FCCB0120964A937843F00403C7
:104270009370944A937843F00803937000BFFB68EF
:104280000133FB60FB68172B7EF757AF8E4B1B7813
:10429000DBB2032B40F01B86002200218B4809F083
:1042A0007DFE00220F218A4809F078FE00221021AD
:1042B000874809F073FE00220521844809F06EFE4C
:1042C00000220621814809F069FE824B1B68032BFE
:1042D00000F3028100237B498A7963F386128A7195
:1042E00078498A7963F3C7128A7176494A7963F308
:1042F00000024A7173494A7963F341024A71714974
:104300004A7963F386124A716E494A7963F3C71298
:104310004A716C498A7963F382028A7169498A79A0
:1043200063F3C3028A71012366498A7963F3041235
:104330008A7164498A7963F345128A7161494A79BD
:1043400063F382024A715F494A7963F3C3024A7197
:104350005C494A7963F304124A715A494A7963F312
:1043600045124A7157498A7963F300028A715549A7
:104370008A7963F341028A71012352498A7863F38F
:1043800086128A704F498A7863F3C7128A704D4942
:104390000A7963F345120A714A490A7963F30412F0
:1043A0000A714849CA7963F34102CA714549CA7919
:1043B00063F30002CA714349CA7863F38612CA7074
:1043C0004049CA7863F3C712CA7001233D498A780D
:1043D00063F304128A703B498A7863F345128A704A
:1043E00038490A7963F3C7120A7136490A7963F3C7
:1043F00086120A713349CA7963F3C302CA7131491B
:10440000CA7963F38202CA712E49CA7863F304122F
:10441000CA702C49CA7863F34512CA70012329492E
:104420008A7863F341028A7026498A7863F300022E
:104430008A7024490A7963F382020A7121490A7950
:1044400063F3C3020A711F49CA7963F34512CA7143
:104450001C49CA7963F30412CA711A49CA7863F312
:104460008202CA701749CA7863F3C302CA70012373
:1044700014498A7863F3C3028A7012498A7863F315
:1044800082028A700F490A7963F341020A710D4969
:104490000A7963F300020A710A49CA7963F3C71201
:1044A000CA710849CA7963F38612CA710549CA7884
:1044B00063F30002CA700349CA7863F34102CA7009
:1044C00000F005BDE872002010D10120C0F00F40BF
:1044D00000F00F406C7000207D4B1B68072B00F331
:1044E000FB8001237B498A7963F386128A717949BB
:1044F0008A7963F3C7128A7176494A7963F30002B5
:104500004A7174494A7963F341024A7171494A799F
:1045100063F386124A716F494A7963F3C7124A718D
:104520006C498A7963F382028A716A498A7963F3F2
:10453000C3028A71002367498A7963F304128A717E
:1045400064498A7963F345128A7162494A7963F34F
:1045500082024A715F494A7963F3C3024A715D4935
:104560004A7963F304124A715A494A7963F345124E
:104570004A7158498A7963F300028A7155498A79E8
:1045800063F341028A71012352498A7863F38612E8
:104590008A7050498A7863F3C7128A704D490A7944
:1045A00063F345120A714B490A7963F304120A71E5
:1045B0004849CA7963F34102CA714649CA7963F32B
:1045C0000002CA714349CA7863F38612CA7041492E
:1045D000CA7863F3C712CA7001233E498A7863F32D
:1045E00004128A703B498A7863F345128A7039490C
:1045F0000A7963F3C7120A7136490A7963F386129E
:104600000A713449CA7963F3C302CA713149CA795C
:1046100063F38202CA712F49CA7863F30412CA7025
:104620002C49CA7863F34512CA70012329498A7854
:1046300063F341028A7027498A7863F300028A7023
:1046400024490A7963F382020A7122490A7963F3E1
:10465000C3020A711F49CA7963F34512CA711D4921
:10466000CA7963F30412CA711A49CA7863F38202E1
:10467000CA701849CA7863F3C302CA700123154986
:104680008A7863F3C3028A7012498A7863F38202DC
:104690008A7010490A7963F341020A710D490A7957
:1046A00063F300020A710B49CA7963F3C712CA7136
:1046B0000849CA7963F38612CA710649CA7863F356
:1046C0000002CA700349CA7863F34102CA70FEE36C
:1046D0006C700020E87200207D4B1B680B2B00F3F0
:1046E000FB8001237B498A7963F386128A717949B9
:1046F0008A7963F3C7128A7176494A7963F30002B3
:104700004A7174494A7963F341024A7171494A799D
:1047100063F386124A716F494A7963F3C7124A718B
:104720006C498A7963F382028A716A498A7963F3F0
:10473000C3028A71012367498A7963F304128A717B
:1047400064498A7963F345128A7162494A7963F34D
:1047500082024A715F494A7963F3C3024A715D4933
:104760004A7963F304124A715A494A7963F345124C
:104770004A7158498A7963F300028A7155498A79E6
:1047800063F341028A71002352498A7863F38612E7
:104790008A7050498A7863F3C7128A704D490A7942
:1047A00063F345120A714B490A7963F304120A71E3
:1047B0004849CA7963F34102CA714649CA7963F329
:1047C0000002CA714349CA7863F38612CA7041492C
:1047D000CA7863F3C712CA7001233E498A7863F32B
:1047E00004128A703B498A7863F345128A7039490A
:1047F0000A7963F3C7120A7136490A7963F386129C
:104800000A713449CA7963F3C302CA713149CA795A
:1048100063F38202CA712F49CA7863F30412CA7023
:104820002C49CA7863F34512CA70012329498A7852
:1048300063F341028A7027498A7863F300028A7021
:1048400024490A7963F382020A7122490A7963F3DF
:10485000C3020A711F49CA7963F34512CA711D491F
:10486000CA7963F30412CA711A49CA7863F38202DF
:10487000CA701849CA7863F3C302CA700123154984
:104880008A7863F3C3028A7012498A7863F38202DA
:104890008A7010490A7963F341020A710D490A7955
:1048A00063F300020A710B49CA7963F3C712CA7134
:1048B0000849CA7963F38612CA710649CA7863F354
:1048C0000002CA700349CA7863F34102CA70FEE26B
:1048D0006C700020E87200207D4B1B680F2B00F3EA
:1048E000FB8001237B498A7963F386128A717949B7
:1048F0008A7963F3C7128A7176494A7963F30002B1
:104900004A7174494A7963F341024A7171494A799B
:1049100063F386124A716F494A7963F3C7124A7189
:104920006C498A7963F382028A716A498A7963F3EE
:10493000C3028A71012367498A7963F304128A7179
:1049400064498A7963F345128A7162494A7963F34B
:1049500082024A715F494A7963F3C3024A715D4931
:104960004A7963F304124A715A494A7963F345124A
:104970004A7158498A7963F300028A7155498A79E4
:1049800063F341028A71012352498A7863F38612E4
:104990008A7050498A7863F3C7128A704D490A7940
:1049A00063F345120A714B490A7963F304120A71E1
:1049B0004849CA7963F34102CA714649CA7963F327
:1049C0000002CA714349CA7863F38612CA7041492A
:1049D000CA7863F3C712CA7000233E498A7863F32A
:1049E00004128A703B498A7863F345128A70394908
:1049F0000A7963F3C7120A7136490A7963F386129A
:104A00000A713449CA7963F3C302CA713149CA7958
:104A100063F38202CA712F49CA7863F30412CA7021
:104A20002C49CA7863F34512CA70012329498A7850
:104A300063F341028A7027498A7863F300028A701F
:104A400024490A7963F382020A7122490A7963F3DD
:104A5000C3020A711F49CA7963F34512CA711D491D
:104A6000CA7963F30412CA711A49CA7863F38202DD
:104A7000CA701849CA7863F3C302CA700123154982
:104A80008A7863F3C3028A7012498A7863F38202D8
:104A90008A7010490A7963F341020A710D490A7953
:104AA00063F300020A710B49CA7963F3C712CA7132
:104AB0000849CA7963F38612CA710649CA7863F352
:104AC0000002CA700349CA7863F34102CA70FEE16A
:104AD0006C700020E87200207D4B1B68132B00F3E4
:104AE000FB8001237B498A7963F386128A717949B5
:104AF0008A7963F3C7128A7176494A7963F30002AF
:104B00004A7174494A7963F341024A7171494A7999
:104B100063F386124A716F494A7963F3C7124A7187
:104B20006C498A7963F382028A716A498A7963F3EC
:104B3000C3028A71012367498A7963F304128A7177
:104B400064498A7963F345128A7162494A7963F349
:104B500082024A715F494A7963F3C3024A715D492F
:104B60004A7963F304124A715A494A7963F3451248
:104B70004A7158498A7963F300028A7155498A79E2
:104B800063F341028A71012352498A7863F38612E2
:104B90008A7050498A7863F3C7128A704D490A793E
:104BA00063F345120A714B490A7963F304120A71DF
:104BB0004849CA7963F34102CA714649CA7963F325
:104BC0000002CA714349CA7863F38612CA70414928
:104BD000CA7863F3C712CA7001233E498A7863F327
:104BE00004128A703B498A7863F345128A70394906
:104BF0000A7963F3C7120A7136490A7963F3861298
:104C00000A713449CA7963F3C302CA713149CA7956
:104C100063F38202CA712F49CA7863F30412CA701F
:104C20002C49CA7863F34512CA70002329498A784F
:104C300063F341028A7027498A7863F300028A701D
:104C400024490A7963F382020A7122490A7963F3DB
:104C5000C3020A711F49CA7963F34512CA711D491B
:104C6000CA7963F30412CA711A49CA7863F38202DB
:104C7000CA701849CA7863F3C302CA700123154980
:104C80008A7863F3C3028A7012498A7863F38202D6
:104C90008A7010490A7963F341020A710D490A7951
:104CA00063F300020A710B49CA7963F3C712CA7130
:104CB0000849CA7963F38612CA710649CA7863F350
:104CC0000002CA700349CA7863F34102CA70FEE069
:104CD0006C700020E8720020C74B1B68172B00F394
:104CE000F6800123C5498A7963F386128A71C34924
:104CF0008A7963F3C7128A71C0494A7963F3000263
:104D00004A71BE494A7963F341024A71BB494A7903
:104D100063F386124A71B9494A7963F3C7124A713B
:104D2000B6498A7963F382028A71B4498A7963F356
:104D3000C3028A710123B1498A7963F304128A712B
:104D4000AE498A7963F345128A71AC494A7963F3B3
:104D500082024A71A9494A7963F3C3024A71A74999
:104D60004A7963F304124A71A4494A7963F34512FC
:104D70004A71A2498A7963F300028A719F498A794C
:104D800063F341028A7101239C498A7863F3861296
:104D90008A709A498A7863F3C7128A7097490A79A8
:104DA00063F345120A7195490A7963F304120A7193
:104DB0009249CA7963F34102CA719049CA7963F38F
:104DC0000002CA718D49CA7863F38612CA708B4992
:104DD000CA7863F3C712CA70012388498A7863F3DB
:104DE00004128A7085498A7863F345128A70834970
:104DF0000A7963F3C7120A7180490A7963F386124C
:104E00000A717E49CA7963F3C302CA717B49CA79C0
:104E100063F38202CA717949CA7863F30412CA70D3
:104E20007649CA7863F34512CA70012373498A78B8
:104E300063F341028A7071498A7863F300028A70D1
:104E40006E490A7963F382020A716C490A7963F345
:104E5000C3020A716949CA7963F34512CA71674985
:104E6000CA7963F30412CA716449CA7863F382028F
:104E7000CA706249CA7863F3C302CA7000235F49EB
:104E80008A7863F3C3028A705C498A7863F382028A
:104E90008A705A490A7963F341020A7157490A79BB
:104EA00063F300020A715549CA7963F3C712CA71E4
:104EB0005249CA7963F38612CA715049CA7863F3BA
:104EC0000002CA704D49CA7863F34102CA700023D8
:104ED000BB6006E14A4ABB6852F82330002B00F061
:104EE000A980BB68052B00F2F98001A252F823F0DB
:104EF000094F0000394F0000694F0000994F000032
:104F0000C94F0000055000003C4A13786FF30003BE
:104F100013703B4ABB68063352F82330002B05D090
:104F2000364A13786FF341031370D7E0334A13788E
:104F300043F002031370D1E0304A13786FF3820319
:104F400013702F4ABB68063352F82330002B05D06C
:104F50002A4A13786FF3C3031370BFE0274A13780C
:104F600043F008031370B9E0244A13786FF3041375
:104F70001370234ABB68063352F82330002B05D048
:104F80001E4A13786FF345131370A7E01B4A13787A
:104F900043F020031370A1E0184A13786FF38613CF
:104FA0001370174ABB68063352F82330002B05D024
:104FB000124A13786FF3C71313708FE00F4A1378F8
:104FC00043F08003137089E00C4A53786FF30003B9
:104FD00053700B4ABB68063352F82330002B05D0C0
:104FE000064A53786FF34103537077E0034A5378CE
:104FF00043F00203537071E06C700020E8720020EF
:10500000505A0020644A53786FF382035370634A06
:10501000BB68063352F82330002B05D05E4A537824
:105020006FF3C303537059E05B4A537843F00803AE
:10503000537053E0BB68052B50D801A252F823F0FF
:10504000595000006F500000855000009B50000038
:10505000B1500000C75000004F4A137843F00103DD
:1050600013704D4A137843F00203137036E04A4A36
:10507000137843F004031370474A137843F008038E
:1050800013702BE0444A137843F010031370424A24
:10509000137843F02003137020E03F4A137843F065
:1050A000400313703C4A137843F08003137015E0FB
:1050B000394A537843F001035370374A537843F029
:1050C000020353700AE0344A537843F004035370E8
:1050D000314A537843F00803537000BFBB68013373
:1050E000BB60BB68052B7FF7F5AE2D4B1B68002B13
:1050F0001AD02B4B5B68002B10D0294B9B68002BE0
:1051000005D0284B1B6803F00103D9B200E0002151
:10511000214A537861F30413537015E01E4A537803
:1051200043F0100353700FE01D4B9B68002B05D01C
:105130001C4B1B6803F00103D9B200E00121164AA1
:10514000537861F3041353700822134916480AF088
:1051500063FC0346002B1BD008220F4912480AF0BB
:105160002FFB0D4B3B6000237B600DE00F4A7B68FB
:10517000134418787B683A68134401221946FDF7F6
:1051800005FB7B6801337B607B68072BEEDD00E06D
:1051900000BF1037BD4680BDE8720020505A002085
:1051A000080000207870002074CC01201801010054
:1051B00080B582B000AF00237B601BE000233B7012
:1051C0007B68DBB2503BDBB27B700023BB701223E9
:1051D000FB703B46042219463C20FDF7D7FA7B685A
:1051E0009B01084A134440211846FDF789FA7B6861
:1051F00001337B607B68032BE0DD00BF00BF083715
:10520000BD4680BDACCD012080B588B002AFC34B98
:105210001B78DBB2002B40F0778200237B6146E0F5
:10522000BF4A7B6952F8233007EE903AB8EEE77A2E
:10523000DFEDBC6AC7EE267AC7ED007ABA4A7B6911
:105240009B001344D3ED007A9FEDB81AD7ED000A06
:10525000B0EE670A08F083FFF0EE407AB24A7B694D
:105260009B001344C3ED007AB14A7B699B00134451
:10527000D3ED006AAC4A7B699B001344D3ED007AFE
:1052800097ED007A77EE677A9FEDAA1AF0EE670A3B
:10529000B0EE660A08F063FFF0EE407AA44A7B693C
:1052A0009B001344C3ED007A7B6901337B617B690A
:1052B000032BB5DDA04B1A68A04B1968A048134614
:1052C0005B001344DB000B440C3350F82330002BFD
:1052D00000F06C819B4802F063FC002300931023D4
:1052E00024220021002002F099FB934B1A68934B73
:1052F0001968934813465B001344DB000B44843366
:1053000050F823303B613B69002B08DD0E230093EE
:105310000A238D4A0221012002F0EEFA16E03B69D1
:10532000002B0BDA0E2300930A23884A0221012066
:1053300002F0E2FA3B695B423B6107E00E23009317
:105340000A23834A0221012002F0D6FA3B69814AEE
:1053500082FB03129210DB17D31A092B70D801A21B
:1053600052F823F08D5300009F530000B15300000A
:10537000C3530000D5530000E7530000F953000069
:105380000B5400001D5400002F5400000E23009306
:105390000A236F4A02210D2002F0AEFA50E00E23DC
:1053A00000930A236C4A02210D2002F0A5FA47E07F
:1053B0000E2300930A23694A02210D2002F09CFA71
:1053C0003EE00E2300930A23654A02210D2002F0DD
:1053D00093FA35E00E2300930A23624A02210D203E
:1053E00002F08AFA2CE00E2300930A235E4A02217F
:1053F0000D2002F081FA23E00E2300930A235B4A7A
:1054000002210D2002F078FA1AE00E2300930A23FD
:10541000574A02210D2002F06FFA11E00E2300938B
:105420000A23544A02210D2002F066FA08E00E23F6
:1054300000930A23504A02210D2002F05DFA00BFBA
:105440003969444B83FB01239A10CB17D21A1346B8
:105450009B0013445B00CA1A092A00F2A38001A32F
:1054600053F822F08D5400009F540000B154000006
:10547000C3540000D5540000E7540000F954000064
:105480000B55000081550000935500000E2300933A
:105490000A233A4A0221192002F02EFA82E00E2352
:1054A00000930A232C4A0221192002F025FA79E000
:1054B0000E2300930A23294A0221192002F01CFA24
:1054C00070E00E2300930A23254A0221192002F0DE
:1054D00013FA67E00E2300930A23224A02211920BF
:1054E00002F00AFA5EE00E2300930A231E4A02210C
:1054F000192002F001FA55E00E2300930A231B4AFB
:105500000221192002F0F8F94CE00E2300930A233F
:10551000174A0221192002F0EFF943E010D10120CF
:10552000506A002000F07F457CCC01206F12833A46
:10553000ACCB0120CDCC4C3F687000206C700020BB
:10554000505A00201C300020205600209455002086
:105550005C72002067666666A85000203451002007
:10556000C05100204C520020D8520020645300202B
:10557000F05300207C540020085500201C500020CF
:105580000E2300930A23C54A0221192002F0B4F920
:1055900008E00E2300930A23C14A0221192002F0D9
:1055A000ABF900BFBF4B01221A600DE0BE4802F00C
:1055B000F7FA00230093202324220021002002F088
:1055C0002DFAB84B01221A60002300931D231722E5
:1055D0000021272002F022FA0023FB6090E0B34A6A
:1055E000FB6852F823300A334FF47A7200211846D0
:1055F00008F018FE07EE900AB8EEE77ADFEDAC6A25
:10560000C7EE267AC7ED017A786808F073FB024688
:105610000B4643EC102BFCF7BFF953EC102B104654
:10562000194608F03BFB03467B60A24AFB689B00DF
:105630001344D3ED006A9F4AFB689B001344D3EDEB
:10564000007A97ED017AB4EEE77AF1EE10FA02DD16
:10565000DFED997A01E0DFED997AB0EE671AD7EDC8
:10566000010AB0EE660A08F07AFDF0EE407A914A3F
:10567000FB689B001344C3ED007A8E4AFB689B00D5
:105680001344D3ED007AB3EE0B7A67EE877AFDEE22
:10569000E77A1B22002117EE900A08F0C3FD0246AC
:1056A0008749FB6841F82320FA6813465B001344DE
:1056B0005B0003F12800824AFB6852F82330C3F1F3
:1056C0001C01012300930123032202F0A7F9FA68C9
:1056D00013465B0013445B0003F12700784AFB6824
:1056E00052F82330C3F11D01754AFB6852F823308C
:1056F00001220092052202F091F9FB680133FB6060
:10570000FB68032B7FF76BAF6E4B1B78DBB2022B72
:1057100040F0FB80634B01221A606B4802F040FAB4
:105720006A4B9B68092B00F387800E2300930A23A2
:10573000674A0221142002F0DFF80E2300930A23A7
:10574000634A0221202002F0D7F8604B9B68092BA6
:1057500000F2DC8001A252F823F000BF8557000060
:1057600097570000A9570000BB570000CD57000015
:10577000DF570000F15700000358000015580000E3
:10578000275800000E2300930A23524A02211A20B0
:1057900002F0B2F8BAE00E2300930A234E4A022127
:1057A0001A2002F0A9F8B1E00E2300930A234B4A15
:1057B00002211A2002F0A0F8A8E00E2300930A2389
:1057C000474A02211A2002F097F89FE00E23009327
:1057D0000A23444A02211A2002F08EF896E00E2392
:1057E00000930A23404A02211A2002F085F88DE036
:1057F0000E2300930A233D4A02211A2002F07CF86E
:1058000084E00E2300930A23394A02211A2002F071
:1058100073F87BE00E2300930A23204A02211A200A
:1058200002F06AF872E00E2300930A231C4A022158
:105830001A2002F061F869E00E2300930A23264A39
:105840000221142002F058F8204B9968294B83FB61
:1058500001239A10CB17D31A1A4692001A44530008
:105860001A468B1A022B47D0022B4FDC002B02D09A
:10587000012B09D04AE00E2300930A23154A022186
:10588000202002F039F841E00E2300930A23124A47
:105890000221202002F030F838E000BF7C540020C4
:1058A00008550020707000201C300020506A002035
:1058B00000007A4400CC01206666663F0AD7A33B0D
:1058C0008CCC012010D101201C380020BC6A0020A3
:1058D0005C7200201C500020A85000203451002091
:1058E000C05100204C520020D852002064530020A8
:1058F000F0530020676666660E2300930A23B24ABF
:105900000221202001F0F8FF00E000BFAF4B1B7820
:10591000DBB2012B40F0DB86AD4BDB68002B00F0E7
:105920006285AC4B1B68052B00F2598501A252F829
:1059300023F000BF4D590000015B0000CF5C000068
:105940007F5E00003B600000EB610000A24BBB608B
:10595000A24B1B68002B5DD0BB6803F5307300229F
:10596000DA77BA6802F53072DB7F9377BB6803F5AC
:10597000507300225A77BA6802F540725B7F537702
:10598000BB6803F53073002283F83C20BA6802F547
:10599000307293F83C3082F83B30BB6803F55073AB
:1059A000002283F83D20BA6802F5407293F83D303A
:1059B00082F83D30BB6803F5A8630022DA77BA6845
:1059C00002F5A862DB7F9377BB6803F5A063002232
:1059D0005A77BA6802F598625B7F5377BB6803F524
:1059E000A863002283F83C20BA6802F5A86293F805
:1059F0003C3082F83B30BB6803F5A063002283F89B
:105A00003D20BA6802F5986293F83D3082F83D3047
:105A100000F0E5BCBB6803F53072FF23D377BB68A9
:105A200003F53073D27F9A77BA6802F530729B7FA4
:105A30005377BB6803F55073FF225A77BA6802F5B3
:105A400040725B7F5377BB6803F53072FF2382F8A7
:105A50003D30BB6803F5307392F83D2083F83C205D
:105A6000BA6802F5307293F83C3082F83B30BB687C
:105A700003F55073FF2283F83D20BA6802F54072A7
:105A800093F83D3082F83D30BB6803F5A862FF23F0
:105A9000D377BB6803F5A863D27F9A77BA6802F51B
:105AA000A8629B7F5377BB6803F5A063FF225A77F8
:105AB000BA6802F598625B7F5377BB6803F5A8620A
:105AC000FF2382F83D30BB6803F5A86392F83D20C0
:105AD00083F83C20BA6802F5A86293F83C3082F85B
:105AE0003B30BB6803F5A063FF2283F83D20BA6812
:105AF00002F5986293F83D3082F83D3000F06FBCBB
:105B0000374BBB60354B1B68002B6BD0BB6803F574
:105B100030730022DA77BA6802F53072DB7F937750
:105B2000BB6803F5507300225A77BA6802F54072D9
:105B30005B7F5377BB6803F53073002283F83C200A
:105B4000BA6802F5307293F83C3082F83B30BB689B
:105B500003F55073002283F83D20BA6802F54072C5
:105B600093F83D3082F83D30BB6803F5A86300220E
:105B7000DA77BA6802F5A862DB7F9377BB6803F532
:105B8000A06300225A77BA6802F598625B7F537768
:105B9000BB6803F5A863002283F83C20BA6802F5CD
:105BA000A86293F83C3082F83B30BB6803F5A063F1
:105BB000002283F83D20BA6802F5986293F83D30E0
:105BC00082F83D3000F00BBC3451002010D1012090
:105BD00008000020BC6A00201C0000207870002013
:105BE0001C080020BB6803F53072FF23D377BB6825
:105BF00003F53073D27F9A77BA6802F530729B7FD3
:105C00005377BB6803F55073FF225A77BA6802F5E1
:105C100040725B7F5377BB6803F53072FF2382F8D5
:105C20003D30BB6803F5307392F83D2083F83C208B
:105C3000BA6802F5307293F83C3082F83B30BB68AA
:105C400003F55073FF2283F83D20BA6802F54072D5
:105C500093F83D3082F83D30BB6803F5A862FF231E
:105C6000D377BB6803F5A863D27F9A77BA6802F549
:105C7000A8629B7F5377BB6803F5A063FF225A7726
:105C8000BA6802F598625B7F5377BB6803F5A86238
:105C9000FF2382F83D30BB6803F5A86392F83D20EE
:105CA00083F83C20BA6802F5A86293F83C3082F889
:105CB0003B30BB6803F5A063FF2283F83D20BA6840
:105CC00002F5986293F83D3082F83D3087E39D4BB2
:105CD000BB609D4B1B68002B5CD0BB6803F5307329
:105CE00000225A76BA6802F530725B7E1376BB6882
:105CF00003F550730022DA75BA6802F54072DB7D55
:105D0000D375BB6803F53073002283F83C20BA6872
:105D100002F5307293F83C3082F83B30BB6803F5F3
:105D20005073002283F83D20BA6802F5407293F860
:105D30003D3082F83D30BB6803F5A86300225A76F7
:105D4000BA6802F5A8625B7E1376BB6803F5A063B0
:105D50000022DA75BA6802F59862DB7DD375BB68FC
:105D600003F5A863002283F83C20BA6802F5A86214
:105D700093F83C3082F83B30BB6803F5A063002207
:105D800083F83D20BA6802F5986293F83D3082F8B6
:105D90003D3024E3BB6803F53072FF235376BB68C4
:105DA00003F53073527E1A76BA6802F530721B7EA4
:105DB000D375BB6803F55073FF22DA75BA6802F534
:105DC0004072DB7DD375BB6803F53072FF2382F828
:105DD0003D30BB6803F5307392F83D2083F83C20DA
:105DE000BA6802F5307293F83C3082F83B30BB68F9
:105DF00003F55073FF2283F83D20BA6802F5407224
:105E000093F83D3082F83D30BB6803F5A862FF236C
:105E10005376BB6803F5A863527E1A76BA6802F51A
:105E2000A8621B7ED375BB6803F5A063FF22DA75F9
:105E3000BA6802F59862DB7DD375BB6803F5A8628A
:105E4000FF2382F83D30BB6803F5A86392F83D203C
:105E500083F83C20BA6802F5A86293F83C3082F8D7
:105E60003B30BB6803F5A063FF2283F83D20BA688E
:105E700002F5986293F83D3082F83D30AFE2334B43
:105E8000BB60314B1B68002B62D0BB6803F53073DD
:105E900000225A76BA6802F530725B7E1376BB68D0
:105EA00003F550730022DA75BA6802F54072DB7DA3
:105EB000D375BB6803F53073002283F83C20BA68C1
:105EC00002F5307293F83C3082F83B30BB6803F542
:105ED0005073002283F83D20BA6802F5407293F8AF
:105EE0003D3082F83D30BB6803F5A86300225A7646
:105EF000BA6802F5A8625B7E1376BB6803F5A063FF
:105F00000022DA75BA6802F59862DB7DD375BB684A
:105F100003F5A863002283F83C20BA6802F5A86262
:105F200093F83C3082F83B30BB6803F5A063002255
:105F300083F83D20BA6802F5986293F83D3082F804
:105F40003D304CE21C100020787000201C1800200E
:105F5000BB6803F53072FF235376BB6803F53073DB
:105F6000527E1A76BA6802F530721B7ED375BB6812
:105F700003F55073FF22DA75BA6802F54072DB7DD3
:105F8000D375BB6803F53072FF2382F83D30BB68E0
:105F900003F5307392F83D2083F83C20BA6802F58F
:105FA000307293F83C3082F83B30BB6803F5507395
:105FB000FF2283F83D20BA6802F5407293F83D3025
:105FC00082F83D30BB6803F5A862FF235376BB68B7
:105FD00003F5A863527E1A76BA6802F5A8621B7EA2
:105FE000D375BB6803F5A063FF22DA75BA6802F5C2
:105FF0009862DB7DD375BB6803F5A862FF2382F846
:106000003D30BB6803F5A86392F83D2083F83C203F
:10601000BA6802F5A86293F83C3082F83B30BB685E
:1060200003F5A063FF2283F83D20BA6802F5986269
:1060300093F83D3082F83D30D1E1A34BBB60A34BD8
:106040001B68002B5CD0BB6803F5307300225A76C6
:10605000BA6802F530725B7E1376BB6803F5507345
:106060000022DA75BA6802F54072DB7DD375BB6831
:1060700003F53073002283F83C20BA6802F53072D1
:1060800093F83C3082F83B30BB6803F55073002234
:1060900083F83D20BA6802F5407293F83D3082F8EB
:1060A0003D30BB6803F5A86300225A76BA6802F552
:1060B000A8625B7E1376BB6803F5A0630022DA75E5
:1060C000BA6802F59862DB7DD375BB6803F5A863F7
:1060D000002283F83C20BA6802F5A86293F83C30AD
:1060E00082F83B30BB6803F5A063002283F83D20B3
:1060F000BA6802F5986293F83D3082F83D306EE15F
:10610000BB6803F53072FF235376BB6803F5307329
:10611000527E1A76BA6802F530721B7ED375BB6860
:1061200003F55073FF22DA75BA6802F54072DB7D21
:10613000D375BB6803F53072FF2382F83D30BB682E
:1061400003F5307392F83D2083F83C20BA6802F5DD
:10615000307293F83C3082F83B30BB6803F55073E3
:10616000FF2283F83D20BA6802F5407293F83D3073
:1061700082F83D30BB6803F5A862FF235376BB6805
:1061800003F5A863527E1A76BA6802F5A8621B7EF0
:10619000D375BB6803F5A063FF22DA75BA6802F510
:1061A0009862DB7DD375BB6803F5A862FF2382F894
:1061B0003D30BB6803F5A86392F83D2083F83C208E
:1061C000BA6802F5A86293F83C3082F83B30BB68AD
:1061D00003F5A063FF2283F83D20BA6802F59862B8
:1061E00093F83D3082F83D30F9E0394BBB60374BD6
:1061F0001B68002B6ED0BB6803F53073002283F858
:106200002A20BA6802F5307293F82A3082F82930D1
:10621000BB6803F55073002283F82820BA6802F5A2
:10622000407293F8283082F82830BB6803F5307349
:10623000002283F83C20BA6802F5307293F83C30B3
:1062400082F83B30BB6803F55073002283F83D2091
:10625000BA6802F5407293F83D3082F83D30BB6871
:1062600003F5A863002283F82A20BA6802F5A86221
:1062700093F82A3082F82930BB6803F5A063002226
:1062800083F82820BA6802F5986293F8283082F8DB
:106290002830BB6803F5A863002283F83C20BA6865
:1062A00002F5A86293F83C3082F83B30BB6803F5F6
:1062B000A063002283F83D20BA6802F5986293F843
:1062C0003D3082F83D3089E01C20002078700020AD
:1062D0001C280020BB6803F53072FF2382F82A30A7
:1062E000BB6803F5307392F82A2083F82920BA6836
:1062F00002F5307293F8293082F82830BB6803F534
:106300005073FF2283F82820BA6802F5407293F890
:10631000283082F82830BB6803F53072FF2382F8FA
:106320003D30BB6803F5307392F83D2083F83C2084
:10633000BA6802F5307293F83C3082F83B30BB68A3
:1063400003F55073FF2283F83D20BA6802F54072CE
:1063500093F83D3082F83D30BB6803F5A862FF2317
:1063600082F82A30BB6803F5A86392F82A2083F8E4
:106370002920BA6802F5A86293F8293082F82830FB
:10638000BB6803F5A063FF2283F82820BA6802F5F2
:10639000986293F8283082F82830BB6803F5A86229
:1063A000FF2382F83D30BB6803F5A86392F83D20D7
:1063B00083F83C20BA6802F5A86293F83C3082F872
:1063C0003B30BB6803F5A063FF2283F83D20BA6829
:1063D00002F5986293F83D3082F83D3000BFB8680E
:1063E00001F0DEFB70E1C94BBB60C94B1B68002BA1
:1063F00068D0BB6803F53073002283F83720BA6891
:1064000002F5307293F8373082F83630BB6803F506
:106410005073002283F83520BA6802F5407293F871
:10642000353082F83530BB6803F53073002283F8CD
:106430003C20BA6802F5307293F83C3082F83B3069
:10644000BB6803F55073002283F83D20BA6802F55B
:10645000407293F83D3082F83D30BB6803F5A86385
:10646000002283F83720BA6802F5A86293F8373023
:1064700082F83630BB6803F5A063002283F835202C
:10648000BA6802F5986293F8353082F83530BB6807
:1064900003F5A863002283F83C20BA6802F5A862DD
:1064A00093F83C3082F83B30BB6803F5A0630022D0
:1064B00083F83D20BA6802F5986293F83D3082F87F
:1064C0003D3083E0BB6803F53072FF2382F837303C
:1064D000BB6803F5307392F8372083F83620BA682A
:1064E00002F5307293F8363082F83530BB6803F528
:1064F0005073FF2283F83520BA6802F5407293F892
:10650000353082F83530BB6803F53072FF2382F8EE
:106510003D30BB6803F5307392F83D2083F83C2092
:10652000BA6802F5307293F83C3082F83B30BB68B1
:1065300003F55073FF2283F83D20BA6802F54072DC
:1065400093F83D3082F83D30BB6803F5A862FF2325
:1065500082F83730BB6803F5A86392F8372083F8D8
:106560003620BA6802F5A86293F8363082F83530E2
:10657000BB6803F5A063FF2283F83520BA6802F5F3
:10658000986293F8353082F83530BB6803F5A8621D
:10659000FF2382F83D30BB6803F5A86392F83D20E5
:1065A00083F83C20BA6802F5A86293F83C3082F880
:1065B0003B30BB6803F5A063FF2283F83D20BA6837
:1065C00002F5986293F83D3082F83D30B86801F0EA
:1065D000E7FAFCF7AFFC4F4B5B68002BB8BF5B42A0
:1065E000092B71D801A252F823F000BF15660000F4
:1065F00027660000396600004B6600005D660000FB
:106600006F6600008166000093660000A5660000CA
:10661000B76600000723009305233F4A0D2137206A
:1066200001F06AF950E00723009305233B4A0D214E
:10663000372001F061F947E0072300930523384A2A
:106640000D21372001F058F93EE007230093052380
:10665000344A0D21372001F04FF935E0072300932C
:106660000523314A0D21372001F046F92CE007239C
:10667000009305232D4A0D21372001F03DF923E039
:106680000723009305232A4A0D21372001F034F90E
:106690001AE0072300930523264A0D21372001F035
:1066A0002BF911E0072300930523234A0D213720FE
:1066B00001F022F908E00723009305231F4A0D216A
:1066C000372001F019F900BF1D4B01221A6001F0BB
:1066D0000BFB1B4B1B68002B15D04FF48072194924
:1066E000194809F099F90346002B0BD04FF480723A
:1066F0001449154809F064F8FEF75AFD104B0022C2
:106700001A6000E000BF1837BD4680BD1C40002065
:1067100078700020BC6A0020AC560020D0560020C3
:10672000F4560020185700203C57002060570020E6
:1067300084570020A8570020CC570020F057002095
:1067400070700020ACCD01209CCC012080B582B0BF
:1067500000AF2E4B9B68002B1DD100237B6017E000
:106760002B4A7B68FC339B00134493ED007A294A43
:106770007B681B0113440833D3ED007AB4EE677ACB
:10678000F1EE10FA01D0FBF79FFF7B6801337B60CD
:106790007B68172BE4DD204B1B68204A52F823202E
:1067A0001F4B1B689A422CDC00233B6026E01D4AED
:1067B0003B689B00134493ED007A1B4A3B689B00A7
:1067C0001344D3ED007A77EE677AB0EE670A08F0EB
:1067D000DCFFF0EE407A9FED157AF4EEC77AF1EE29
:1067E00010FA08DD602210490E4808F0E9FF01F0B8
:1067F00063FA00BF05E03B6801333B603B68172B41
:10680000D5DD00BF0837BD4680BD00BF08000020B1
:10681000505A0020E86E0020BC6A00203C5800203E
:10682000B0CE012010CC0120C0580020295C8F3D43
:1068300080B500AF72B600BF0E4B1B680E4A52F80F
:1068400023200E4B1B68D31A032B07DC094B1B6854
:10685000094A52F82330043B084A13606022084971
:10686000084808F0ADFFBFF34F8F00BF62B600BF0E
:1068700000BF80BDBC6A00203C580020B0CE012083
:10688000C058002010CC012080B500AF0C4B9B6895
:106890009BB21A46920013441A4691001A460B46C0
:1068A00013441A46D200D31A9BB203F26C739BB204
:1068B0001A460021034804F051FC00BF80BD00BF10
:1068C000BC6A002000C00C4080B582B000AF08F068
:1068D000EEFE08F0B0FD08F090FE01F063FAFBF761
:1068E00013FD07F026FEFBF761FC0020FBF70CFB15
:1068F00000237B6025E07B682C2202FB03F3434AE4
:1069000013440421DFED422A9FED422ADFED401AB5
:106910009FED411AF7EE000A9FED3E0A184607F078
:1069200098FC7B681B013D4A13449FED3A1AF7EE31
:10693000000A9FED380A184607F0A9FD7B6801336D
:106940007B607B68172BD6DDFBF748FF00233B609D
:1069500004E007F0EEFD3B6801333B603B680E2B23
:10696000F7DD2F4B1E221A61FBF78EFAFBF76AFB4D
:1069700018222C493C20FBF709FFFCF7DBFA2A4BD5
:1069800003F520431B8801339AB2274B03F52043BC
:106990001A80264B9B689BB21A46920013441A46F3
:1069A00091001A460B4613441A46D200D31A9BB2E2
:1069B00003F26C739BB21A4600211D4804F0CEFB13
:1069C0001C4B1B68092B07DC1A4B1B680133194A47
:1069D0001360194B00221A60184B1B785A1CD1B255
:1069E000164A11701E2B06D9FFF7B0FE134B00227A
:1069F0001A70FEF709FC01F083FAFBF71FFFFCF7A2
:106A0000F5FAFBF7B7FCFBF71DFBD9E7C86A0020D6
:106A1000CDCC4C3E000000000AD7233CE86E00209D
:106A20000800002014580020A82B0120BC6A002078
:106A300000C00C409CCD01206870002011D10120C5
:106A400080B582B000AF00212A4807F010FB7860C3
:106A50007A680021274807F01FFB274B1B78DBB221
:106A6000012B05D0254B1B680133244A136002E03B
:106A7000224B00221A60224B1B680133204A13600C
:106A80001F4B19681F4BA3FB0123DA0913461B0296
:106A90009B1ACA1A002A05D11B4B1B68C3F10103BC
:106AA000194A1360154B1B687D2B13D1174B1B68BC
:106AB000174A52F82320174B1B689A4203DD154BE7
:106AC0001B68013301E0134B1B68124A13600B4B28
:106AD00000221A60104B1B68002B04D00E4B1B6861
:106AE000013B0D4A1360BFF34F8F00BF00BF083753
:106AF000BD4680BD0070034010D10120A0CD012013
:106B0000747000208180808078700020BC6A002032
:106B10003C580020B0CE0120FCCB012090B58DB0B8
:106B200000AF4FF000033B61BD4B1B78032B00F21D
:106B3000818601A252F823F025780000496B0000FD
:106B4000616F00009F7300000023FB620023BB62A3
:106B50002BE0B44ABB6A043352F8233007EE903A74
:106B6000B8EEE77AB04B1B68B04A52F82310B04831
:106B7000BA6A13465B001344DB000B44843350F8BD
:106B8000233007EE903AF8EEE77A27EE277ADFED2A
:106B9000A96AC7EE267AFDEEE77A17EE902AFB6A1D
:106BA0001344FB62BB6A0133BB62BB6A042BD0DDBA
:106BB0000021A148FBF718F807EE900AB8EE677AB3
:106BC000DFED9E6AC7EE267AC7ED047A964B1B6806
:106BD000964A52F823309A4A9B001344D3ED007A28
:106BE000914B1B68914A52F823409FED961AD7EDBE
:106BF000040AB0EE670A07F0B2FAF0EE407A904A63
:106C0000A3001344C3ED007A874B1B68874A52F8F0
:106C100023301B018C4A9C18834B1B68834A52F813
:106C200023302C2202FB03F3884A134497ED040A15
:106C3000184607F060FBF0EE407AB0EE670A204697
:106C4000FBF760F8F0EE407A9FED7C7A67EE877A8A
:106C5000FDEEE77A744B1B68744A52F8233017EE46
:106C6000901A7B4A42F823107A4B1B691E2B20D1C5
:106C70006D4B1B686D4A52F823302C2202FB03F344
:106C8000724A134497ED040A184607F034FBF0EEFD
:106C9000407A9FED6A7A67EE877AFDEEE77A624B7B
:106CA0001B68624A52F8233017EE901A684A42F87D
:106CB00023105D4B1B685D4A52F82330644A52F83A
:106CC0002320FB6A134440F6FF720021184607F0A8
:106CD000A9FA0146544B1B68544A52F823305E4AC5
:106CE00042F82310504B1B68504A52F82330584A40
:106CF00052F823301A46FB6A134407EE903AF8EE36
:106D0000E77A9FED4E1ADFED550AB0EE670A07F0FD
:106D100060FAF0EE407AB7EE002ADFED501A9FEDF0
:106D2000501ADFED4E0AB0EE670AFAF773FF87EDEF
:106D3000030AD7ED037A9FED4B7AF4EEC77AF1EEB2
:106D400010FA10D59FED482ADFED441A9FED451A41
:106D5000DFED420A97ED030AFAF75CFFF0EE407AA6
:106D6000FDEEE77A1FE0B7EE002ADFED3C1AB7EE42
:106D7000001ADFED3C0A97ED030AFAF74BFFF0EE3D
:106D8000407AB0EE670A07F0DAF9F0EE407AB0EE3A
:106D9000671ADFED2A0A9FED340A07F0E0F9F0EEFA
:106DA000407AFDEEE77AC7ED027A304B1B78DBB212
:106DB000032B09D01C4B1B681C4A52F82330BA68BD
:106DC0002B4941F8232025E0284B1B78DBB2032B0D
:106DD00020D1154B1B68154A52F823309A08254BD1
:106DE0001B68002B00DA03339B109A4209D10E4B2B
:106DF0001B680E4A52F82330BA681D4941F8232017
:106E000008E0094B1B68094A52F82330184A002150
:106E100042F82310184B38225A6000237B623EE070
:106E200012D10120506A0020A4CD0120B800010039
:106E3000505A00200000C84200B0034000F07F45D7
:106E4000C05800200AD7233CE86E0020C86A002002
:106E50002059002008000020805900200000000078
:106E600000007A450AD7A33B0000FA4410D1012064
:106E7000E05900206C70002080F00F40C54B1A686C
:106E80007B6A42FA03F3DBB203F00103DBB21A467A
:106E9000796AC14807F082F87B6A01337B627B6ABA
:106EA000022BEBD9BB4B1B68002B00DA03339B1082
:106EB0001A46BA4B53F82230002B0BD1B54B1B6846
:106EC000B74A52F823309BB21A460021B54804F065
:106ED00045F910E0AF4B1B681846F9F799FAF0EE48
:106EE000407AFCEEE77A17EE903A9BB21A46002100
:106EF000AC4804F033F900220321A74807F04EF80C
:106F000001220321A84807F049F800221221A648CF
:106F100007F044F801221321A34807F03FF80023AB
:106F20003B6210E0396A9B4B1A683B6A42FA03F3F2
:106F3000DBB203F00103DBB21A469B4807F02EF8E0
:106F40003B6A01333B623B6A022BEBDD974B02222B
:106F50001A70974A0021974803F086FB00F06ABC3C
:106F60000023FB620023BB622CE0934ABB6A04331C
:106F700052F8233007EE903AB8EEE77A854B1B685B
:106F800008338E4A52F823108448BA6A13465B00CD
:106F90001344DB000B44843350F8233007EE903A5F
:106FA000F8EEE77A27EE277ADFED856AC7EE267AD4
:106FB000FDEEE77A17EE902AFB6A1344FB62BB6A88
:106FC0000133BB62BB6A042BCFDD00217948FAF79D
:106FD0000BFE07EE900AB8EE677ADFED846AC7EE23
:106FE000267AC7ED047A6B4B1B680833734A52F854
:106FF0002330744A9B001344D3ED007A654B1B6821
:1070000008336E4A52F823409FED6F1AD7ED040AF9
:10701000B0EE670A07F0A3F8F0EE407A694AA300E1
:107020001344C3ED007A5B4B1B680833634A52F884
:1070300023301B01654A9C18564B1B6808335F4A76
:1070400052F823302C2202FB03F3614A134497EDDC
:10705000040A184607F04FF9F0EE407AB0EE670ADE
:107060002046FAF74FFEF0EE407A9FED607A67EE29
:10707000877AFDEEE77A474B1B6808334F4A52F890
:10708000233017EE901A534A42F82310524B1B69D3
:107090001E2B22D13F4B1B680833484A52F823303D
:1070A0002C2202FB03F34A4A134497ED040A1846C4
:1070B00007F021F9F0EE407A9FED4C7A67EE877A7F
:1070C000FDEEE77A334B1B6808333C4A52F8233015
:1070D00017EE901A3F4A42F823102E4B1B680833D4
:1070E000364A52F823303B4A52F82320FB6A1344B5
:1070F00040F6FF720021184607F094F80146254B30
:107100001B6808332D4A52F82330344A42F82310C2
:10711000204B1B680833294A52F823302D4A52F875
:1071200023301A46FB6A134407EE903AF8EEE77AEA
:107130009FED2E1ADFED2B0AB0EE670A07F049F833
:10714000F0EE407AB7EE002ADFED261A9FED241A02
:10715000DFED240AB0EE670AFAF75CFD87ED030A5B
:10716000D7ED037A9FED207AF4EEC77AF1EE10FAAC
:1071700040D59FED1F2ADFED1B1A9FED1B1ADFED97
:10718000190A97ED030AFAF745FDF0EE407AFDEE95
:10719000E77A4FE0A4CD012080F00F40505A002044
:1071A000E059002000D00C4040F00F4012D10120E7
:1071B0006C58002000B00340506A0020B800010065
:1071C0000000C842C05800200AD7233CE86E0020C7
:1071D000C86A0020205900200800002080590020A3
:1071E00000007A45000000000AD7A33B00F07F456D
:1071F0000000FA44B7EE002A5FED061AB7EE001A57
:107200005FED070A97ED030AFAF704FDF0EE407A06
:10721000B0EE670A06F093FFF0EE407AB0EE671A20
:107220005FED0E0A1FED0E0A06F099FFF0EE407AB0
:10723000FDEEE77AC7ED027A5B4B1B78DBB2032BDE
:107240000AD05A4B1B680833594A52F82330BA689F
:10725000584941F8232028E0534B1B78DBB2032B1D
:1072600023D1524B1B680833514A52F823309A08F5
:10727000514B1B68002B00DA03339B109A420AD152
:107280004A4B1B6808334A4A52F82330BA684949C6
:1072900041F8232009E0454B1B680833444A52F863
:1072A0002330444A002142F82310444B38225A60CC
:1072B0000023FB6110E03D4B1A68FB6942FA03F3BF
:1072C000DBB203F00103DBB21A46F9693B4806F072
:1072D00065FEFB690133FB61FB69022BEBD9334B84
:1072E0001B680833002B00DA03339B101A46344B1B
:1072F00053F82230002B0CD12C4B1B6808332D4A3D
:1073000052F823309BB21A4600212E4803F026FF84
:1073100011E0264B1B6808331846F9F779F8F0EEB0
:10732000407AFCEEE77A17EE903A9BB21A460021BB
:10733000244803F013FF00220421204806F02EFE0B
:1073400001220321204806F029FE012212211E48B5
:1073500006F024FE002213211B4806F01FFE002326
:10736000BB6110E0B969114B1A68BB6942FA03F3BB
:10737000DBB203F00103DBB21A46134806F00EFE3F
:10738000BB690133BB61BB69022BEBDD0F4B0322F1
:107390001A700F4A00210F4803F066F94AE20023F1
:1073A000FB620023BB6244E010D10120A4CD012088
:1073B000B8000100E05900206C70002080F00F4000
:1073C000505A002000D00C4040F00F4012D1012054
:1073D0006C58002000B00340BA4ABB6A043352F82C
:1073E000233007EE903AB8EEE77AB74B1B681033BC
:1073F000B64A52F82310B648BA6A13465B001344E3
:10740000DB000B44843350F8233007EE903AF8EE5B
:10741000E77A27EE277ADFEDAF6AC7EE267AFDEE30
:10742000E77A17EE902AFB6A1344FB62BB6A0133CA
:10743000BB62BB6A042BCFDD0021A748FAF7D4FB5F
:1074400007EE900AB8EE677ADFEDA46AC7EE267AF7
:10745000C7ED047A9C4B1B6810339C4A52F82330CA
:107460009F4A9B001344D3ED007A974B1B6810335F
:10747000964A52F823409FED9B1AD7ED040AB0EECE
:10748000670A06F06CFEF0EE407A954AA3001344BA
:10749000C3ED007A8C4B1B6810338C4A52F82330B2
:1074A0001B01914A9C18884B1B681033874A52F87D
:1074B00023302C2202FB03F38C4A134497ED040A79
:1074C000184606F018FFF0EE407AB0EE670A204644
:1074D000FAF718FCF0EE407A9FED807A67EE877A33
:1074E000FDEEE77A784B1B681033784A52F8233068
:1074F00017EE901A7E4A42F823107E4B1B691E2B12
:1075000022D1714B1B681033704A52F823302C2261
:1075100002FB03F3754A134497ED040A184606F07C
:10752000EAFEF0EE407A9FED6D7A67EE877AFDEE27
:10753000E77A654B1B681033644A52F8233017EE24
:10754000901A6B4A42F823105F4B1B6810335F4A56
:1075500052F82330664A52F82320FB6A134440F65F
:10756000FF720021184606F05DFE0146564B1B686F
:107570001033564A52F823305F4A42F82310524BD8
:107580001B681033514A52F82330594A52F82330BD
:107590001A46FB6A134407EE903AF8EEE77A9FED3D
:1075A0004F1ADFED560AB0EE670A06F012FEF0EE53
:1075B000407AB7EE002ADFED511A9FED511ADFED48
:1075C0004F0AB0EE670AFAF725FB87ED030AD7EDFD
:1075D000037A9FED4C7AF4EEC77AF1EE10FA10D5EB
:1075E0009FED492ADFED451A9FED461ADFED430A6C
:1075F00097ED030AFAF70EFBF0EE407AFDEEE77A1C
:107600001FE0B7EE002ADFED3D1AB7EE001ADFEDFE
:107610003D0A97ED030AFAF7FDFAF0EE407AB0EE74
:10762000670A06F08CFDF0EE407AB0EE671ADFEDE7
:107630002B0A9FED350A06F092FDF0EE407AFDEE42
:10764000E77AC7ED027A314B1B78DBB2032B0AD005
:107650001D4B1B6810331D4A52F82330BA682C4961
:1076600041F8232028E0294B1B78DBB2032B23D1E0
:10767000154B1B681033154A52F823309A08254BD6
:107680001B68002B00DA03339B109A420AD10E4B81
:107690001B6810330D4A52F82330BA681C4941F870
:1076A000232009E0084B1B681033084A52F82330A6
:1076B000174A002142F82310174B38225A60002342
:1076C0007B613CE0506A0020A4CD0120B80001009D
:1076D000505A00200000C84200B0034000F07F452F
:1076E000C05800200AD7233CE86E0020C86A00205A
:1076F00020590020080000208059002000000000D0
:1077000000007A450AD7A33B0000FA4410D10120BB
:10771000E05900206C70002080F00F40494B1A683F
:107720007B6942FA03F3DBB203F00103DBB21A46D2
:107730007969454806F032FC7B6901337B617B69DE
:10774000022BEBD93F4B1B681033002B00DA0333BD
:107750009B101A463D4B53F82230002B0CD1394B6D
:107760001B6810333A4A52F823309BB21A46002164
:10777000384803F0F3FC11E0324B1B681033184615
:10778000F8F746FEF0EE407AFCEEE77A17EE903A14
:107790009BB21A4600212F4803F0E0FC002205218D
:1077A000294806F0FBFB274B1B680133254A136071
:1077B000244B1B685A4203F0070302F0070258BF2C
:1077C0005342204A136000220321234806F0E6FBBF
:1077D00001221221204806F0E1FB012213211E485C
:1077E00006F0DCFB00237B6010E07968154B1A681B
:1077F0007B6842FA03F3DBB203F00103DBB21A4603
:10780000154806F0CBFB7B6801337B607B68022B5D
:10781000EBD9124B01221A70114A0021114802F0D3
:1078200023FF07E000210F48FAF7DEF90B4B012296
:107830001A7000BFBFF34F8F00BF00BF3437BD4683
:1078400090BD00BFA4CD012080F00F40505A002011
:10785000E059002000D00C4040F00F4012D1012030
:107860006C58002000B0034080B582B000AF0948DA
:1078700003F014FF78607968064803F027FF0020C2
:1078800000F016FBBFF34F8F00BF00BF0837BD46A7
:1078900080BD00BF40F00F4080B582B000AF094806
:1078A00003F0FCFE78607968064803F00FFF0120C2
:1078B00000F0FEFABFF34F8F00BF00BF0837BD4690
:1078C00080BD00BFC0F00F4080B582B000AF094856
:1078D00003F0E4FE78607968064803F0F7FE0220C2
:1078E00000F0E6FABFF34F8F00BF00BF0837BD4678
:1078F00080BD00BF80F00F4090B488B000AFF8604A
:10790000B9607A603B603C68631E7B612346184621
:107910004FF000014FF000024FF00003CB0043EAAC
:107920005073C2007B683B610023BB616AE00023A7
:10793000FB6160E02246FB6903FB02F33A691A44EB
:10794000BB6913441B78002B28D1BA69FB68D11896
:10795000FA69BB681344002B00DA0733DB101A46C0
:1079600093010B442C49CB5C59B2F869BB680344C2
:10797000584203F0070300F0070058BF43420120BC
:1079800000FA03F35BB20B4358B2B969FB681944C0
:1079900093010B44C1B2204AD15429E0BA69FB6873
:1079A000D118FA69BB681344002B00DA0733DB10E7
:1079B0001A4693010B441849CB5C59B2F869BB686D
:1079C0000344584203F0070300F0070058BF434246
:1079D000012000FA03F35BB2DB435BB20B4058B209
:1079E000B969FB68194493010B44C1B20A4AD154E6
:1079F000FB690133FB61FA69BB6A9A429ADBBB6996
:107A00000133BB61BA693B689A4290DB00BF00BF9B
:107A10002037BD4690BC7047ACCD012080B487B004
:107A200000AFF860B9607A603B60FB687B6154E04E
:107A3000BB683B6148E03B6A002B22D03B69002BCE
:107A400000DA0733DB101A4691017B690B442949A0
:107A5000CB5C59B23B69584203F0070300F00700C2
:107A600058BF4342012000FA03F35BB2DB435BB231
:107A70000B4059B292017B691344C9B21D4AD154DB
:107A80001FE03B69002B00DA0733DB101A46910137
:107A90007B690B441749CB5C59B23B69584203F0F0
:107AA000070300F0070058BF4342012000FA03F328
:107AB0005BB20B4359B292017B691344C9B20D4AC0
:107AC000D1543B6901333B61BA683B6813443A695E
:107AD0009A42B0DB7B6901337B61FA687B681344AF
:107AE0007A699A42A4DB00BF00BF1C37BD465DF82F
:107AF000047B7047ACCD012080B485B000AFF86046
:107B0000B9607A607B68002B22D0BB68002B00DA5A
:107B10000733DB101A469101FB680B441F49CB5C0D
:107B200059B2BB68584203F0070300F0070058BF82
:107B30004342012000FA03F35BB2DB435BB20B402C
:107B400059B29201FB681344C9B2144AD1541FE0E0
:107B5000BB68002B00DA0733DB101A469101FB6883
:107B60000B440E49CB5C59B2BB68584203F0070383
:107B700000F0070058BF4342012000FA03F35BB254
:107B80000B4359B29201FB681344C9B2034AD15462
:107B900000BF1437BD465DF8047B7047ACCD0120B3
:107BA00080B487B000AF78607B68FB6000237B61A6
:107BB00057E000233B614EE03B699B01FA681A44A1
:107BC0007B6913441B78002B20D03B69002B00DA23
:107BD0000733DB101A4691017B690B442649CB5CC5
:107BE00059B23B69584203F0070300F0070058BF41
:107BF0004342012000FA03F35BB20B4359B29201F6
:107C00007B691344C9B21C4AD15421E03B69002B63
:107C100000DA0733DB101A4691017B690B441649E1
:107C2000CB5C59B23B69584203F0070300F00700F0
:107C300058BF4342012000FA03F35BB2DB435BB25F
:107C40000B4059B292017B691344C9B20A4AD1541C
:107C50003B6901333B613B691F2BADDD7B69013320
:107C60007B617B693F2BA4DD00BF00BF1C37BD4695
:107C70005DF8047B704700BFACCD012080B485B0B7
:107C800000AF78600023FB6009E07B68D9B2094A45
:107C9000FB6813440A461A70FB680133FB60FB68FB
:107CA000FF2BF2DD00BF00BF1437BD465DF8047B3B
:107CB000704700BFACCD012080B400AF72B600BFEA
:107CC000074B00221A60074B00221A60BFF34F8F48
:107CD00000BF62B600BF00BFBD465DF8047B7047C1
:107CE000ACCE0120B0CE012080B500AF294B1B687F
:107CF000294A52F82320294B1B689A4247DC254B1E
:107D00001B68254A52F82330002B40D0214B5B687A
:107D1000002B16DAFF20FFF7B1FF214B1B685A42F8
:107D200003F03F0002F03F0358BF58421C4B1B6852
:107D3000002B00DA3F339B1101221946FFF7DCFECE
:107D400015E00020FFF79AFF154B1B685A4203F01D
:107D50003F0002F03F0358BF5842114B1B68002BF5
:107D600000DA3F339B1100221946FFF7C5FE0C4B8A
:107D70001B6801330A4A1360094B1B685A42C3F35C
:107D80000A03C2F30A0258BF5342054A136000BFF8
:107D900080BD00BFBC6A00203C580020B0CE01204E
:107DA000ACCE012080B483B000AF00237B6007E03D
:107DB000084A7B68134400221A707B6801337B6099
:107DC0007B68022BF4DD00BF00BF0C37BD465DF8B9
:107DD000047B7047B4CE012090B585B000AF7860C9
:107DE0000023FB737B68022B2BD07B68022B39DCD2
:107DF0007B68002B03D07B68012B11D032E011216E
:107E0000264806F0ABFB0346DBB25B00DCB2102178
:107E1000224806F0A3FB0346DBB22343FB7321E0B9
:107E200004211F4806F09AFB0346DBB25B00DCB27C
:107E300007211B4806F092FB0346DBB22343FB738A
:107E400010E00721174806F089FB0346DBB25B0010
:107E5000DCB20621134806F081FB0346DBB2234364
:107E6000FB7300BF104A7B6813441B7803F00F02BA
:107E7000FB7B0E4992000A44134419780A4A7B6836
:107E800013440A461A70084A7B6813441B7823F08F
:107E90000F03DBB218461437BD4690BD40F00F40CB
:107EA000C0F00F4080F00F40B4CE0120240101004B
:107EB00080B584B000AF78607868FFF78DFF034627
:107EC000FB73FB7B102B09D10C4A7B6852F82330E3
:107ED0005A1C0A497B6841F823200BE0FB7B202BCE
:107EE00008D1064A7B6852F823305A1E03497B6842
:107EF00041F8232000BF1037BD4680BD54580020F4
:107F0000B0B596B000AFAC4B1B680133AA4A136002
:107F1000A94B1B685A4203F0030302F0030258BF47
:107F20005342A54A1360A44B1B68022B40F3B38352
:107F30003B1D00221A605A609A600023FB620023F6
:107F4000BB6200237B6200237B659FE39B4A7B6DC2
:107F500052F823309A497A6D51F822209B1A1A461A
:107F60007B6D9B0007F158010B4443F8542C7B6D4B
:107F70009B0007F15802134453F8543C002B01DDD9
:107F8000012301E04FF0FF333B627B6D9B0007F163
:107F90005802134453F8543C07EE903AF8EEE77A4F
:107FA000F1EE000AB0EE670AF9F78AFB87ED070ADF
:107FB0007B6D012B12D1D7ED077AFDEEE77A17EE34
:107FC000900A07F06AFD02463B6A03FB02F27B6DF2
:107FD0009B0007F158010B4443F8542C774A7B6D02
:107FE00052F823301946764A7B6D42F823107B6D98
:107FF0009B0007F15802134453F8543C002B01D066
:10800000FFF75AFE7B6D022B00F01E817B6D022B69
:1080100000F339837B6D002B04D07B6D012B00F0C6
:10802000298230E3674B1B78002B40F02783664B97
:108030001B68FB627B6D9B0007F15802134453F8E9
:10804000543C002B0DDC7B6D9B0007F15802134460
:1080500053F8543C002B02DA4FF0FF3302E00023C8
:1080600000E001233B61584B1A683B69134404222A
:108070000021184606F084FA0346534A1360524B17
:108080001B68FA6A9A4200F0F982504B196850480E
:10809000FA6A13465B001344DB000B44843350F848
:1080A0002330002B18D1494B19684948FA6A134606
:1080B0005B001344DB000B440C33002240F8232008
:1080C000424B19684348FA6A13465B001344DB00CD
:1080D0000B44002240F823203B4B1B683B65A8E083
:1080E000394AFB6A1360394B1B68FB643FE038492F
:1080F0003A6D13465B001344DB00FA6C13440C33F7
:1081000051F82330002B09D02F4A3B6D13602F4AC2
:10811000FB6C1360304B01221A60BDE20023BB648C
:1081200000237B6410E02A497A6C13465B001344F9
:10813000DB00FA6C13440C3351F82330BA6C13444F
:10814000BB647B6C01337B647B6C042BEBDDBB6C11
:10815000002B09D11C4A3B6D13601C4AFB6C136059
:108160001D4B01221A6097E2FB6C0133FB64FB6C30
:10817000172BBCDD154B1B68013B3B6452E01449D7
:108180003A6D13465B001344DB003A6C13440C3326
:1081900051F82330002B09D00B4A3B6D13600B4A7A
:1081A0003B6C13600C4B01221A6075E20023FB63E9
:1081B0000023BB6323E000BFB8CE01205458002049
:1081C000BCCE012010D10120687000206C7000200E
:1081D000505A00207C700020707000209C49BA6BBF
:1081E00013465B001344DB003A6C13440C3351F824
:1081F0002330FA6B1344FB63BB6B0133BB63BB6B74
:10820000042BEBDDFB6B002B09D1924A3B6D136015
:10821000914A3B6C1360914B01221A603CE23B6C2B
:10822000013B3B643B6C002BA9DA3A6D3B6913447C
:108230003B653B6D042B03DC3B6D002BBFF650AF61
:10824000864B01221A6019E2854B1B78032B16D14D
:10825000814B1B68BB62804B1A687B6D9B0007F1EA
:1082600058010B4453F8543C9B00D31A17220021A9
:10827000184606F085F9B861774ABB691360784BF8
:108280001B78002B40F0FC81734B1B68BB627B6D3D
:108290009B0007F15802134453F8542C6E4B1B6893
:1082A000134417220021184606F06AF978617A69AA
:1082B000BB6A9A4214BF01230023DBB219467B6DCF
:1082C0009B0007F15802134453F8543CDB0FDAB219
:1082D0007B69002B0CBF01230023DBB21340DBB210
:1082E00041EA03027B6D9B0007F158010B4453F8F0
:1082F000543C002BCCBF01230023D9B27B69172B40
:108300000CBF01230023DBB20B40DBB21343002B75
:108310001AD0544B1B68002B12D14E4B1A684C4993
:1083200013465B001344DB00BA6A13440C3351F864
:108330002330002B04D14B4B40F2DC521A60A2E1F7
:10834000484B40F2DC521A60434A7B691360424B4F
:108350001B68BA6A9A4200F09381434B1B6803F58D
:108360008073414A1360404B1B6823F0FF033E4A71
:1083700013603E4B00221A6000237B6300237B6363
:1083800000233B6328E0334B1B683A6B9A4220D0B2
:10839000314B19682E483A6B13465B001344DB00DF
:1083A0000B440C3350F82330002B12D001237B6395
:1083B000294B1B68BA6A9A4205DA274B1B680133BE
:1083C000254A13600BE0244B1B68013B224A1360D3
:1083D00005E03B6B01333B633B6B042BD3DD7B6BD5
:1083E000002BCBDC1C4B1B68172B03DC1A4B1B68C8
:1083F000002B02DA184ABB6A1360164B1A6814493C
:1084000013465B001344DB00BA6A1344843351F80B
:108410002330002B18D10F4B1A680D4913465B000F
:108420001344DB00BA6A13440C33002241F82320C2
:10843000084B1A680E4913465B001344DB00BA6A06
:108440001344002241F82320044B01221A6017E153
:10845000505A0020687000206C700020707000205E
:1084600010D10120FCCB0120747000207870002016
:108470007C70002005218A4806F070F80346002B26
:1084800000F0C880874B1B78002B73D1864B1A688D
:10849000864B1968864813465B001344DB000B4487
:1084A0000C3350F82330002B64D07F4B1A687F4B7D
:1084B00019687F4813465B001344DB000B44843388
:1084C00050F823307B62784B1A68784B19687848EB
:1084D00013465B001344DB000B44843350F8232025
:1084E0007B6D9B0007F158010B4453F8543C134437
:1084F0006D4A14686D4A156863226FF06201184670
:1085000006F03EF802466A4923465B002344DB003E
:108510002B44843341F82320634B1A68634B19685A
:10852000634813465B001344DB000B44843350F86C
:1085300023307A6A9A421DD0FAF7C6F85A4B196866
:108540005A4B1C68584B1A68584B1868584D0B46C4
:108550005B000B44DB002344843355F82310554C57
:1085600013465B001344DB00034444F82310524BD2
:1085700001221A604B4B1B78012B40F083804F4B3C
:10858000DB68002B12D04E4B1A687B6D9B0007F105
:1085900058010B4453F8543C13440522002118465B
:1085A00005F0EEFF0346464A13606BE07B6D9B00CF
:1085B00007F15802134453F8543C002B62D0404B4F
:1085C0005A687B6D9B0007F158010B4453F8543CEB
:1085D000134408226FF00701184605F0D1FF034647
:1085E000374A5360364B5B68002B4BD1344B5A688B
:1085F0007B6D9B0007F158010B4453F8543C134426
:1086000008226FF00701184605F0BAFF03462C4A0E
:10861000536037E0234B1B78022B0FD07B6D9B0000
:1086200007F15802134453F8543C002B2AD01D4B39
:1086300002221A70204B01221A6023E0204B9B6813
:108640007B621F4B9A687B6D9B0007F158010B44BE
:1086500053F8543C13440C220021184605F090FFB7
:108660000346174A9360164B9B687A6A9A4209D070
:10867000FEF70AF9104B01221A6003E000BF02E086
:1086800000BF00E000BF7B6D01337B657B6D022B7B
:108690007FF75CAC00E000BF5837BD46B0BD00BFFF
:1086A00000F00F4010D10120687000206C70002095
:1086B000505A00207C7000207070002008000020BC
:1086C000BC6A002080B582B000AF786039607B68FA
:1086D000002B02D1064804F0F1FD7B681B68396865
:1086E000184601F05FFE034618460837BD4680BDB8
:1086F0004001010080B582B000AF78607B68002B3C
:1087000002D1064804F0DAFD7B681B68184605F0C4
:10871000A6FF034618460837BD4680BD5801010034
:1087200080B582B000AF786039607B68002B02D1E1
:10873000064804F0C3FD7B681B683968184601F0E1
:108740006FFE034618460837BD4680BD7001010024
:1087500080B58EB000AF78607B68002B02D11A48DC
:1087600004F0ACFD07F12C0300221A605A6007F1F7
:108770000C0320220021184607F024F800237B6315
:108780000C23FB6000233B6103233B7502237B75B5
:108790000E4BBB6207F10C033B630023FB627B685B
:1087A0001B6807F12C021146184605F0F1FF7863AB
:1087B0007B6B002B02D040F2097300E000231846C7
:1087C0003837BD4680BD00BF880101000800F9FFB1
:1087D00080B586B000AFF860B9607A60BB68002BE6
:1087E00002D1134804F06AFDFB681B68B96818469B
:1087F00005F0CEFF78617B69002B10D0BB681B6849
:10880000002B02D0F868FFF7A3FF7B68002B08D08D
:108810007B68013B7B607B69002BE5D102E000BFF8
:1088200000E000BF7B6918461837BD4680BD00BF19
:10883000A001010080B58EB000AF78607B68002B8E
:1088400002D11E4804F03AFD07F12C0300221A6001
:108850005A6007F10C0320220021184606F0B2FFEF
:1088600000237B630D23FB607B685B6A1B043B6119
:1088700001237B7507F10C033B630023FB6207F1C7
:108880002C03032219467868FFF7A2FF78637B6BFD
:10889000002B0BD1BB6903F48073002BEAD0BB69BA
:1088A0005B0A03F00F03072B02D1E3E700BF00E0F0
:1088B00000BF7B6B18463837BD4680BDB80101004C
:1088C00080B594B000AF786039607B68002B02D12E
:1088D000314804F0F3FC07F13C0300221A605A60AF
:1088E00007F11C0320220021184606F06BFF07F158
:1088F000080300221A605A609A60DA601A61002345
:10890000FB647B683033BB6404220021B86C06F042
:1089100059FF7868FFF78EFF0346002B02D04FF413
:10892000E36335E07B685B6A19467868FFF7CAFE47
:108930000346002B02D040F2157329E01623FB6199
:10894000012387F825300423FB6001233B61BB6CC6
:108950007B6107F11C033B6407F10803FB637B6841
:108960001B6807F13C021146184605F011FFF86438
:10897000FB6C002B0BD1BA6A084B1340002B06D1BD
:10898000BB6C1B687B647B6C1ABA3B681A60FB6C1F
:1089900018465037BD4680BDD00101000800F9FFE0
:1089A00080B58EB000AF78607B68002B02D118488C
:1089B00004F084FC07F12C0300221A605A6007F1CE
:1089C0000C0320220021184606F0FCFE00237B63E6
:1089D0000323FB6000233B6108237B7507F10C0335
:1089E0003B630023FB627B681B6807F12C02114686
:1089F000184605F0CDFE78637B6B002B03D1BB6975
:108A00001A0C7B685A627B6B18463837BD4680BDAE
:108A1000E801010080B594B000AFF860B9607A60F9
:108A20003B60FB68002B02D12A4804F047FCBB6D79
:108A3000002B02D1284804F041FC07F14403002236
:108A40001A605A6007F1240320220021184606F01C
:108A5000B9FE07F1100300221A605A609A60DA60CA
:108A60001A610023FB6406237B62BB68DB0763F0AB
:108A70007F43BB62BA6A7B689B000F2101FA03F354
:108A8000DB431340BB62BA6A7B689B00396801FA1A
:108A900003F31343BB62012387F82D3040237B612E
:108AA0000123BB61BB6DFB6107F12403BB6407F1CC
:108AB00010037B64FB681B6807F1440211461846EB
:108AC00005F066FEF864FB6C002BFB6C1846503713
:108AD000BD4680BD000201001802010080B584B0CF
:108AE00000AF786039607B68002B02D1584804F0F1
:108AF000E5FB3B68002B02D1564804F0DFFB7B68A6
:108B000003F51A73FB603B681B681B0FDAB2FB6846
:108B10001A703B681B681B0EDBB203F00F03DAB25E
:108B2000FB685A703B681B68DB0DDBB203F0010386
:108B3000DBB2002B06D0FB685B8843F001039AB2DE
:108B4000FB685A803B681B681B0DDBB203F0070310
:108B5000DAB2FB681A713B681B681B0CDBB203F0CE
:108B60000F03DAB2FB685A713B681B68DB0BDBB2A0
:108B700003F00103DBB2002B06D0FB685B8843F0F7
:108B800002039AB2FB685A803B681B689B0ADBB2FF
:108B900003F01E03DAB2FB689A713B681B68DBB214
:108BA00003F00303DAB2FB68DA713B685A68FB68CA
:108BB0009A60FB685B78022B0ED0022B1ADC002B2C
:108BC00002D0012B04D015E07B6801229A6214E0E8
:108BD0007B6802229A6210E07B6804229A627B68BA
:108BE000B3F86A3203F00203002B05D07B68082239
:108BF0009A6201E000BF00E000BF7B6893F86D322D
:108C000003F00403002B05D07B68DB6A43F0040209
:108C10007B68DA627B6893F86F3203F00103002B04
:108C200005D07B68DB6A43F080027B68DA627B6890
:108C300093F86F3203F00203002B05D07B68DB6AE8
:108C400043F040027B68DA6200BF1037BD4680BD4A
:108C5000300201004802010080B59AB000AF786090
:108C60007B68002B02D1484804F028FB07F1400341
:108C700000221A605A6007F12003202200211846C2
:108C800006F0A0FD07F10C0300221A605A609A60FA
:108C9000DA601A617B6830337B6600233B6608220A
:108CA0000021786E06F08EFD7B685B6A1946786855
:108CB000FFF708FD0346002B02D040F215735EE07B
:108CC00033233B62012387F8293000237B6208238A
:108CD0003B6101237B617B6EBB6107F10C033B644D
:108CE00007F120037B647B681B6807F14002114693
:108CF000184605F04DFD38663B6E002B3ED1FA6AF2
:108D0000224B1340002B39D17B681B685B7A022B06
:108D100006D0022B2ADC002B2BD0012B11D025E012
:108D20007B6E1B68BB65BB6D1ABA7B6E1A607B6E6F
:108D300004331A687B6E0433FA65FA6D12BA1A604E
:108D400018E07B6E1B68FB64FB6C5BBABB64BA6C9F
:108D50007B6E1A607B6E04331A687B6E04337A650F
:108D60007A6D52BA3A653A6D1A6003E04FF4E163E6
:108D700005E000BF796E7868FFF7B0FE3B6E1846DD
:108D80006837BD4680BD00BF600201000800F9FFE2
:108D900080B5A0B002AFF860B9607A60FB68002BC4
:108DA00002D1974804F08AFAFB6830337B6707F1F9
:108DB000100300221A605A609A6000233B67402229
:108DC0000021786F06F0FEFCFB689B6A012B06D938
:108DD000FB68B3F8503203F48063002B02D14FF4E8
:108DE000E16329E17B6F00937B68BA680021F86832
:108DF000FFF710FE0346002B02D040F209731BE17F
:108E0000FB681B685B7A022B06D0022B66DC002B0A
:108E100067D0012B2CD061E07B6F1B68FB65FB6D7D
:108E20001ABA7B6F1A607B6F04331A687B6F043346
:108E30003A663A6E12BA1A607B6F08331A687B6F13
:108E400008337A667A6E12BA1A607B6F0C331A682E
:108E50007B6F0C33BA66BA6E12BA1A607B6F10332E
:108E60001A687B6F1033FA66FA6E12BA1A6039E02C
:108E70007B6F1B68BB63BB6B5BBA7B637A6B7B6F7F
:108E80001A607B6F04331A687B6F04333A643A6C60
:108E900052BAFA63FA6B1A607B6F08331A687B6FF9
:108EA0000833BA64BA6C52BA7A647A6C1A607B6F0F
:108EB0000C331A687B6F0C333A653A6D52BAFA6418
:108EC000FA6C1A607B6F10331A687B6F1033BA65C7
:108ED000BA6D52BA7A657A6D1A6003E04FF4E163B5
:108EE000AAE000BF7B6F1B689BB27B837B6F043360
:108EF0001B681B0C9BB23B837B6F04331B689BB2CC
:108F0000FB827B6F08331B681B0C9BB2BB827B6FA1
:108F100008331B689BB27B827B6F0C331B681B0C76
:108F20009BB23B827B6F0C331B681B029AB27B6F38
:108F300010331B681B0E13433B67BB685B0007F1D4
:108F40007802134433F8683C1A467B6842FA03F30C
:108F500003F00103002B09D0BB689B003A6F22FA93
:108F600003F303F00F037A689A4202D04FF4E163EF
:108F700062E07B6F00937B68BA680121F868FFF7B5
:108F800049FD0346002B02D040F2097354E0FB6810
:108F90001B685B7A022B06D0022B2EDC002B31D013
:108FA000012B13D029E07B6F0C331A687B6F0C33D5
:108FB000FA62FA6A12BA1A607B6F10331A687B6F12
:108FC00010333A633A6B12BA1A601CE07B6F0C33B1
:108FD0001A687B6F0C333A623A6A52BAFA61FA69DC
:108FE0001A607B6F10331A687B6F1033BA62BA6AEB
:108FF00052BA7A627A6A1A6005E04FF4E1631BE0C4
:109000007802010000BF7B6F0C331B681B029AB211
:109010007B6F10331B681B0E13433B67BB689B00C1
:109020003A6F22FA03F303F00F037A689A4202D0F0
:1090300040F2167300E0002318467837BD4680BD25
:1090400080B58EB000AF786039607B68002B02D1AC
:10905000224804F033F907F12C0300221A605A6009
:1090600007F10C0320220021184606F0ABFB002379
:109070007B637B685B6A19467868FFF723FB0346CE
:10908000002B02D040F2157323E00623FB6001237E
:109090007B753B68002B03D03B68012B03D005E0B8
:1090A00000233B6104E002233B6101E0042310E064
:1090B00007F10C033B630023FB627B681B6807F12D
:1090C0002C021146184605F063FB78637B6B002B7E
:1090D0007B6B18463837BD4680BD00BF900201004B
:1090E00080B584B000AF786039607B68002B02D116
:1090F0008D4804F0E3F83B68002B02D18B4804F064
:10910000DDF87B6803F51373FB603B680C331B6869
:109110009B0FDAB2FB681A703B680C331B681B0CA0
:10912000DAB2FB685A703B680C331B681B0ADAB270
:10913000FB689A703B680C331B68DAB2FB68DA7024
:109140003B6808331B681B0D9AB2FB689A803B682A
:1091500008331B681B0CDBB203F00F03DAB2FB68A9
:109160009A713B6808331B6803F40043002B06D058
:10917000FB681B8943F001039AB2FB681A813B68C4
:1091800008331B6803F48043002B06D0FB681B895F
:1091900043F001039AB2FB681A813B6808331B68ED
:1091A00003F40053002B06D0FB681B8943F0040333
:1091B0009AB2FB681A813B6808331B6803F480533A
:1091C000002B06D0FB681B8943F008039AB2FB68AA
:1091D0001A81FB681B78002B02D0012B79D0A8E004
:1091E0003B6808331B689A0040F6FC731340FA682A
:1091F000D360FB68DA683B6804331B689B0F1A4333
:10920000FB68DA603B6804331B68DB0EDBB203F0FB
:109210000703DAB2FB681A743B6804331B681B0E41
:10922000DBB203F00703DAB2FB685A743B6804331D
:109230001B681B0DDBB203F00E03DAB2FB689A74F5
:109240003B6804331B689B0CDBB203F00703DAB204
:10925000FB68DA743B6804331B68DB0BDBB203F09A
:109260000703DAB2FB681A75FB68DB685A1CFB68F7
:109270001B7D02339A407B68C3F88822FB689B7988
:109280001A46012303FA02F27B68C3F88C227B683A
:10929000D3F88C32B3F5007F4AD07B68D3F888329C
:1092A0007A68D2F88C2202FB03F27B68C3F888222A
:1092B0007B684FF40072C3F88C227B68D3F8882255
:1092C0007B68D3F88C32B2FBF3F27B68C3F8882258
:1092D0002EE07B684FF40072C3F88C223B680833A1
:1092E0001B681B0403F47C12FB68DA60FB68DA6815
:1092F0003B6804331B681B0C1A43FB68DA60FB688D
:10930000DB684FF6FE72934205D97B68DB6A43F057
:1093100010027B68DA62FB68DB6801339A027B68C3
:10932000C3F8882205E000BFA8020100C0020100C6
:1093300000BF3B6804331B689B0BDBB203F00103E7
:10934000DBB2002B06D0FB681B8943F010039AB2F6
:10935000FB681A813B6804331B68DB09DBB203F04E
:109360007F03DAB2FB685A753B6804331B68DBB2D3
:1093700003F07F03DAB2FB689A753B681B689B0EAB
:10938000DBB203F00703DAB2FB68DA753B681B68EF
:109390009B0DDBB203F00F03DAB2FB681A763B6871
:1093A0001B685B0DDBB203F00103DBB2002B06D0C0
:1093B000FB681B8943F040039AB2FB681A813B6843
:1093C0001B68DB0BDBB203F00103DBB2002B06D022
:1093D000FB681B8943F080039AB2FB681A813B68E3
:1093E0001B689B0BDBB203F00103DBB2002B06D042
:1093F000FB681B8943F480739AB2FB681A813B684F
:109400001B685B0BDBB203F00103DBB2002B06D061
:10941000FB681B8943F400739AB2FB681A813B68AE
:109420001B681B0BDBB203F00103DBB2002B06D081
:10943000FB681B8943F480639AB2FB681A813B681E
:109440001B689B0ADBB203F00303DAB2FB685A76AF
:1094500000BF1037BD4680BD80B58EB000AF7860CC
:109460007B68002B02D1214803F028FF07F12C0371
:1094700000221A605A6007F10C03202200211846CE
:1094800006F0A0F900237B630923FB607B685B6A1D
:109490001B043B6103237B7507F10C033B63002333
:1094A000FB627B681B6807F12C021146184605F029
:1094B0006FF978637B6B002B10D17B6803F1300070
:1094C00007F10C030C331022194606F079F97B687A
:1094D000303319467868FFF703FE02E040F2097363
:1094E0007B637B6B18463837BD4680BDD8020100D0
:1094F00080B584B000AF786039607B68002B02D102
:109500002E4803F0DBFE3B68002B02D12C4803F011
:10951000D5FE7B6803F50E73FB603B680C331B685C
:109520001B0EDAB2FB681A703B680C331B681B0A0F
:109530009AB2FB685A803B680C331B68DAB2FB684E
:109540001A713B6808331B681B0EDAB2FB685A714C
:109550003B6808331B681B0CDAB2FB689A713B68E6
:1095600008331B681B0ADAB2FB68DA713B68083300
:109570001B68DAB2FB681A723B6804331B681B0E67
:10958000DAB2FB685A723B6804331B681A02FB6844
:10959000DA60FB68DA683B681B681B0E1A43FB68DD
:1095A000DA603B681B681B0A9BB2C3F30B039AB2D9
:1095B000FB681A8200BF1037BD4680BDF002010073
:1095C0000803010080B58CB000AF78607B68002B89
:1095D00002D11E4803F072FE07F1280300221A6030
:1095E0005A6007F1080320220021184606F0EAF825
:1095F0000223BB600023FB6003237B7407F1080395
:10960000FB620023BB627B681B6807F128021146DE
:10961000184605F0BDF80346002B11D17B6803F115
:10962000300007F108030C331022194606F0C8F881
:109630007B68303319467868FFF75AFF002301E052
:1096400040F2097318463037BD4680BD2003010043
:1096500080B58EB000AF786039607B68002B02D196
:10966000304803F02BFE07F1280300221A605A60ED
:1096700007F1080320220021184606F0A3F8012371
:109680007B6364233B632923BB603B68FB6004234B
:109690007B743DE000217868FFF714F80346002B47
:1096A00000D035E007F10803FB620023BB627B6852
:1096B0001B6807F128021146184605F069F878631F
:1096C0007B6B002B02D040F2097327E07B69002BF3
:1096D0001BDA7B6903F08043002B05D07B68DB6AD3
:1096E00043F002027B68DA627B6903F08073002B2F
:1096F00005D07B68DB6A43F020027B68DA627A6916
:109700007B68C3F83422002308E00A2000F0BCFE86
:109710003B6B5A1E3A63002BBCD17B6B1846383723
:10972000BD4680BD3803010080B58EB000AF7860C3
:109730007B68002B02D1214803F0C0FD07F128030C
:1097400000221A605A6007F10803202200211846FF
:1097500006F038F80A237B6300233B630823BB60D1
:109760004FF4D573FB6009237B7407F10803FB6298
:109770000023BB627B681B6807F12802114618466C
:1097800005F006F838633B6B002B09D17B69DBB22F
:10979000AA2B03D040F20C733B6301E000233B6330
:1097A0007B6B013B7B637B6B002B02D03B6B002B05
:1097B000E0D13B6B18463837BD4680BD50030100F1
:1097C00080B584B000AF78607B68002B02D132484E
:1097D00003F074FD40F21B73FB607B6893F89332D7
:1097E000032B28D0012200217868FFF7D1FAF86016
:1097F000FB68002B19D17B68012283F890227B68DB
:109800001A687B685B69002B06D07B685B6923491B
:109810008B4228BF0B4600E0204B1946104604F04F
:10982000F6FE02467B681A6230E0FB68B3F5E16F32
:109830002CD100232BE07B6893F89032012B22D8A7
:10984000012200217868FFF7A3FAF860FB68002B7B
:109850001BD17B68012283F890227B681A687B68A1
:109860005B69002B06D07B685B690C498B4228BF83
:109870000B4600E0094B1946104604F0C8FE0246AC
:109880007B681A6201E000BF00E000BFFB68184679
:109890001037BD4680BD00BF6803010080F0FA02AA
:1098A00080B582B000AF786039607B68002B02D150
:1098B0003E4803F003FD3B68002B02D13C4803F017
:1098C000FDFC3B681B689B0FDAB27B6883F874224F
:1098D0003B681B685B0FDBB203F00103DAB27B6805
:1098E00083F875223B681B689AB27B68A3F87622DE
:1098F0003B685A687B68C3F878223B6808331B686A
:109900001B0EDAB27B6883F87C223B6808331B6845
:109910001B0CDAB27B6883F87D223B6808331B6836
:109920001B0BDBB203F00F03DAB27B6883F87E22F5
:109930003B6808331B689BB21B029AB23B680C332E
:109940001B681B0E9BB213439AB27B68A3F880225C
:109950003B680C331B681B0CDBB29B08DAB27B68DC
:1099600083F882223B680C331B681B0CDBB203F0CC
:109970000303DAB27B6883F883223B680C331B68ED
:109980001B0ADBB21B09DAB27B6883F884223B68CE
:109990000C331B681B0ADBB203F00F03DAB27B68DF
:1099A00083F8852200BF0837BD4680BD80030100D3
:1099B0009803010080B598B000AF78607B68002BF9
:1099C00002D1534803F07AFC0023FB6507F1400302
:1099D00000221A605A6007F1200320220021184655
:1099E00005F0F0FE07F10C0300221A605A609A603D
:1099F000DA601A610023BB657B6830337B654022E7
:109A00000021786D05F0DEFE7868FEF713FF03464F
:109A1000002B02D04FF4E36375E07B685B6A194664
:109A20007868FEF74FFE0346002B02D040F2157314
:109A300069E00D233B62012387F8293040233B6115
:109A400001237B617B6DBB6107F120037B6407F120
:109A50000C033B647B681B6807F140021146184603
:109A600004F096FEB865BB6D002B04D1FA6A294B51
:109A70001340002B02D040F2097344E07B681B685E
:109A80005B7A022B06D0022B34DC002B35D0012B65
:109A900017D02FE00023FB650FE0FB6D9B007A6D74
:109AA00013441A68FB6D9B00796D0B443A653A6D5F
:109AB00012BA1A60FB6D0133FB65FB6D0F2BECD9FD
:109AC0001CE00023FB6511E0FB6D9B007A6D1344E5
:109AD0001A68FB6D9B00796D0B44FA64FA6C52BAFC
:109AE000BA64BA6C1A60FB6D0133FB65FB6D0F2B1A
:109AF000EAD903E04FF4E16305E000BF796D7868CF
:109B0000FFF7CEFE002318466037BD4680BD00BF7C
:109B1000B00301000800F9FF80B582B000AF7860A3
:109B20000B46FB707B68002B02D1084803F0C6FB94
:109B30007B6818687B685B6AFA78194600F0F2FB6C
:109B4000034618460837BD4680BD00BFC803010064
:109B500080B594B000AFF860B9607A603B60FB6894
:109B6000002B02D1404803F0A9FBBB68002B02D1B7
:109B70003E4803F0A3FBBB6D002B02D13C4803F031
:109B80009DFB3B68B3F5007F02D03A4803F096FB9B
:109B900007F1480300221A605A6007F128032022C7
:109BA0000021184605F00EFE07F1140300221A608A
:109BB0005A609A60DA601A61FB68DB6A03F002039C
:109BC000002B03D03B68B3F5007F0ED1FB68D3F8C0
:109BD0008C323A689A4208D83B68B3F5805F04D863
:109BE0003B6803F00303002B02D040F20C7337E014
:109BF000F868FEF71FFE0346002B02D04FF4E36324
:109C00002EE03B68BB61BB6DFB61BB683B6201231F
:109C10003B75BB6D012B01D1112300E01223BB6208
:109C20007B68FB62FB68DB6A03F00203002B04D154
:109C3000FB6ABA6902FB03F3FB62012387F8313048
:109C40000D4B7B6407F12803FB6407F11403BB642D
:109C500007F1480303221946F868FEF7B9FD0346E9
:109C600018465037BD4680BDE0030100F8030100EF
:109C7000100401002C0401000800F9FF80B594B025
:109C800000AFF860B9607A603B60FB68002B02D1DE
:109C90004F4803F013FBBB68002B02D14D4803F083
:109CA0000DFBBB6D002B02D14B4803F007FB3B685B
:109CB000B3F5007F02D0494803F000FB07F14403ED
:109CC00000221A605A6007F124032022002118465E
:109CD00005F078FD07F1100300221A605A609A60BF
:109CE000DA601A61FB68DB6A03F00203002B03D021
:109CF0003B68B3F5007F0ED1FB68D3F88C323A682D
:109D00009A4208D83B68B3F5805F04D83B6803F0FB
:109D10000303002B02D040F20C7354E0F868FEF706
:109D200089FD0346002B02D04FF4E3634BE000BFF4
:109D3000FB681B68184604F07CFC0346002BF7D137
:109D400001233B743B687B61012387F82D30244B52
:109D50003B64BB6D012B01D1182300E019237B620A
:109D60007B68BB62FB68DB6A03F00203002B04D153
:109D7000BB6A7A6902FB03F3BB62FB6DBA6D1A60C2
:109D8000BB6DBB61BB683B6207F12403BB6407F199
:109D900010037B6407F1440303221946F868FEF7B9
:109DA00017FDF864FB6C002B0CD0F96DF868FEF71A
:109DB00087FD0346002B05D1FB6D1B68002B01D0EE
:109DC0000023FB64FB6C18465037BD4680BD00BFC6
:109DD000680401008004010098040100B40401003B
:109DE0000800F9FF80B582B000AF78607B68002B77
:109DF00002D10D4803F062FA7B68B3F8543203F4E1
:109E00000073002B06D17B68B3F8543203F48063EF
:109E1000002B01D0012300E0002303F00103DBB29B
:109E200018460837BD4680BDF004010080B58CB0EF
:109E300002AFF860B9607A603B60FB68002B02D12A
:109E4000484803F03BFABB68002B02D1464803F0B8
:109E500035FA3B68002B02D1444803F02FFA3A68E8
:109E60007B681A44FB68D3F888329A4202D940488A
:109E700003F024FA0023FB61BB687B610123FB76BE
:109E8000FB68303323F0030304333B613B683B62E0
:109E90005FE0FB695B02BA6813447B61FB685B7F30
:109EA00083F00103DBB2002B15D0FB7E83F00103AE
:109EB000DBB2002B04D17B6903F00303002B0AD033
:109EC00001237B624FF400720021386905F07AFCAF
:109ED0000023FB7610E03B6AB3F5803F08D33B6A72
:109EE000A3F57F43FF3B3B624FF6FF737B6203E0CA
:109EF0003B6A7B6200233B62FB7E002B01D07969C9
:109F000000E039697A68FB691A447B6A00934FF470
:109F10000073F868FFF71CFE0346002B02D040F2E6
:109F200009731AE0FA697B6A1344FB61FB685B7F83
:109F300083F00103DBB2002B0BD0FB7E83F0010327
:109F4000DBB2002B05D04FF400723969786905F057
:109F500037FC3B6A002B9CD1002318462837BD46AE
:109F600080BD00BF08050100200501003805010083
:109F70005405010080B58CB002AFF860B9607A601A
:109F80003B60FB68002B02D1494803F097F9BB689E
:109F9000002B02D1474803F091F93B68002B02D116
:109FA000454803F08BF93A687B681A44FB68D3F89C
:109FB00088329A4202D9414803F080F900237B623B
:109FC00000233B6100233B620123FB77FB683033B6
:109FD00023F003030433BB613B683B625FE03A68F4
:109FE0003B6AD31A5B02BA6813447B61FB685B7FF0
:109FF00083F00103DBB2002B15D0FB7F83F001035C
:10A00000DBB2002B04D17B6903F00303002B0AD0E1
:10A0100001237B624FF400727969B86905F0D0FBC7
:10A020000023FB7709E03B6AB3F5803F03D34FF68B
:10A03000FF737B6201E03B6A7B62FB7F002B01D0F8
:10A04000796900E0B9697A683B681A443B6AD21AB8
:10A0500007F1100301937B6A00934FF40073F868D3
:10A06000FFF70CFE0346002B02D040F209731AE002
:10A070003B693A6AD31A3B62FB685B7F83F001035A
:10A08000DBB2002B0BD0FB7F83F00103DBB2002B94
:10A0900005D04FF400720021B86905F093FB3B6ACC
:10A0A000002B9CD1002318462837BD4680BD00BF39
:10A0B00094050100AC050100C4050100E0050100A4
:10A0C00080B584B000AF78607B68002B02D1224855
:10A0D00003F0F4F80023FB600023BB60FB6843F44B
:10A0E0004813FB607B68012283F893227868FEF7AF
:10A0F00001FB0346002B03D040F21373BB6026E044
:10A100007868FFF711FB0346002B0AD1FB6843F088
:10A110008043FB607B68DB6A43F008027B68DA629D
:10A1200009E07868FEF7E6FA0346002B03D040F218
:10A130001373BB600BE0F9687868FFF789FA034690
:10A14000002B03D040F21473BB6000E000BFBB687B
:10A1500018461037BD4680BD2006010080B582B08C
:10A1600000AF78607B68002B02D14A4803F0A6F864
:10A170007B681B7F012B02D0474803F09FF87B6868
:10A180000022DA627B681B680021184604F049FB54
:10A190007B681B684149184604F039FA02467B681F
:10A1A0001A627B681B68184604F023FA7868FFF788
:10A1B00087FF034640F22A72934202D140F22A738B
:10A1C00064E07868FFF7FEF90346002B02D040F206
:10A1D0000D735BE07868FEF7E3FB0346002B02D0CB
:10A1E00040F20E7352E07868FFF736F90346002B11
:10A1F00002D040F20F7349E001217868FFF78CFC30
:10A200000346002B02D04FF4E2633FE07B681B68FB
:10A210002349184604F0FBF902467B681A62786805
:10A22000FEF71AFD0346002B02D040F211732DE019
:10A230007B68DB6A03F00403002B0FD001217868F0
:10A24000FEF7FEFE0346002B02D040F212731DE023
:10A250007B681B680121184604F0E3FA4FF4007193
:10A260007868FEF75DFA0346002B02D040F20A73CD
:10A270000CE07868FFF7A4FA0346002B02D040F206
:10A280001B7303E07868FFF795FB00231846083737
:10A29000BD4680BD3806010050060100801A060048
:10A2A00040787D0180B582B000AF78607B68002B7C
:10A2B00002D11A4803F002F87B681B69002B02D117
:10A2C000174802F0FBFF7B681B7F83F00103DBB2C2
:10A2D000002B09D07B681B68184600F0E9F803469C
:10A2E000002B01D0012315E07B681B691B78012B33
:10A2F00004D07B681B691B78022B07D17B681A6826
:10A300007B681B691946104604F021FA7B6801221C
:10A310001A77002318460837BD4680BD7C06010029
:10A320009406010080B58EB000AFF860B9601346A6
:10A33000FB7107F1300300221A605A6007F1100325
:10A3400020220021184605F03DFA07233B61FB79E6
:10A35000002B05D0BB681B047B6101237B7603E0E7
:10A3600000237B6100237B7607F110037B630023CE
:10A370003B6307F130031946F86804F009FA034615
:10A38000002B04D1FA69064B1340002B02D040F297
:10A39000097300E0002318463837BD4680BD00BF72
:10A3A0000800F9FF80B58CB000AF7860396007F124
:10A3B000280300221A605A6007F1080320220021B6
:10A3C000184605F0FFF93723BB603B681B04FB60B0
:10A3D00001237B7407F10803FB620023BB6207F1D2
:10A3E00028031946786804F0D3F90346002B04D1FA
:10A3F0007A690A4B1340002B02D040F2097308E03F
:10A400007B6903F02003002B02D140F20C7300E0C3
:10A41000002318463037BD4680BD00BF0800F9FF55
:10A4200080B58CB000AF7860396007F12803002256
:10A430001A605A6007F1080320220021184605F02F
:10A44000C1F91023BB603B68FB6001237B7407F1FB
:10A450000803FB620023BB6207F1280319467868F2
:10A4600004F096F90346002B04D17A69054B13409A
:10A47000002B02D040F2097300E000231846303769
:10A48000BD4680BD0800F9FF80B582B000AF78609E
:10A490007B684FF47A7202FB03F30449184600F01C
:10A4A000B7FD00BF0837BD4680BD00BF000E2707BF
:10A4B00080B584B000AF78607B68002B02D1124871
:10A4C00002F0FCFE7B689B6D002B02D10F4802F06E
:10A4D000F5FE7B68FB60FB6802225A72FB68022271
:10A4E0009A72FB688022DA60FB6880221A61FB683E
:10A4F0001A68FB6808331946104601F06DFC00230A
:10A5000018461037BD4680BDC0060100E8060100B0
:10A5100080B584B000AF78600023FB6009E00D4A8D
:10A52000FB6852F823307A689A4206D0FB68013300
:10A53000FB60FB68012BF2D900E000BFFB68012B38
:10A5400002D9054802F0BAFEFB6818461037BD462E
:10A5500080BD00BF180701002807010080B584B046
:10A5600000AF786039603B68002B02D13C4802F0B4
:10A57000A5FE7868FFF7CCFF03463A4A52F823302D
:10A58000184604F068F93B685B7803F003023B6807
:10A590001B799B0003F00C031343FB603B685B7962
:10A5A000042B03D0FB6843F01003FB603B68DB78AF
:10A5B0005B0103F06003FA681343FB603B68DB79DF
:10A5C000002B03D0FB6843F08003FB607B68FA68D4
:10A5D0009A607B68DB6823F00F03FB603B685B7964
:10A5E000042B06D03B685B7903F00303FA6813433E
:10A5F000FB603B689B79002B03D0FB6843F00403AE
:10A60000FB603B689B78002B03D0FB6843F008039A
:10A61000FB607B68FA68DA607B681B6A23F00303DF
:10A62000FB603B681B7803F00303FA681343FB608D
:10A630007B68FA681A623B681B7A002B06D07B683D
:10A640005B6A43F008027B685A6205E07B685B6ADC
:10A6500023F008027B685A6200BF1037BD4680BDF8
:10A66000600701002007010080B586B000AFF860E8
:10A67000B9607A60BB68012B02D9134802F01EFE54
:10A680007B68002B02D1114802F018FE7B681B6822
:10A6900003F01F037B617B685B79002B03D07B6930
:10A6A00043F020037B617B681B79002B03D07B691F
:10A6B00043F040037B61FB68BA68796943F8221074
:10A6C00000BF1837BD4680BD84070100B4070100F4
:10A6D00080B584B000AF786039603B68012B02D947
:10A6E0000A4802F0EBFD0023FB607B683A6853F8F0
:10A6F000223003F08003002B03D0FB6843F080037B
:10A70000FB60FB6818461037BD4680BDD8070100C6
:10A7100080B483B000AF7860084B1B6823F44022FC
:10A720007B689B0403F44023044913430B6000BF80
:10A730000C37BD465DF8047B704700BF00700440D5
:10A7400080B483B000AF78600B4B03F580530433C3
:10A750001B6823F440327B681B0403F44033064932
:10A760001A4301F5805304331A6000BF0C37BD460D
:10A770005DF8047B704700BF0070044080B582B074
:10A7800000AF174B1B7BDBB203F00303022B1CD083
:10A79000022B1DD8002B02D0012B0BD018E0114B3F
:10A7A0001B68002B02D1104802F088FD0D4B1B687E
:10A7B0007B6010E00D4B1B68002B02D10C4802F0AF
:10A7C0007DFD0A4B1B687B6005E00A4B7B6002E065
:10A7D00000237B6000BF7B6818460837BD4680BDFC
:10A7E00000400640C8CE012008080100CCCE012060
:10A7F00030080100006CDC0280B582B000AFFFF7CA
:10A80000BDFF7860254B1B78DBB2DB08DBB203F0C1
:10A810000703FB70FB787A6822FA03F37B601F4B17
:10A820005B78DBB21B09DBB203F00303BB701B4B8D
:10A830001B7BDBB203F003037B70BB78002B02D0E1
:10A840007B78002B02D07B78022B21D1FB78072B61
:10A8500014D0072B19DC052B02DC002B03DA14E0E3
:10A86000062B04D011E07B685B097B6011E07B68FC
:10A870000B4AA2FB03231B097B600AE07B68094AA1
:10A88000A2FB0323DB087B6003E000237B6000E086
:10A8900000BF7B6818460837BD4680BD00400640B3
:10A8A000CDCCCCCCABAAAAAA80B483B000AF0E4B5F
:10A8B0009B79DBB203F00103002B03D10B4B1B6828
:10A8C0007B600AE00A4B1A68074B1B7ADBB25B0815
:10A8D00003F0070322FA03F37B607B6818460C370A
:10A8E000BD465DF8047B704700400640605800207C
:10A8F0006458002080B582B000AF094B9B79DBB271
:10A9000003F01003002B03D1FFF776FF786002E01D
:10A91000044B1B687B607B6818460837BD4680BDCA
:10A92000004006406058002080B485B000AF7860D9
:10A930007B6849F69702934202D80023FB7308E034
:10A940007B68074A934202D80123FB7301E002238C
:10A95000FB73FB7B18461437BD465DF8047B7047DC
:10A9600000127A0080B582B000AF0C4B1B78DBB2CE
:10A970005BB2002B0ADA0A4B1B68002B02D1094894
:10A9800002F09CFC064B1B687B6001E000237B60AF
:10A990007B6818460837BD4680BD00BF00500640A2
:10A9A000C8CE01205808010080B582B000AF184B16
:10A9B0001B689B0C03F00303032B1DD0032B1FD834
:10A9C000002B02D0022B0CD01AE0FFF7CBFF03467E
:10A9D000B3F5004F02D14FF4004300E000237B6049
:10A9E00011E00C4B1B68002B02D10B4802F066FCF7
:10A9F000084B1B687B6006E04FF47A737B6002E0D3
:10AA000000237B6000BF7B6818460837BD4680BDC9
:10AA100000700440CCCE01207808010080B582B0DF
:10AA200000AF124B03F5805304331B681B0C03F07B
:10AA30000303032B0ED0032B0FD8002B02D0012BC6
:10AA400004D00AE000F008F9786009E000F05EF94F
:10AA5000786005E0064B7B6002E000237B6000BF6E
:10AA60007B6818460837BD4680BD00BF00700440B3
:10AA7000006CDC0280B584B000AF0346FB71FB794B
:10AA8000132B00F28E8001A252F823F0DDAA000001
:10AA9000DDAA0000FDAA00001DAB00003DAB0000D8
:10AAA000A3AB00005DAB000065AB00006DAB000028
:10AAB000A3AB0000A3AB000075AB00007DAB0000B2
:10AAC00085AB00008DAB0000A3AB0000A3AB000082
:10AAD000A3AB000095AB00009BAB000000F08AF830
:10AAE0000246344B03F5825304331B681B0F03F0FB
:10AAF0000F030133B2FBF3F3FB6055E000F07AF88B
:10AB000002462C4B03F5825304331B681B0E03F0E3
:10AB10000F030133B2FBF3F3FB6045E000F06AF88A
:10AB20000246244B03F5825304331B681B0D03F0CC
:10AB30000F030133B2FBF3F3FB6035E000F05AF88A
:10AB400002461C4B03F5825304331B681B0C03F0B5
:10AB50000F030133B2FBF3F3FB6025E0FFF75EFF69
:10AB6000F86021E0FFF720FFF8601DE0FFF7FAFE34
:10AB7000F86019E003F0B8FFF86015E000F0AEF8F7
:10AB8000F86011E000F068F8F8600DE000F0BEF841
:10AB9000F86009E0084BFB6006E04FF47A73FB6055
:10ABA00002E00023FB6000BFFB6818461037BD467B
:10ABB00080BD00BF00700440006CDC0280B582B034
:10ABC00000AF78600A497B685A6801F58253043304
:10ABD0001A607B681B781846FFF7B2FD7B685B78CC
:10ABE0001846FFF795FD00BF0837BD4680BD00BF82
:10ABF0000070044080B582B000AF164B9B79DBB289
:10AC00009B0803F003033B603B68032B1AD801A2A7
:10AC100052F823F02DAC000035AC00003DAC000034
:10AC200025AC000000F072F878600EE000F014F837
:10AC300078600AE0FFF738FE786006E0FFF79EFDD7
:10AC4000786002E000237B6000BF7B68184608370D
:10AC5000BD4680BD0040064080B584B000AF1D4BAE
:10AC60005B78DBB203F00203002B06D1194B9B7912
:10AC7000DBB203F02003002B02D00023FB6024E0B2
:10AC8000FFF738FEB860BB68002B02D1BB68FB60E1
:10AC90001BE0104BDB78DBB25B09DBB203F0030394
:10ACA000FB710C4BDB78DBB2DB09DBB203F0010399
:10ACB000BB71FA79BB7908495200134431F813305B
:10ACC0001A46BB6802FB03F3FB60FB6818461037AB
:10ACD000BD4680BD004006400C09010080B582B031
:10ACE00000AF094B1B78DBB203F00203002B02D14B
:10ACF00000237B6002E0FFF7D7FD78607B68184691
:10AD00000837BD4680BD00BF0040064080B584B016
:10AD100000AF1A4B9B79DBB203F04003002B02D14A
:10AD20000023FB6024E003F0D8FEB860BB68002B72
:10AD300002D1134802F0C2FA104B1B79DBB203F0C8
:10AD40001F03DBB20133FB71FB79BA68B2FBF3F38B
:10AD5000BB600A4B5B79DBB203F01F03DBB2183335
:10AD6000BB71BA79BB6802FB03F3BB60BB68FB60D5
:10AD7000FB6818461037BD4680BD00BF0040064046
:10AD80009808010080B485B000AF0346FB71174BF3
:10AD90001B7BDBB203F00302FB799A4202D0012352
:10ADA000FB7301E00023FB73104B1B7BDBB223F032
:10ADB0000303DAB2FB7903F00303DBB20B4913435D
:10ADC000DBB20B73FB7B002B09D040F2DC53BB6082
:10ADD00000E000BFBB685A1EBA60002BF9D1002307
:10ADE00018461437BD465DF8047B704700400640A6
:10ADF00080B584B000AF78607B68002B02D11C481E
:10AE000002F05CFA0023FB737B685B7803F01F039E
:10AE1000DAB2FB7B1343FB73164AFB7B1371154BB2
:10AE20005B79DBB223F01F03DAB27B689B7803F017
:10AE30001F03DBB20F491343DBB24B710D4B1B7980
:10AE4000DAB27B681B781343DBB20A4A43F0400353
:10AE5000DBB2137100BF074B9B79DBB203F04003F9
:10AE6000002BF8D000BF00BF1037BD4680BD00BF2B
:10AE7000B80801000040064080B584B000AF78609B
:10AE80007B681B681846FFF74FFD0346FB737B6822
:10AE90001B791946194803F006FE194B5B78DBB2A3
:10AEA00023F03C03DAB2FB7B1B01DBB203F030037F
:10AEB000DBB21343DAB27B685B7911491343DBB22F
:10AEC0004B707B68063319460C4803F0D2FD7B6853
:10AED0005B79002B0DD0094B1B78DBB25BB2002BEA
:10AEE00007DA00BF064B9B79DBB203F00203002BAD
:10AEF000F8D000BF1037BD4680BD00BF00500640EF
:10AF00000040064080B582B000AF03463960FB7157
:10AF10003B68002B02D1234802F0D0F9224B5B782A
:10AF2000DBB2214A23F00203DBB253701E4B1B78C5
:10AF3000DBB203F03B03DBB21B4A63F07F03DBB2FF
:10AF4000137000BF184B9B79DBB203F01C03082B76
:10AF5000F8D1154B5B79DBB2134A23F04003DBB227
:10AF6000537100BF104B9B79DBB203F02003002B21
:10AF7000F8D13868FFF73CFF0B4B5B79DBB20A4A2C
:10AF800043F04003DBB2537100BF074B9B79DBB248
:10AF900003F02003002BF8D0002318460837BD46E5
:10AFA00080BD00BFD40801000040064080B582B0DB
:10AFB00000AF03463A60FB710B46BB713B68002B48
:10AFC00002D1114802F07AF9FB791846FFF7DAFE50
:10AFD000BB7939681846FFF795FF0C4B1B78DBB23D
:10AFE0000A4A03F03F03DBB2137000BF074B9B79A3
:10AFF000DBB29B0803F00303032BF7D100231846B1
:10B000000837BD4680BD00BFF00801000040064083
:10B01000B0B584B000AF786039607B68002B02D196
:10B020001C4802F04BF97B6818464FF000013B6862
:10B030001A464FF0000302FB01F500FB03F42C4419
:10B04000A0FB020163181946134A4FF0000304F0F5
:10B05000D8FD02460B46C7E90223D7E90223012B9C
:10B0600008BF002A02D30D4802F028F9D7E90201EF
:10B070004FF000024FF00003820842EA81728B0811
:10B08000C7E90223BB68184603F048FD00BF10372C
:10B09000BD46B0BD1C09010040420F00400901003F
:10B0A00080B584B000AF78600023FB6009E00D4AF2
:10B0B000FB6852F823307A689A4206D0FB68013365
:10B0C000FB60FB68012BF2D900E000BFFB68012B9D
:10B0D00002D9054802F0F2F8FB6818461037BD4661
:10B0E00080BD00BF680901007809010080B584B007
:10B0F00000AF786039603B68002B02D1154802F040
:10B10000DDF87868FFF7CCFF0346134A52F8233086
:10B11000184603F013FD7B6893F82130DBB223F06F
:10B120004803FB733B681B78012B03D1FB7B43F087
:10B130004003FB733B685B78002B03D0FB7B43F041
:10B140000803FB737B68FA7B83F8212000BF10376C
:10B15000BD4680BDAC0901007009010080B582B018
:10B1600000AF78600B46FB7013463B80FB780F2BDB
:10B1700002D90D4802F0A2F8FA783B88D9B27B6870
:10B1800003F812103B881B0A9BB2DAB2FB7802F07C
:10B190000F02D1B27A685B0013440A465A7000BFAE
:10B1A0000837BD4680BD00BFCC09010080B584B022
:10B1B00000AF78600B46FB70FB780F2B02D90C4870
:10B1C00002F07CF87B6893F82330DBB203F00F03C6
:10B1D000FB73FB781B01DAB2FB7B1343FB737B68C9
:10B1E000FA7B83F8232000BF1037BD4680BD00BF27
:10B1F000F409010080B582B000AF786039607868EA
:10B2000003F0B6FC0346002B05D0094B1B683968D8
:10B210007868984704E0074B1B6839687868984756
:10B22000BFF34F8F00BF00BF0837BD4680BD00BFD2
:10B23000DCCE0120E0CE012080B500AF074B1B68BB
:10B24000002B02D1064802F039F8044B1B6819465E
:10B250000448FFF7CFFF00BF80BD00BFD0CE012064
:10B260001C0A010000C0024080B500AF074B5B68BC
:10B27000002B02D1064802F021F8044B5B68194606
:10B280000448FFF7B7FF00BF80BD00BFD0CE01204C
:10B29000480A010000D0024080B500AF074B9B6810
:10B2A000002B02D1064802F009F8044B9B681946AE
:10B2B0000448FFF79FFF00BF80BD00BFD0CE012034
:10B2C000740A010000C00A4090B589B000AF7860F0
:10B2D0007B68002B02D1534801F0F0FF7B689B682C
:10B2E0007A68127CDA777B689A687B681B7C5B01E2
:10B2F000134403F580531C331B889BB203F0800377
:10B30000002B14BF01230023BB767B68DB68002B76
:10B310000CD17B681B68002B7FD07B681C687B6826
:10B320005968BA7E00237868A04776E07B689A68FF
:10B330007B681B7C5B01134403F5805318331B6847
:10B340007B617B68DB681A467B699B1A7B617B6942
:10B350005B093B61BB7E002B02D03B69FB760EE0B4
:10B360003B69002B04D03B69DBB2013BDBB205E05B
:10B370007B681B7D5BB2DBB2013BDBB2FB767B689B
:10B380005B7C5AB297F91B309A4213D17B68DB7C05
:10B39000FB737B681B7DBB7397F90F2097F90E3009
:10B3A0009A4204D17B68DB7C5BB2FB6112E0002334
:10B3B000FB610FE0FB7E7A68527C52B29B1AFB6104
:10B3C000FB69002B06DA7B681B7D5BB21A46FB69C2
:10B3D0001344FB6197F91B207B685A747B68DB7C04
:10B3E0005BB2DAB2FB69DBB2D31ADBB25AB27B686A
:10B3F000DA747B681B68002B07D07B681C687B684D
:10B400005968FB69BA7E7868A047BB7E002B04D0E0
:10B410007B689B687A68127C1A7700BF2437BD4628
:10B4200090BD00BFA00A010080B500AF044B1B68AF
:10B430001846FFF749FFBFF34F8F00BF00BF80BD25
:10B44000E4CE012080B500AF044B5B681846FFF7DF
:10B450003BFFBFF34F8F00BF00BF80BDE4CE012094
:10B4600080B500AF044B9B681846FFF72DFFBFF374
:10B470004F8F00BF00BF80BDE4CE012080B500AF7C
:10B48000044BDB681846FFF71FFFBFF34F8F00BF69
:10B4900000BF80BDE4CE012080B500AF044B1B6926
:10B4A0001846FFF711FFBFF34F8F00BF00BF80BDED
:10B4B000E4CE012080B500AF044B5B691846FFF76E
:10B4C00003FFBFF34F8F00BF00BF80BDE4CE01205C
:10B4D00080B500AF044B9B691846FFF7F5FEBFF33C
:10B4E0004F8F00BF00BF80BDE4CE012080B500AF0C
:10B4F000044BDB691846FFF7E7FEBFF34F8F00BF31
:10B5000000BF80BDE4CE012080B500AF044B1B6AB4
:10B510001846FFF7D9FEBFF34F8F00BF00BF80BDB5
:10B52000E4CE012080B500AF044B5B6A1846FFF7FC
:10B53000CBFEBFF34F8F00BF00BF80BDE4CE012024
:10B5400080B500AF044B9B6A1846FFF7BDFEBFF302
:10B550004F8F00BF00BF80BDE4CE012080B500AF9B
:10B56000044BDB6A1846FFF7AFFEBFF34F8F00BFF7
:10B5700000BF80BDE4CE012080B500AF044B1B6B43
:10B580001846FFF7A1FEBFF34F8F00BF00BF80BD7D
:10B59000E4CE012080B500AF044B5B6B1846FFF78B
:10B5A00093FEBFF34F8F00BF00BF80BDE4CE0120EC
:10B5B00080B500AF044B9B6B1846FFF785FEBFF3C9
:10B5C0004F8F00BF00BF80BDE4CE012080B500AF2B
:10B5D000044BDB6B1846FFF777FEBFF34F8F00BFBE
:10B5E00000BF80BDE4CE012080B584B000AF78609C
:10B5F0000023FB6009E00D4AFB6852F823307A68AB
:10B600009A4206D0FB680133FB60FB68042BF2D939
:10B6100000E000BFFB68042B02D9054801F04EFE94
:10B62000FB6818461037BD4680BD00BFD80A010030
:10B63000EC0A010080B586B000AFF860B9607A60AE
:10B640007B68002B02D1144801F038FE01237B6196
:10B650007B681B78002B0AD1FB685A697969BB6843
:10B6600001FA03F3DB431A40FB685A610FE07B6881
:10B670005B781A46B968F86803F08DFAFB685A6976
:10B680007969BB6801FA03F31A43FB685A6100BF8A
:10B690001837BD4680BD00BF200B010080B584B0C7
:10B6A00000AF78607868FFF79FFF0346FB73FB7B72
:10B6B000054A52F82330BB60BB68D3F8A030184667
:10B6C0001037BD4680BD00BFC40A010080B584B0FC
:10B6D00000AF786039607868FFF786FF0346FB7338
:10B6E000FB7B064A52F82330BB60BB683A68C3F85C
:10B6F000A02000BF1037BD4680BD00BFC40A0100B6
:10B7000080B584B000AF78600023FB6009E00D4A8B
:10B71000FB6852F823307A689A4206D0FB680133FE
:10B72000FB60FB68022BF2D900E000BFFB68022B34
:10B7300002D9054801F0C2FDFB6818461037BD4626
:10B7400080BD00BFD00B0100DC0B010080B584B0D0
:10B7500000AF786039607B68DB78FB737B689B782F
:10B76000BB73BB7B03F02003002B04D1FB7B03F0F6
:10B770001003002B05D0094B1B683968786898477F
:10B7800004E0074B1B68396878689847BFF34F8F10
:10B7900000BF00BF1037BD4680BD00BF30CF0120C5
:10B7A00034CF012080B586B000AFF860B9607A6010
:10B7B000BB68002B02D1314801F080FD7B68002B73
:10B7C00002D12F4801F07AFDF868FFF799FF034690
:10B7D0002C4A52F82330184603F0FAF9FB6800228D
:10B7E0001A70FB6800225A70FB6800229A70FB688E
:10B7F000FF22DA70FB6800225A71FB6850229A71AE
:10B80000FB680022DA71FB689B78DBB203F07F03F0
:10B81000DAB2FB689A7045F21201F86803F0F2F9A7
:10B82000BB685B687A681946F86800F02DF8FB6819
:10B830009B79FB75FB7D03F07F03FB75BB685B7831
:10B84000DB01DAB2FB7D1343FB75FB7D23F00F03B5
:10B85000FB75BB681B7A03F00F03DAB2FB7D134361
:10B86000FB75FB68FA7D9A71BB681B78DB01DAB265
:10B87000FB689A7000BF1837BD4680BD100C0100F0
:10B88000380C0100C40B010080B48DB000AFF8602B
:10B89000B9607A604FF0FF33FB620023BB62002384
:10B8A0007B620123FB61002387F8233044E0FB6ABD
:10B8B000002B46D097F82330FA6902FA03F3BB61F4
:10B8C000002387F822302CE097F82230274A32F8FC
:10B8D00013301A46BB6903FB02F37A68B2FBF3F339
:10B8E0007B61BA687B699A4203D9BA687B69D31ACB
:10B8F00002E07A69BB68D31A3B613A69FB6A9A42F3
:10B900000AD297F82330BB6297F822307B623B69FA
:10B91000FB623B69002B09D097F82230013387F88E
:10B92000223097F822303F2BCED900E000BF97F8A5
:10B930002330013387F8233097F82330022BB6D910
:10B9400000E000BFBB6ADBB29B01DAB27B6ADBB20C
:10B9500003F03F03DBB21343DAB2FB685A7000BF57
:10B960003437BD465DF8047B704700BF440B0100CF
:10B9700080B500AF034B5B6819460348FFF7E6FE4E
:10B9800000BF80BD24CF01200070064080B500AF0D
:10B99000034B9B6819460348FFF7D8FE00BF80BDE4
:10B9A00024CF012000600E4080B584B000AF7860E5
:10B9B0000023FB6006E00B4A7B68934206D0FB68DD
:10B9C0000133FB60FB68002BF5D000E000BFFB6893
:10B9D000002B02D0044801F071FCFB6818461037B8
:10B9E000BD4680BD007003405C0C010080B584B092
:10B9F00000AF786039603B68002B02D11E4801F02F
:10BA00005DFC7868FFF7D0FF1C4B184603F060FA26
:10BA10007B681B6823F002027B681A600023FB73BB
:10BA200012E0FB7B7A681B01134403F584731A68E8
:10BA3000FB7B22F0070279681B010B4403F584733A
:10BA40001A60FB7B0133FB73FB7B032BE9D93B685B
:10BA50001B78002B06D07B681B6823F001027B68F3
:10BA60001A6005E07B681B6843F001027B681A607E
:10BA700000BF1037BD4680BD900C010017003C1080
:10BA800080B584B000AF78600023FB7302E0FB7BDD
:10BA90000133FB73FB7B002B03D1074A7B68934286
:10BAA000F5D1FB7B002B02D0044801F007FCFB7BA7
:10BAB00018461037BD4680BD00100B40B00C010089
:10BAC00080B586B000AF786039603B68002B02D14A
:10BAD0002A4801F0F3FB7B681B697B617B685B692B
:10BAE0003B617B689B69FB603B685B7A002B21D0E4
:10BAF0003B687A69DA603B685B7A032B1AD13B6852
:10BB0000DB681A023B68DA603B691A027B691B0E2C
:10BB10001A433B681A61FB681A023B691B0E1A4301
:10BB20003B685A617B68DB691A02FB681B0E1A438B
:10BB30003B689A613B68DB69002B19D03B685B7AF4
:10BB4000012B0BD03B685B7A022B07D03B685B7AFA
:10BB5000082B03D03B685B7A062B09D13B68DA6976
:10BB60003B68DB681340002B02D040F2A66300E084
:10BB7000002318461837BD4680BD00BFE40C010005
:10BB800080B586B000AF7860396000237B61002308
:10BB90003B613B685B6803F00303002B06D03B6806
:10BBA0005B6823F003031A1D3B685A603B689B687F
:10BBB0003A68526802FB03F39B08FB6026E000BF73
:10BBC000786803F0B9F90246184B1340002BF7D000
:10BBD000786803F0B1F9034603F0B873002B08D07E
:10BBE0003B685B7883F00103DBB2002B01D00123BB
:10BBF0003B613B69002B05D17A693968786803F0AD
:10BC000087FA78610949786803F0A2F93B69002B4B
:10BC100003D17A69FB689A42D1D30549786803F069
:10BC200097F93B6918461837BD4680BD2000700162
:10BC30000200700180B586B000AF786039600023E3
:10BC40007B6100233B613B685B6803F00303002BCF
:10BC500006D03B685B6823F003031A1D3B685A60FB
:10BC60003B689B683A68526802FB03F39B08FB60E1
:10BC700026E000BF786803F05FF90246254B1340C9
:10BC8000002BF7D0786803F057F9034603F0B87338
:10BC9000002B08D03B685B7883F00103DBB2002BFC
:10BCA00001D001233B613B69002B05D17A693968DA
:10BCB000786803F07FFA78611649786803F048F9EC
:10BCC0003B69002B03D17A69FB689A42D1D300BF4C
:10BCD000786803F031F902460F4B1340002BF7D080
:10BCE000786803F029F9034603F0B873002B08D0F5
:10BCF0003B685B7883F00103DBB2002B01D00123AA
:10BD00003B610549786803F023F93B691846183709
:10BD1000BD4680BD100070010200700180B584B086
:10BD200000AF786039600023FB6000BF786803F0E3
:10BD300003F902460F4B1340002BF7D0786803F04D
:10BD4000FBF8034603F47023002B01D00123FB60B2
:10BD5000FB68002B04D139687868FFF7B1FEF86002
:10BD60000449786803F0F4F8FB6818461037BD46BC
:10BD700080BD00BF01000F0080B584B000AF7860C7
:10BD800039600023FB6000BF786803F0D5F80246F5
:10BD90000E4B1340002BF7D0786803F0CDF8024625
:10BDA0000B4B1340002B08D03B685B7883F00103FA
:10BDB000DBB2002B01D00123FB600649786803F059
:10BDC000C7F8FB6818461037BD4680BD02007011E9
:10BDD000000070110A00701180B584B000AF786067
:10BDE00039603B68002B02D13A4801F067FA3B68A2
:10BDF0009B78012B02D1384801F060FA3B689B68C0
:10BE0000002B03D03B689B68802B02D9334801F09C
:10BE100055FA3B685B68002B03D03B685B68802B5E
:10BE200002D92F4801F04AFA7868FFF729FE2D4B16
:10BE3000184603F067F87B68DB6A43F0E0627B68D2
:10BE4000DA627B689B6AFB607B685B6CBB60FB684B
:10BE500023F44E73FB603B681B78002B03D0FB6818
:10BE600043F00803FB603B685B781B0103F0300282
:10BE70003B689B781B0203F440731343FA68134337
:10BE8000FB60BB6803F0FF23BB603B685B68DAB212
:10BE90003B689B681B0403F47F031343BA68134396
:10BEA000BB607B68BA685A647B68FA689A627B6890
:10BEB000DB6A43F007027B68DA627B680A4A5A63EE
:10BEC0007B6800229A637B68074A1A6300BF1037B9
:10BED000BD4680BD080D01002C0D0100640D010060
:10BEE000C80D01001100301037017F1180B58AB0F4
:10BEF00000AFF860B9607A60BB68002B02D1584887
:10BF000001F0DCF97B68002B03D07A68BB689A42A9
:10BF100002D9544801F0D2F900237B6200233B622E
:10BF20000023FB6100237B610023BB61BA687B684F
:10BF3000B2FBF3F37B627B6AB3F5805F01D9002328
:10BF40008AE07B6A002B49D0BA687B6AB2FBF3F3C4
:10BF50007A689A4202D27B6A01337B627B6A102B39
:10BF600032D97B6A1B09FB6102E0FB690133FB618B
:10BF70004FF48073FA69B3FBF2F2F96901FB02F244
:10BF80009B1A002BF1D1FB69012BEED07A6AFB6979
:10BF9000B2FBF3F33B6202E03B6A01333B623B6A74
:10BFA000FA6902FB03F37A6A9A42F5D83B6A002BDE
:10BFB00001D03B6A00E00123BA68B2FBF3F2FB69EF
:10BFC000B2FBF3F3BB610FE07B6A3B620023FB61D2
:10BFD000BA683B6AB2FBF3F3BB6105E000233B6246
:10BFE0000023FB61BB68BB613B6A002B02D03B6A4C
:10BFF000013B3B62FB69002B02D0FB695B08FB61E4
:10C00000FB68DB6A23F00802FB68DA62FB68DB6A24
:10C010007B617B6923F47F2323F47F637B613B6A2D
:10C020001B01DAB2FB691B029BB21A437B69134303
:10C0300043F460237B61FB687A69DA6200BFFB68C6
:10C040005B6A03F00803002BF9D0FB68DB6A43F05E
:10C050000802FB68DA62BB6918462837BD4680BD16
:10C06000280E01004C0E010080B582B000AF786050
:10C0700039603B68002B02D11A4801F01FF93B6878
:10C080001B68B3F5005F02D3174801F017F93B684E
:10C090005B68B3F5803F02D3144801F00FF97B6869
:10C0A0005B6803F460423B681B68C3F30C013B68A8
:10C0B0005B681B040B431A437B685A603B689A68B1
:10C0C0007B689A603B68DB681B0603F07C523B6828
:10C0D0001969074B0B401A437B68DA6000BF0837C9
:10C0E000BD4680BD940E0100B80E0100200F010076
:10C0F0003700FB0080B48BB000AFF8607A603B6023
:10C100000B46FB7200237B623B6B3B627B68002B20
:10C1100002D03B68002B05D1FB7A012B0BD0FB7AB8
:10C12000022B08D03B6B002B05D07B6B002B02D081
:10C13000FB7A012B02D104237B627FE0FB7A022B86
:10C1400008D13B6A03F00303002B03D04FF4D563FF
:10C150007B6273E0FB7A022B70D17B6B03F00303ED
:10C16000002B04D07B6B23F0030304337B637B6BD6
:10C17000364AA2FB0323DB0B0133BB613B689B0008
:10C18000DB08BA699A4202D903237B6256E07B68D6
:10C190007B610023FB6147E03A6A3B6BD31A9B004B
:10C1A0007A6BD31AB3F5803F1ED2FB69DB007A6944
:10C1B00013443A6A5A603A6A3B6BD31A9B007A6B13
:10C1C000D21AFB69DB0079690B4412041A60FB691F
:10C1D000DB007A6913441A68FB69DB0079690B4458
:10C1E00042F023021A601CE0FB69DB007A69134409
:10C1F0003A6A5A60FB69DB007A691344144A1A6090
:10C20000FB69DB007A6913441A68FB69DB00796912
:10C210000B4442F021021A603B6A03F57F43FC3372
:10C220003B62FB690133FB61FA69BB699A42B3D394
:10C23000FB6800221A607A68FB689A657B6A184678
:10C240002C37BD465DF8047B704700BF018000803D
:10C250000000FCFF80B58AB002AFF860B9607A6078
:10C260003B603B68002B02D13C4801F027F80023DB
:10C27000BB61FB689B6A1B0A03F00303FB773B6807
:10C280005B687B613B681B683B617B69002B07D067
:10C290003B69002B06D03B699B68B3F5803F01D317
:10C2A000042356E000BFF86802F060FE034603F086
:10C2B0000103002BF7D13B69002B07D0F86802F08F
:10C2C00055FE034603F00203002BF4D13B69002B1B
:10C2D0001FD0BB68002B1CD03B69DB68002B02D051
:10C2E0003B69DB6801E03B691B693A69926839691F
:10C2F000496801FB02F2F97F019200937B68BA68FA
:10C30000F868FFF7F7FEB861BB69002B01D0002386
:10C31000FB77FB7F3A697969F86802F04DFE79692D
:10C32000F868FFF7FBFCB861BB69002B01D0BB6963
:10C330000FE03B69002B0BD0FB7F3A69F968184688
:10C3400002F0AFFFB861BB69002B01D0BB6900E010
:10C35000002318462037BD4680BD00BF880F01006E
:10C3600080B500AF094B1B68002B02D1084800F0D4
:10C37000A5FF084B1B68054A1268114606489847F6
:10C38000BFF34F8F00BF00BF80BD00BF38CF01207B
:10C39000AC0F01003CCF012000100B4080B500AF76
:10C3A0000B4BD3F888300A4A43F47003C2F8883044
:10C3B000084B4CF22052DA81064B4DF62812DA81F6
:10C3C000044B4FF4E9721A8002F0DFFF00BF80BD1A
:10C3D00000ED00E00020054080B483B000AF78603D
:10C3E0000B4B03F5805304331B6823F040527B68EA
:10C3F0001B0703F0405306491A4301F580530433E9
:10C400001A6000BF0C37BD465DF8047B704700BF63
:10C410000070044080B400AF054B03F58253043331
:10C420004FF092721A6000BFBD465DF8047B704702
:10C430000070044080B483B000AF7860044A7B6829
:10C44000136000BF0C37BD465DF8047B704700BF2A
:10C45000C8CE012080B483B000AF7860044A7B6806
:10C46000136000BF0C37BD465DF8047B704700BF0A
:10C47000CCCE012080B582B000AF78600B46FB7057
:10C480001B4802F089FF1B4B1B6903F48073002BD0
:10C4900009D17968174802F0B5FF164B1B69154A98
:10C4A00043F480731361FB78002B06D0114B1B699A
:10C4B000104A23F40073136105E00E4B1B690D4A0B
:10C4C00043F4007313614FF40040FFF7C3FF094BBF
:10C4D0005B6903F00103002B03D0064B054A1B6880
:10C4E0001360034802F072FF00BF0837BD4680BDED
:10C4F0001D003C1000D0034080B483B000AF034661
:10C50000FB710B4B1B78DBB223F03803DAB2FB79FB
:10C51000DB00DBB203F03803DBB205491343DBB2C7
:10C520000B7000BF0C37BD465DF8047B704700BF41
:10C530000040064080B500AFFFF76CFF01214FF4CB
:10C54000A050FFF797FF0E48FEF796FC0D4B1846DC
:10C55000FFF770FF00231846FFF7CEFF00230A4ABB
:10C5600000211846FEF722FD0848FEF727FB084B7E
:10C57000084A1A600220FFF72FFF00BF80BD00BFEE
:10C58000EC0F01000024F400E00F0100E40F0100B3
:10C5900068580020000E270780B483B000AF034620
:10C5A000FB7197F90730002B0BDBFB7903F01F02BF
:10C5B000074997F907305B09012000FA02F241F8B8
:10C5C000232000BF0C37BD465DF8047B704700BFD9
:10C5D00000E100E080B483B000AF03463960FB7136
:10C5E00097F90730002B0ADB3B68DAB20C4997F960
:10C5F00007301201D2B20B4483F800230AE03B68F3
:10C60000DAB20849FB7903F00F03043B1201D2B2FE
:10C610000B441A7600BF0C37BD465DF8047B7047AB
:10C6200000E100E000ED00E080B500AF11491248E4
:10C63000FDF794FF0021104802F019FF032319466B
:10C640000D4802F0D6F9002319460B4802F0B5F95F
:10C65000094802F01AF9094A00210748FEF704F8D0
:10C6600001212720FFF7B6FF272002F0EAFE00BFD6
:10C6700080BD00BFF40F010000B003406C580020E3
:10C6800080B500AF11491248FDF768FF002110483E
:10C6900002F0EDFE032319460D4802F0AAF901232A
:10C6A00019460B4802F089F9094802F0EEF8094AE8
:10C6B00000210748FDF7D8FF01214920FFF78AFF35
:10C6C000492002F0BEFE00BF80BD00BF0010010087
:10C6D00000B00B407458002080B500AF09490A48EB
:10C6E000FEF704FD002200210748FEF737FD002178
:10C6F0000548FEF75BFD0121034802F0D4FE00BFB0
:10C7000080BD00BF0C10010000C00C4080B500AF20
:10C7100009490A48FEF7EAFC002200210748FEF713
:10C720001DFD00210548FEF741FD0121034802F0EF
:10C73000BAFE00BF80BD00BF1010010000D00C4049
:10C7400080B500AF0220FEF795F903461A46064968
:10C750000648FFF727F84021044802F080FA182025
:10C7600002F06FFE00BF80BD1410010000600640A3
:10C7700080B500AF0220FEF77DF903461A46034953
:10C780000348FFF70FF800BF80BD00BF2010010075
:10C7900000600E40B0B500AF29492A48FFF726F9DE
:10C7A0000220FEF767F9034618464FF000010246E3
:10C7B0000B464FF000044FF000055D0145EAD265DD
:10C7C000540122462B46121A63EB01034FF000047A
:10C7D0004FF000059D0045EA9275940022462B46D5
:10C7E000121841EB03034FF000004FF00001D90095
:10C7F00041EA5271D00002460B4610461946124AD1
:10C800004FF0000303F0FDF902460B461346013BCF
:10C810001A4600210B4802F087FE02220021094837
:10C8200002F065FE02213020FFF7D4FE302002F036
:10C8300008FE0021034802F08BFE00BFB0BD00BF20
:10C840002C1001000070034040420F0080B59CB0E6
:10C8500000AFD94802F0D7FED84802F0D4FED8483D
:10C8600002F0D1FED74802F0CEFED74802F0CBFE50
:10C87000002387F86C30002387F86D3007F16C03D4
:10C880001A460521D148FEF7D5FE002387F8683007
:10C89000002387F8693007F168031A460E21CB4858
:10C8A000FEF7C8FE012387F86430002387F865305F
:10C8B00007F164031A460F21C448FEF7BBFE0123AB
:10C8C00087F86030002387F8613007F160031A466B
:10C8D0001021BE48FEF7AEFE012387F85C3000232E
:10C8E00087F85D3007F15C031A460021B848FEF76F
:10C8F000A1FE012387F85830002387F8593007F14B
:10C9000058031A460121B248FEF794FE012387F826
:10C910005430002387F8553007F154031A4602219A
:10C92000AB48FEF787FE012387F85030002387F8D5
:10C93000513007F150031A460321A548FEF77AFE4D
:10C94000002387F84C30002387F84D3007F14C0363
:10C950001A4610219E48FEF76DFE002387F84830E6
:10C96000002387F8493007F148031A4611219848F7
:10C97000FEF760FE974B1B88A7F8443007F144038D
:10C980001A4612219248FEF755FE924B1B88A7F8D3
:10C99000403007F140031A4613218D48FEF74AFE46
:10C9A000012387F83C30002387F83D3007F13C0332
:10C9B0001A4600218848FEF73DFE012387F83830EB
:10C9C000002387F8393007F138031A4601218248DD
:10C9D000FEF730FE012387F83430002387F8353026
:10C9E00007F134031A4602217B48FEF723FE012398
:10C9F00087F83030002387F8313007F130031A46CA
:10CA000003217548FEF716FE724B1B88BB8507F1A4
:10CA10002C031A4604217048FEF70CFE6D4B1B8850
:10CA20003B8507F128031A4605216B48FEF702FEF5
:10CA3000002387F82430002387F8253007F12403EA
:10CA40001A4606216448FEF7F5FD002387F82030DA
:10CA5000002387F8213007F120031A4607215E489A
:10CA6000FEF7E8FD01233B7700237B7707F11C03EA
:10CA70001A4600215948FEF7DDFD00233B760023CE
:10CA80007B7607F118031A4601215448FEF7D2FDC0
:10CA900000233B7500237B7507F114031A4604211C
:10CAA0004E48FEF7C7FD01233B7400237B7407F15A
:10CAB00010031A4605214948FEF7BCFD01233B73CC
:10CAC00000237B7307F10C031A4606214348FEF747
:10CAD000B1FD00233B7200237B7207F108031A4665
:10CAE00007213E48FEF7A6FD00233B7100237B7122
:10CAF0003B1D1A461A213A48FEF79CFD05220C21DF
:10CB0000384802F09AFD374B1B6B23F0807323F0FB
:10CB10000403344A43F00403136305220D21314812
:10CB200002F08BFD2F4B5B6B23F0807323F004032B
:10CB30002C4A43F00403536301220E21294802F0DA
:10CB40007CFD284B9B6B23F0807323F00703254A61
:10CB500043F00703936301220F21224802F06DFD89
:10CB6000204BDB6B23F0807323F004031D4A43F05A
:10CB70000403D363012210211A4802F05EFD194B11
:10CB80001B6C23F0807323F00403164A43F0040364
:10CB9000136400221121134802F04FFD114B5B6C0E
:10CBA00023F0807323F004030E4A43F0040353641C
:10CBB0000122052118E000BF090038100A003810D2
:10CBC0000B0038100C0038100D00381000F00F402A
:10CBD00040F00F403010010080F00F40C0F00F40D7
:10CBE00000F10F4000900440BF4802F026FDBE4B0C
:10CBF0005B6923F0807323F04603BB4A43F00603CE
:10CC0000536101220021B94802F017FDB74B1B68A0
:10CC100023F0807323F00403B44A43F00403136049
:10CC200001220121B14802F008FDB04B5B6823F0FE
:10CC3000807323F00403AD4A43F0040353600022E1
:10CC40000A21AA4802F0F9FCA84B9B6A23F08073E2
:10CC500023F00403A54A43F00403936200220B214E
:10CC6000A24802F0EAFCA14BDB6A23F0807323F0B8
:10CC700004039E4A43F00403D362012210219B481F
:10CC800002F0DBFC0B221021984802F0F3FC974BDA
:10CC90001B6C23F0807323F00703944A43F00703CF
:10CCA000136401221121914802F0C7FC0B221121CB
:10CCB0008E4802F0DFFC8D4B5B6C23F0807323F019
:10CCC00007038A4A43F0070353640122122187486D
:10CCD00002F0B3FC854B9B6C23F0807323F00403BC
:10CCE000824A43F004039364012213217F4802F037
:10CCF000A4FC7E4BDB6C23F0807323F004037B4A9F
:10CD000043F00403D36401220221784802F095FC29
:10CD1000764B9B6823F0807323F00403734A43F03F
:10CD20000403936001220321704802F086FC6F4BDC
:10CD3000DB6823F0807323F004036C4A43F00403A0
:10CD4000D360012200216A4802F077FC684B1B681F
:10CD500023F0807323F00403654A43F00403136057
:10CD600001220121624802F068FC614B5B6823F0FC
:10CD7000807323F004035E4A43F0040353600022EF
:10CD80000A215B4802F059FC594B9B6A23F08073DF
:10CD900023F00403564A43F00403936200220B215C
:10CDA000534802F04AFC524BDB6A23F0807323F0B5
:10CDB00004034F4A43F00403D362012202214C488A
:10CDC00002F03BFC4A4B9B6823F0807323F0040382
:10CDD000474A43F00403936001220321444802F0D0
:10CDE0002CFC434BDB6823F0807323F00403404AA0
:10CDF00043F00403D360012204213D4802F01DFCEE
:10CE00003B4B1B6923F0807323F00403384A43F043
:10CE10000403136101220521354802F00EFC344B56
:10CE20005B6923F0807323F00403314A43F0040369
:10CE30005361012206212E4802F0FFFB0B2206213E
:10CE40002B4802F017FC2A4B9B6923F0807323F0D8
:10CE50000703274A43F0070393610122072124486F
:10CE600002F0EBFB0B220721214802F003FC204BD0
:10CE7000DB6923F0807323F007031D4A43F00703A7
:10CE8000D361002208211A4802F0D7FB184B1B6A15
:10CE900023F0807323F00403154A43F00403136264
:10CEA00000220921124802F0C8FB114B5B6A23F0F3
:10CEB000807323F004030E4A43F0040353620122FB
:10CEC00000210C4802F0B9FB0A4B1B6823F0807369
:10CED00023F00403074A43F00403136001220121F5
:10CEE000044802F0AAFB07E00090044000A00440C0
:10CEF00000B0044000C00440734B5B6823F08073B3
:10CF000023F00703704A43F007035360072202210E
:10CF10006D4802F092FB6C4B9B6823F0807323F00A
:10CF20000403694A43F0040393600722032166481F
:10CF300002F083FB644BDB6823F0807323F004036F
:10CF4000614A43F00403D360012204215E4802F0E9
:10CF500074FB0B2204215C4802F08CFB5A4B1B69CA
:10CF600023F0807323F00703574A43F0070313614C
:10CF700001220521544802F060FB534B5B6923F00A
:10CF8000807323F00403504A43F0040353610122E9
:10CF900006214D4802F051FB4B4B9B6923F08073F7
:10CFA00023F00403484A43F004039361012207215C
:10CFB000454802F042FB0B220721434802F05AFB8E
:10CFC000414BDB6923F0807323F007033E4A43F0B3
:10CFD0000703D361042200213C4802F02EFB3B4BA7
:10CFE0001B6823F0807323F04703384A43F0430360
:10CFF000136004220121354802F01FFB334B5B68AC
:10D0000023F0807323F04703304A43F04303536017
:10D01000042202212D4802F010FB2C4B9B682B4A66
:10D0200023F0807323F00403936000221921274822
:10D0300002F003FB254B5B6E23F0807323F00403A7
:10D04000224A43F00403536601221A211F4802F0CA
:10D05000F4FA1E4B9B6E23F0807323F007031B4AE8
:10D0600043F00703936604220321184802F0E5FA0F
:10D07000164BDB6823F0807323F04703134A43F019
:10D080004303D36004220421104802F0D6FA0F4B68
:10D090001B6923F0807323F047030C4A43F04303DA
:10D0A000136104220521094802F0C7FA074B5B69A6
:10D0B00023F0807323F04703044A43F04303536192
:10D0C00000BF7037BD4680BD00C0044000D00440A2
:10D0D00080B483B000AF0346FB7197F90730002B93
:10D0E0000BDBFB7903F01F02074997F907305B0957
:10D0F000012000FA02F241F8232000BF0C37BD46A0
:10D100005DF8047B704700BF00E100E080B483B0AD
:10D1100000AF03463960FB7197F90730002B0ADB3B
:10D120003B68DAB20C4997F907301201D2B20B44CE
:10D1300083F800230AE03B68DAB20849FB7903F080
:10D140000F03043B1201D2B20B441A7600BF0C3716
:10D15000BD465DF8047B704700E100E000ED00E0B3
:10D1600080B500AF0621054802F0BDFA0346012B49
:10D170000CBF01230023DBB2184680BD00F10F4035
:10D1800098B500AF0E4802F0DDFA034603F0400305
:10D19000002B0ED00B4B9B68002B0AD0094B9C68D0
:10D1A000FFF7DEFF03461A46064B1B691946104679
:10D1B000A0474FF0FF31024802F0D1FA00BF98BDFE
:10D1C00000D00440C0CF012080B582B000AF7860AD
:10D1D0003960164B64225A60144B00221A70134BAC
:10D1E000134ADA60114A7B689360104A3B68136106
:10D1F0000B2206210F4802F088FA06213F20FFF794
:10D2000085FF3F2002F059FA06210B4802F06BFA25
:10D210000346012B06D17B68002B03D07B6839685D
:10D220000120984700BF0837BD4680BDC0CF012010
:10D2300061D1000000D0044000F10F4090B585B0EE
:10D2400000AFF860B9607A603B60FB68002B02D1E8
:10D25000144800F033F8144B144ADA62124B2022BF
:10D260001A63FB68104A1A60FB681B68104A1A6050
:10D27000FB681C680020FDF7FDFB03466360FB684C
:10D280001B680C4A9A65FB680B4A1A613968B868D2
:10D29000FFF79AFF79685120FFF738FF00BF143776
:10D2A000BD4690BD34100100D4CF012040CF0120F5
:10D2B00000100B4038D00120C0CF012010B50F491D
:10D2C00004460F4802F092FB0C49204602F08EFB08
:10D2D0000C49D1F88030013B002BC1F8803008DBCD
:10D2E0008B6F5A1C8A670A221A70BDE8104000F042
:10D2F0000BB878310A2002F087FAF6E7C0D0012097
:10D300005410010048D0012018200149ABBE7047DD
:10D3100026000200DFED0A0AB5EEC00AF1EE10FAAF
:10D32000F0EE407A4FF001014CBF70EEC00A77EE8C
:10D33000A00A084648BFB1EE400AF4F7B9BB00BFE7
:10D34000DB0FC93F2DE9F041D5685769EB028046F4
:10D350000E46144605D5384602F0EBFD45F01005A3
:10D36000A061124B2B408BB1A169384602F0F3FD4E
:10D37000002806DAE36843F08003E3604FF0FF30F3
:10D3800011E025F4003525F01005E56032464146F0
:10D39000384602F0ECFD20F00041761AA1690E44F7
:10D3A000A6610028E6D1BDE8F08100BF10000200B0
:10D3B000F8B5304E3468002851D10020F8BD2368FC
:10D3C000B3F1805F39D1D4E9013252B11168B1F1C2
:10D3D000805F06D1516803330B4463609368A36098
:10D3E000F1E7AB4207DB9E4505DB20464FF00053DB
:10D3F00040F80C3BE2E7634511D920464FF000515D
:10D40000656040F80C1B5B1B00EB8501A160033BD2
:10D410004FF0805440F82540C1E90132CEE762B9AF
:10D42000A0EB830000F060F90130C6D04FF000534C
:10D43000C4E9003504F10C00C0E72746A468002CBD
:10D44000BDD10C3000F050F9431CB6D04FF0005362
:10D45000C0E90035846057B930600C30AEE7C31CBA
:10D460009D08002705F10A0C05F1030EE7E7B860F7
:10D47000F3E700BF04D1012010B5FFF799FF044680
:10D4800028B90449172202F072FDFFF73DFF20463C
:10D4900010BD00BF691001002DE9F843C6683D4B7F
:10D4A000334004460D4690461BB902273846BDE876
:10D4B000F883D0F81490484602F041FD0746002852
:10D4C000F3D1B8F1010F2CD0B8F1020F2ED0B8F182
:10D4D000000FEAD1002DE8DBB00404D52368E26A2E
:10D4E0009A4238BFE362A169A9420EDC2368E26A6E
:10D4F000934238BF134622695818801AA84204DBA9
:10D50000206B01EB000CAC4534DC0023C4E9013393
:10D5100046F02006A56226F4032626F04006E660C3
:10D52000C4E7204600F038F80544D3E7484602F047
:10D5300000FDB0F1000CE26804DA42F08002E26023
:10D540000127B3E723681846A3691946E36A98429E
:10D550002CBF0918C9180B4621699206A3EB0103D9
:10D5600003D5A26A9342B8BF13466345ACBFED181A
:10D570006544AFE76D1AB10744BF281AA060F107F0
:10D5800044BF9B1AEB1A154448BF6360256026F020
:10D590002006C0E703001000C3689A0705D10E4BB0
:10D5A00021221A604FF0FF30704703F020021B0366
:10D5B00009D512B1806A0138704703688269006931
:10D5C0001344181AF7E70AB1806A70470368826942
:10D5D00000691344181A7047FCD0012010B5174A8F
:10D5E0001749002002F083FA4FF480734FF48062F1
:10D5F0000021124802F032FA124A1349012002F0C7
:10D6000076FA4FF480730F484FF48062002102F0E5
:10D6100025FA0E4B1B68022B0EDD0D4A0A4902202B
:10D6200002F065FABDE8104009484FF480734FF4EA
:10D630008062002102F012BA10BD00BF48D0012064
:10D640008110010084D001208310010050100100DE
:10D65000C0D00120B5EE400AF1EE10FA04D100234B
:10D660009FED100A0360704710EE103AC3F3C752E3
:10D67000A2F17E0192B9C3F31602520012F4000F18
:10D6800001F1FF31F9D003F00043C2F31602134356
:10D6900043F07C5300EE103A0160704723F0FF43E3
:10D6A000F6E700BF00000000B5EE400AF1EE10FA08
:10D6B00015D010EE103AC3F3C7521044FE2807DD10
:10D6C000084B22221A604FF0FF4000EE100A70470C
:10D6D000002804DD23F0FF4343EAC050F5E70020B3
:10D6E000F3E700BFFCD0012070B50B4D2B680BB9E0
:10D6F0000A4B2B6003302E6820F00304344420468C
:10D7000000F032F810B92C60304670BD044B0C228A
:10D710001A604FF0FF36F7E700D1012018D1012041
:10D72000FCD00120F7B5044698B103B0BDE8F04045
:10D7300002F047BA07FB046002F043FA002818BF62
:10D740004FF0FF350134019BA342F3DC284603B0C0
:10D75000F0BD034B034E1B68019305463C27F2E7DF
:10D760005010010048D00120044B23B1984234BF2F
:10D770000020012070471846704700BF18E10120C3
:10D780002DE9F0471D4681EA0506C1F30A5C1446FF
:10D790000B462F4640F2FF7E06F00046BCF1000F1C
:10D7A00006D0F44504D0C5F30A520AB1724507D138
:10D7B0005B0013F5001F55D358D00020334943E0D8
:10D7C000C1F3130343F48015630DE402A5FB048940
:10D7D00043EAC7270CEB020A47F000474A460023FA
:10D7E000E7FB0523A4FB0045C4464FF00009A8460B
:10D7F000E0FB078918EB0C0C4FF0000E49EB0E0E06
:10D8000012EB0E0243F10003B3F5801F4CEA9404BF
:10D810001CD2901843EB030140EAD472AAF580654C
:10D820000B466400E10F521843F1000340F2FD7112
:10D83000B4F1004F174608BF22F001078D4208D807
:10D840001E4306EB05513846BDE8F087AAF2FF35C6
:10D85000E8E7002D03DB46F0FF4646F4E006002033
:10D860003146F1E77A0012F5001FF8D3084A7F002D
:10D870009742A2D813424FF000009FD017429DD08C
:10D8800046F0FF4141F4E001DEE700BF0000F87F11
:10D890000000E0FF2DE9F04FC1F30A578946144616
:10D8A0008C46804640F2FF72594037B1974204D00F
:10D8B000C3F30A5008B1904207D1454A4FEA4C00E1
:10D8C000904259D90020434954E022463F1A4FEA7A
:10D8D000585040EAC92C500D40EAC32343F0004B96
:10D8E0004CF000455D454FEAC8244FEAC22A08BF04
:10D8F000544522BF630843EAC5736A084FEA5A08D1
:10D9000025BF1C46154607F2FD3007F2FE3048EAF7
:10D91000CB784FEA5B09352200234D4508BF4445CB
:10D920004FEA430305D3B4EB080465EB090543F064
:10D93000010324196D41212A08BF1E46013AECD18A
:10D940004D4508BF444502D3013308BF013601F0FD
:10D95000004240F2FD71884204D802EB0052911956
:10D96000184607E00028A4BF42F0FF4242F4E0025C
:10D9700000201146BDE8F08F5C0014F5001FA1D80F
:10D9800043EA0C0312EA430301D11249E8E710EA23
:10D99000020501F0004302D119462846EAE7224079
:10D9A00005D143F0FF4141F4E0011046E2E714F5F0
:10D9B000001F05D043F0FF41002041F4E001D9E70A
:10D9C00010F5001F4FF000003FF47DAF1946D1E77E
:10D9D0000000E0FF0000F87F944693EA0102F0B5F2
:10D9E0000E4605469E4607D503F100452B46624686
:10D9F000BDE8F04000F0C8B88B4203D8844509D395
:10DA00008B4207D102F1004256408EEA020E2A46AE
:10DA100065469446C6F30A5240F2FF714FEA1E5023
:10DA20008A424FEA1657C0EB165400F09F8094428A
:10DA300000F09880C6F31302CEF313031F2C42F4B8
:10DA4000801143F480134ED823FA04F2891A00F1AE
:10DA50002002D21B93402CFA04F41C432C1B38BF29
:10DA600001F1FF311CFA02F3254603D05B42651E2B
:10DA700004B9013911F4C01F53D1EA0FDB0F42EA98
:10DA8000410243EA450352EA03046CD0BC1E510B29
:10DA900023D0510C01BF190F41EA02121B01043CB3
:10DAA000D10C01BF990F41EA82029B00023C110D8B
:10DAB00002BFD90F41EA420204F1FF344FEAD671A6
:10DAC00008BF5B00B1EBD42F4FF0000006BF02EBA4
:10DAD0000451184606F00041F0BD190E41EA022239
:10DAE0001B02083CD3E7352C1BD8203C23FA04F258
:10DAF000AA1AC4F1200003FA00F338BF01F1FF3184
:10DB00002CFA04F45FEA0C60154643EA040306D0DD
:10DB100043F0FF035B42551E1AB9013901E0002BA7
:10DB2000F8D1CA0209D4013F7A050FD0EA0F42EAC0
:10DB30004101DA0F42EA45055B00002B21F4801217
:10DB40004FEA075405DB11192846C5E73905104689
:10DB5000C2E7013508BF0132B3F1004F08BF25F01D
:10DB60000105F0E75CB921462046B5E733034FF0E5
:10DB7000000001D00349AFE70CB90249F4E7314690
:10DB8000E2E700BF0000F87F2DE9F0431D4695EA6B
:10DB9000010F0E460346AE46174605D505F1004374
:10DBA000BDE8F043FFF718BF8D4284BF2E468E4676
:10DBB00040F2FF7CC6F30A5184BF134607464FEA82
:10DBC0001E5061454FEA1652C0EB16545CD08C4291
:10DBD00055D0C6F3130CCEF313011F2C4CF4801553
:10DBE00041F4801127D82030801A21FA04FC27FA4A
:10DBF00004F4814021435B18654428BF013507FACE
:10DC000000F1A8022BD5013308BF013509B923F073
:10DC10000203360D360506EB5506710011F5001F9F
:10DC200037BFED070132314645EA530024BF0020DB
:10DC30001105BDE8F083352CE3D8203C21FA04F02F
:10DC40001B18C4F1200001FA00F127FA04F428BFE0
:10DC500001352143380618BF41F0FF01D1E7002903
:10DC600002F1FF3207DA013308BF0135B1F1004F8D
:10DC700008BF23F0010305EB02511846D9E74CB960
:10DC800006F000412046D4E732034FF0000001D0F7
:10DC90000149CEE73146F0E70000F87F21F000436C
:10DCA00030B503F1474505F57005B5F17E6F01F01C
:10DCB000004210D2410F03F14843C40041EAC303BC
:10DCC000C0F300700344B4F1004F08BF23F0010318
:10DCD00043EA020030BD002D01DA1046FAE74C009D
:10DCE00014F5001F8CBF024842F0FF40F2E700BF6E
:10DCF0000000C07FC31013F07F610AD0B1F17F6FC5
:10DD00004FEA407243F0E04308D003F14841104627
:10DD1000704703F0004300201946704752EA03326F
:10DD2000014A18BF1346F6E70000F87F08B5FDF773
:10DD30007BFB08BD08B5FDF785FB08BD08B5FDF701
:10DD40008FFB08BD08B5FDF799FB08BD08B5FDF7C9
:10DD5000A3FB08BD08B5FDF7ADFB08BD08B5FDF791
:10DD6000B7FB08BD08B5FDF7C1FB08BD08B5FDF759
:10DD7000CBFB08BD08B5FDF7D5FB08BD08B5FDF721
:10DD8000DFFB08BD08B5FDF7E9FB08BD08B5FDF7E9
:10DD9000F3FB08BD08B5FDF7FDFB08BD08B5FDF7B1
:10DDA00007FC08BD08B5FDF711FC08BD08B5F2F782
:10DDB00058FA08BD08B5F2F754FA08BD08B5F2F7ED
:10DDC00050FA08BD08B5F2F74CFA08BD08B5F2F7ED
:10DDD00048FA08BD08B5F2F744FA08BD08B5F2F7ED
:10DDE00040FA08BD08B5F2F73CFA08BD08B5FDF7E2
:10DDF000BFFD08BD08B5FDF71FFA08BD08B5FDF762
:10DE000033FA08BD08B5F2F72CFA08BD08B5F2F7E9
:10DE100028FA08BD08B5F2F724FA08BD08B5F2F7EC
:10DE200020FA08BD08B5F2F71CFA08BD08B5F2F7EC
:10DE300018FA08BD08B5F2F714FA08BD08B5F2F7EC
:10DE400010FA08BD08B5F2F70CFA08BD08B5F2F7EC
:10DE500008FA08BD08B5F2F704FA08BD08B5F2F7EC
:10DE600000FA08BD08B5F2F7FCF908BD08B5F2F7ED
:10DE7000F8F908BD08B5F2F7F4F908BD08B5F2F7EE
:10DE8000F0F908BD08B5F2F7ECF908BD08B5F2F7EE
:10DE9000E8F908BD08B5F2F7E4F908BD08B5F2F7EE
:10DEA000E0F908BD08B5F2F7DCF908BD08B5F2F7EE
:10DEB000D8F908BD08B5F2F7D4F908BD08B5F2F7EE
:10DEC000D0F908BD08B5F2F7CCF908BD08B5F2F7EE
:10DED000C8F908BD08B5F2F7C4F908BD08B5F2F7EE
:10DEE000C0F908BD08B5F2F7BCF908BD08B5F2F7EE
:10DEF000B8F908BD08B5F2F7B4F908BD08B5FDF7E3
:10DF0000CBF908BD08B5F2F7ACF908BD08B5F2F7D2
:10DF1000A8F908BD08B5F2F7A4F908BD08B5F2F7ED
:10DF2000A0F908BD08B5F2F79CF908BD08B5F2F7ED
:10DF300098F908BD08B5F2F794F908BD08B5FDF7E2
:10DF400025FD08BD08B5F2F78CF908BD08B5F2F754
:10DF500088F908BD08B5F2F784F908BD08B5F2F7ED
:10DF600080F908BD08B5F2F77CF908BD08B5F2F7ED
:10DF700078F908BD08B5FEF7F3F908BD08B5F2F762
:10DF800070F908BD08B5F2F76CF908BD08B5F2F7ED
:10DF900068F908BD08B5F2F764F908BD80B487B028
:10DFA00000AFF860B9601346FB7101237B61FB7918
:10DFB000002B05D17A69BB689A40FB689A6004E03F
:10DFC0007A69BB689A40FB685A6000BF1C37BD463F
:10DFD0005DF8047B704780B483B000AF786039602F
:10DFE0007B681A693B6822FA03F303F001031846C1
:10DFF0000C37BD465DF8047B704780B483B000AF3A
:10E00000786039603B6803F48053002B09D07B684B
:10E010009B79DAB23B681B0ADBB21343DAB27B6846
:10E020009A713B6803F48043002B09D07B689B798D
:10E03000DAB23B681B0ADBB21343DAB27B689A712F
:10E040003B68DAB27B68DA7000BF0C37BD465DF81A
:10E05000047B704780B582B000AF78603960396862
:10E060007868FFF7CAFF00BF0837BD4680BD80B49F
:10E0700083B000AF78600B46FB70FB787A681B01B9
:10E08000134403F586731B6803F0010318460C372D
:10E09000BD465DF8047B704780B485B000AFF86082
:10E0A0000B467A60FB72FB7AFA681B01134403F596
:10E0B00086737A681A6000BF1437BD465DF8047B2A
:10E0C000704780B485B000AF87ED030AC7ED020A40
:10E0D00087ED011A97ED037AD7ED017A27EE277ABB
:10E0E000F7EE006AD7ED017A76EEE76AD7ED027AAD
:10E0F00066EEA77A77EE277AB0EE670A1437BD4648
:10E100005DF8047B704780B483B000AF87ED010AEF
:10E11000C7ED000A97ED017AD7ED007AB4EEE77A01
:10E12000F1EE10FA01D57B6800E03B6807EE903A0B
:10E13000B0EE670A0C37BD465DF8047B704780B4CB
:10E1400083B000AF87ED010AD7ED017A67EEA77AB9
:10E15000B0EE670A0C37BD465DF8047B704780B4AB
:10E1600085B000AF87ED030AC7ED020A87ED011AFB
:10E1700097ED027AD7ED037A37EE677AD7ED017A19
:10E1800027EE277AD7ED037A77EE277AB0EE670A83
:10E190001437BD465DF8047B704780B483B000AF90
:10E1A00087ED010AC7ED000A97ED017AD7ED007AF5
:10E1B000B4EEE77AF1EE10FA01DD7B6800E03B682F
:10E1C00007EE903AB0EE670A0C37BD465DF8047B67
:10E1D000704780B485B000AF87ED030AC7ED020A2F
:10E1E00087ED011A97ED037AD7ED017AB4EEE77A5D
:10E1F000F1EE10FA0CD597ED037AD7ED027AB4EE72
:10E20000E77AF1EE10FA01DDFB6802E0BB6800E09E
:10E210007B6807EE903AB0EE670A1437BD465DF8AA
:10E22000047B704780B485B000AFF860B9607A6055
:10E23000FA687B689A4205DABA68FB689342B8BF0D
:10E24000134600E07B6818461437BD465DF8047B32
:10E25000704780B489B000AFF86187ED060AC7ED5A
:10E26000050A87ED041AC7ED031A87ED022AC7EDE8
:10E27000012A3960FB6900225A62FB693A689A6296
:10E28000FB69BA691A60FB697A695A60FB693A6985
:10E290009A60FB699A68FB69DA60FB697A681A61BF
:10E2A000FB69BA685A61FB69BA689A61FB69FA68E6
:10E2B000DA61FB6993ED017AFB69D3ED007A77EEC1
:10E2C000676AFB6993ED017AFB69D3ED007A37EE5B
:10E2D000677AFB69D3ED027A77EEA77A37EE677A31
:10E2E000C6EE877AFB69C3ED087A00BF2437BD46C6
:10E2F0005DF8047B704780B52DED028B82B000AFD6
:10E30000786087ED000A7B68D3ED067A7B6893ED31
:10E31000077AB0EE471AD7ED000AB0EE670AFFF7AA
:10E320001EFFF0EE407A7B68C3ED067A7B6893EDC2
:10E33000067A7B68D3ED056A7B68D3ED037A76EEC7
:10E34000E77AB4EEE77AF1EE10FA0FD57B6893ED39
:10E35000067A7B68D3ED037A77EE277A7B68C3ED84
:10E36000057A7B689A6A7B685A621EE07B6893ED47
:10E37000067A7B68D3ED056A7B68D3ED037A76EE87
:10E38000A77AB4EEE77AF1EE10FA0EDD7B6893ED32
:10E39000067A7B68D3ED037A77EE677A7B68C3ED04
:10E3A000057A7B689A6A7B685A627B685B6A002B95
:10E3B00029DD7B685B6A5A1E7B685A627B6893ED35
:10E3C000038A7B68D3ED027AB6EE007A67EE878A1D
:10E3D0007B68D3ED047A77EEA77AF7EE000AB0EE09
:10E3E000670AFFF790FEF0EE407AB0EE671AF0EEA3
:10E3F000680AB0EE480AFFF7B2FEF0EE407A7B689A
:10E40000C3ED037A15E07B68D3ED037A7B6893ED67
:10E41000027A7B68D3ED046AB0EE661AF0EE470A22
:10E42000B0EE670AFFF79BFEF0EE407A7B68C3ED23
:10E43000037A7B6893ED057A7B68D3ED026A7B688B
:10E44000D3ED007A76EEA77A37EE677A7B68D3ED64
:10E45000087A27EE277A7B68D3ED007A77EE277A61
:10E460007B6893ED007A7B68D3ED016AB0EE661AA3
:10E47000F0EE470AB0EE670AFFF7ABFEF0EE407A27
:10E48000B0EE670A0837BD46BDEC028B80BD80B494
:10E4900085B000AFF86087ED020AC7ED010A87ED8D
:10E4A000001AFB68BA681A60FB687A685A60FB68F1
:10E4B0003A68DA60FB68DA68FB689A6000BF143774
:10E4C000BD465DF8047B704780B483B000AF7860D0
:10E4D00087ED000A7B683A689A6000BF0C37BD463A
:10E4E0005DF8047B704780B483B000AF78600B4662
:10E4F000FB70FB78002B06D07B681B6843F00102A1
:10E500007B681A6005E07B681B6823F001027B686A
:10E510001A6000BF0C37BD465DF8047B704780B4BD
:10E5200085B000AF786000BF1437BD465DF8047B4E
:10E53000704780B483B000AF0123FB8000E000BFD0
:10E54000FB889BB25A1C92B2FA80002BF7D100BF15
:10E5500000BF0C37BD465DF8047B704780B483B0C4
:10E5600000AF786039607B681A693B6822FA03F370
:10E5700003F0010318460C37BD465DF8047B704775
:10E5800080B485B000AFF860B9607A60FA687B68E3
:10E590009A4205DABA68FB689342B8BF134600E0B6
:10E5A0007B6818461437BD465DF8047B704704202D
:10E5B0007146084202D0EFF3098001E0EFF30880D2
:10E5C00081690A884BF6AB639A4200D0FEE70231BC
:10E5D000816120210160704700BF80B483B000AF2B
:10E5E00078607B685B6A18460C37BD465DF8047B33
:10E5F000704780B582B000AF78607B681B6864218B
:10E60000184600F09CFE00BF0837BD4680BD80B5AF
:10E6100082B000AF786039607B6818687B685B689F
:10E620003A681946FDF762FC034618460837BD46AE
:10E6300080BD80B582B000AF78607B681B681846EB
:10E64000FFF7CBFF034603F08073B3F1807F14BF65
:10E6500001230023DBB218460837BD4680BD80B5D4
:10E660008CB000AF786007F1280300221A605A606E
:10E6700007F1080320220021184601F0A3F8002327
:10E68000BB6007F10803FB620023BB6207F12803AC
:10E690001946786800F07CF80346002B02D040F25F
:10E6A000097300E0002318463037BD4680BD80B4B2
:10E6B00083B000AF786039607B685A6B3B681A435F
:10E6C0007B685A6300BF0C37BD465DF8047B70471A
:10E6D00080B483B000AF78607B685B6A18460C3703
:10E6E000BD465DF8047B704780B483B000AF7860AE
:10E6F0000B46FB707B689B6A23F00602FB785B008D
:10E7000003F006031A437B689A6200BF0C37BD46CC
:10E710005DF8047B704780B483B000AF78600B462F
:10E72000FB70FB78002B06D07B689B6A43F00802E5
:10E730007B689A6205E07B689B6A23F008027B682D
:10E740009A6200BF0C37BD465DF8047B704780B508
:10E7500084B000AF786039607B681B68FB603B6801
:10E76000002B01D101230FE07B683A68DA650121B3
:10E77000F868FFF7D0FF4021F868FFF798FF802185
:10E78000F868FFF794FF002318461037BD4680BD98
:10E7900080B584B000AF786039600023FB607B688F
:10E7A00018687B68D96A7B681A6B3B68FDF752FD75
:10E7B000F860FB6840F2A4629342F0D0FB68002B43
:10E7C00006D00123FB607B681B68184600F005F843
:10E7D000FB6818461037BD4680BD80B584B000AFD9
:10E7E00078600023FB607868FFF772FFF860FB68D1
:10E7F00003F00103002B05D064224FF0007178680C
:10E8000000F074FDFB6803F00203002B05D06422C6
:10E810004FF08061786800F069FD00BF1037BD4699
:10E8200080BD80B582B000AF786039607B681A68BF
:10E830003B68002B06D03B68012B01D1012302E08D
:10E84000022300E0002319461046FFF74DFF00BFEA
:10E850000837BD4680BD80B485B000AF78607B6866
:10E860001B0C03F1804303F58E23FB60FB681968E2
:10E870007B689BB201229A40FB680A431A6000BF82
:10E880001437BD465DF8047B704780B586B000AF95
:10E8900078600023FB7500233B617B681B6A03F0F3
:10E8A0004003002B07D00123FB757B681B6A23F014
:10E8B00040027B681A627B685B6A43F0C0027B6837
:10E8C0005A620AE0786800F0B3F8034603F04003A8
:10E8D000002B02D001233B6108E000217868FBF7A0
:10E8E000F7FE034603F08003002BEBD07B681B6927
:10E8F000FB7D002B05D07B681B6A43F040027B68E0
:10E900001A62786800F094F8034603F04003002B85
:10E9100001D001233B613B69002B01D03B6948E0FA
:10E920007B68DB6CFB607B689B6CFA681344FB6064
:10E930007B685B6CFA681344FB607B681B6CFA684D
:10E940001344FB607B68DB6BFA681344FB607B68F5
:10E950009B6BFA681344FB60FB685B0843F400435D
:10E96000FB607B68FA68DA627B68DB6EFB607B6861
:10E970009B6EFA681344FB607B685B6EFA68134415
:10E98000FB607B681B6EFA681344FB607B68DB6D81
:10E99000FA681344FB607B689B6DFA681344FB6064
:10E9A000FB685B0843F40043FB607B68FA681A630A
:10E9B000002318461837BD4680BD80B483B000AF31
:10E9C00078600B46FB70FB78002B06D17B68DB6818
:10E9D00023F010027B68DA6005E07B68DB6843F0B7
:10E9E00010027B68DA6000BF0C37BD465DF8047B1F
:10E9F000704780B485B000AF78600B46FB707B68D1
:10EA00005B6A23F00703FB60FB78042B07D0FB78DD
:10EA100003F00302FB68134343F00403FB607B68CD
:10EA2000FA685A6200BF1437BD465DF8047B704730
:10EA300080B485B000AF78600023FB607B681B6A00
:10EA400003F08003002B03D0FB6843F08003FB60DE
:10EA50007B685B6A03F04003002B03D0FB6843F044
:10EA60004003FB60FB6818461437BD465DF8047B25
:10EA7000704780B485B000AF786039607B681B78E0
:10EA8000FB73FB7B03F05F03FB733B681A78FB7B34
:10EA90001343FB737B68FA7B1A7000BF1437BD46C3
:10EAA0005DF8047B704780B485B000AF78600B469A
:10EAB000FB707B681B78FB73FB7B23F00F03FB73FE
:10EAC000FA7BFB781343FB737B68FA7B1A7000BFF9
:10EAD0001437BD465DF8047B704780B500AFFBF787
:10EAE0004DFE0346184680BD80B582B000AFFBF7EF
:10EAF00001FF3860FCF77EF80346DB083A689A426B
:10EB000005D83B68002B02D03B687B6001E0002306
:10EB10007B607B6818460837BD4680BD80B483B0F3
:10EB200000AF78607B681846A0F101000028FBD197
:10EB300000BF0C37BD465DF8047B704780B485B0DC
:10EB400000AF78607B681B0C03F1804303F58E23D4
:10EB5000FB60FB6819687B689BB201229A40FB68E6
:10EB60000A431A6000BF1437BD465DF8047B704746
:10EB700080B485B000AF78600023FB737B681B68AE
:10EB8000002B01DA0123FB73FB7B18461437BD46CB
:10EB90005DF8047B704780B487B000AFF860B9605F
:10EBA0001346FB7101237B61FB79002B05D17A6948
:10EBB000BB689A40FB689A6004E07A69BB689A4037
:10EBC000FB685A6000BF1C37BD465DF8047B704788
:10EBD00080B485B000AF78607B681B0C03F1804384
:10EBE00003F58E23FB60FB6819687B689BB20122EA
:10EBF0009A40FB680A431A6000BF1437BD465DF8AF
:10EC0000047B704780B483B000AF786039603B68A4
:10EC100003F48053002B09D07B689B79DAB23B6800
:10EC20001B0ADBB21343DAB27B689A713B6803F4C8
:10EC30008043002B09D07B689B79DAB23B681B0AC2
:10EC4000DBB21343DAB27B689A713B68DAB27B6855
:10EC5000DA7000BF0C37BD465DF8047B704780B4A6
:10EC600085B000AF786039603B6803F04003002B4B
:10EC700007D07B689B78DBB243F04003DAB27B6855
:10EC80009A703B6803F02003002B0DD07B689B79C2
:10EC9000FB73FB7B23F05003FB73FB7B43F02003F0
:10ECA000FB737B68FA7B9A7100BF1437BD465DF831
:10ECB000047B704780B584B000AF78600B46FB7072
:10ECC0001346BB700023FB60786800F050F8B86012
:10ECD000BB6803F02003002B03D040F24C43FB60E1
:10ECE00014E07B689B78DBB243F03003DAB27B68D8
:10ECF0009A70FB785B00DBB2BA78012A01D101225D
:10ED000000E000221343DAB27B681A71FB681846F0
:10ED10001037BD4680BD80B485B000AF7860002359
:10ED2000FB607B689B78DBB223F03803DAB27B6848
:10ED30009A7042F21073BB6000BF7B68DB78DBB275
:10ED400003F02003002B05D0BB68013BBB60BB6810
:10ED5000002BF2D1BB68002B02D14FF48A63FB6019
:10ED6000FB6818461437BD465DF8047B704780B4D5
:10ED700085B000AF78607B68DB78DBB2FB607B68D6
:10ED80009B79DBB203F04003002B03D0FB6843F414
:10ED90008043FB607B689B79DBB203F01003002BA0
:10EDA00003D0FB6843F48053FB60FB6818461437BC
:10EDB000BD465DF8047B704780B588B000AFF86051
:10EDC000B9607A603B600023FB610023FB7542F26F
:10EDD0001073BB6100BFFB68DB78DBB25BB2002B5A
:10EDE00005DBBB69013BBB61BB69002BF3D1BB6990
:10EDF000002B02D14FF48A6366E0FB680222DA70CE
:10EE0000FB689B78DBB243F01003DAB2FB689A70C0
:10EE10003EE0BB685A1CBA601A78FB681A7142F26D
:10EE20001073BB6100BFFB68DB78DBB203F0020349
:10EE3000002B05D1BB69013BBB61BB69002BF2D143
:10EE4000BB69002B02D14FF48A633DE0FB68DB789D
:10EE5000FB75FB680222DA70FB7D03F01003002BC8
:10EE600005D0FB681022DA7040F24F43FB61FB7D56
:10EE700003F00103002B08D07B68002B05D0FB6852
:10EE80000122DA7040F24E43FB61FB69002B05D191
:10EE90007B685A1E7A60002BBBD100E000BFFB6983
:10EEA000002B04D13B6803F00403002B04D0FB6962
:10EEB00040F24E42934206D1FB680222DA70F868B3
:10EEC000FFF729FFF861FB6918462037BD4680BD72
:10EED00080B485B000AF78607B681B0C03F1804381
:10EEE00003F58E23FB60FB6819687B689BB20122E7
:10EEF0009A40FB680A431A6000BF1437BD465DF8AC
:10EF0000047B704780B485B000AF78607B681B0CD1
:10EF100003F1804303F58E23FB60FB6819687B686F
:10EF20009BB201229A40FB680A431A6000BF143763
:10EF3000BD465DF8047B704780B483B000AF786055
:10EF40007B681B6B18460C37BD465DF8047B704729
:10EF500080B483B000AF786039607B683A681A6328
:10EF600000BF0C37BD465DF8047B704780B483B0AA
:10EF700000AF78607B685B6A18460C37BD465DF869
:10EF8000047B704780B483B000AF786039607B68E1
:10EF90003A681A6200BF0C37BD465DF8047B7047C3
:10EFA00080B483B000AF78607B681B6A18460C376A
:10EFB000BD465DF8047B704780B58AB000AFF8604D
:10EFC000B9607A60FB7000237B6207F110030022B6
:10EFD0001A605A609A60DA601A61BB685B7A012B2A
:10EFE00004D17B6A43F4D0137B6246E0BB685B7A52
:10EFF000022B04D17B6A43F4D8137B623DE0BB68EB
:10F000005B7A032B04D17B6A43F410237B6234E0E8
:10F01000BB685B7A042B04D17B6A43F400337B62C8
:10F020002BE0BB685B7A052B04D17B6A43F4003389
:10F030007B6222E0BB685B7A062B04D17B6A43F4D7
:10F04000D0137B6219E0BB685B7A072B04D17B6A23
:10F0500043F4D8137B6210E0BB685B7A082B04D1C1
:10F060007B6A43F4D0137B6207E0BB685B7A092BB1
:10F0700003D17B6A43F4D0137B62BB681B7A032BFA
:10F0800003D17B6A43F440037B627B68002B29D069
:10F090007B6A43F400137B62FB78002B03D07B6A0E
:10F0A00043F001037B627B68DB68002B03D07B6A43
:10F0B00043F010037B627B689B68012B0BD97B6A52
:10F0C00043F022037B627B681B78002B03D07B6AB2
:10F0D00043F004037B627B685B683B617B689B68F1
:10F0E0007B6103E000233B6100237B61BB685B68BD
:10F0F000BB61BB681B68FB617B6A3B6207F1100365
:10F100001946F868FCF7B0FF00BF2837BD4680BD40
:10F1100090B589B000AFF860B9607A60FB685B6C4D
:10F12000DBB27B61BB685B6803F00303002B06D096
:10F13000BB685B6823F003031A1DBB685A60BB6899
:10F140009B68BA68526802FB03F39B083B617A69CB
:10F150003B699A4202D33B69BB6110E07A693B6923
:10F160009A4208D23A697B68D31A7A699A4202D8DD
:10F170007B69BB6103E03A697B68D31ABB610023FA
:10F18000FB610EE0BB68DA687B68591C79609B0004
:10F19000D418F868FFF704FF03462360FB690133C6
:10F1A000FB61FA69BB699A42ECD37B681846243745
:10F1B000BD4690BD80B588B000AFF860B9607A6098
:10F1C000FB685B6C1B0CDBB27B61BB685B6803F0AC
:10F1D0000303002B06D0BB685B6823F003031A1DF2
:10F1E000BB685A60BB689B68BA68526802FB03F34D
:10F1F0009B083B617A693B699A4202D33B69BB61D8
:10F2000010E07A693B699A4208D23A697B68D31A5E
:10F210007A699A4202D87B69BB6103E03A697B68EC
:10F22000D31ABB610023FB610EE0BB681A697B68DF
:10F23000591C79609B0013441B681946F868FFF756
:10F24000A1FEFB690133FB61FA69BB699A42ECD309
:10F250007B6818462037BD4680BD80B584B000AFBE
:10F26000786039600023FB603B68DB68002B09D0C5
:10F2700039687868FCF784FCF860FB68002B0BD0D9
:10F28000FB680AE039687868FCF7D4FCF860FB6832
:10F29000002B01D0FB6800E0002318461037BD4664
:10F2A00080BD80B586B000AF0346B9607A60FB735D
:10F2B00000237B61FB7B002B09D17968B868FFF7DD
:10F2C000CCFF78617B69002B0BD07B690AE0796801
:10F2D000B868FCF751FD78617B69002B01D07B6930
:10F2E00000E0002318461837BD4680BD80B485B0C5
:10F2F00000AFF860B9607A60FB68DA6ABB6803F057
:10F30000E0631A43FB68DA6205E07B68002B09D0F2
:10F310007B68013B7B60FB68DA6ABB681340002BAB
:10F32000F3D100E000BF7B68002B14BF0123002352
:10F33000DBB218461437BD465DF8047B704780B4D5
:10F3400083B000AF786039607B68DB6A43F00062AD
:10F350007B68DA6205E03B68002B09D03B68013B23
:10F360003B607B68DB6A03F00063002BF3D100E0B5
:10F3700000BF3B68002B14BF01230023DBB21846FB
:10F380000C37BD465DF8047B704780B400AF00BF0A
:10F39000BD465DF8047B704780B485B000AF7860EF
:10F3A0007B681B0C03F1804303F58E23FB60FB6835
:10F3B00019687B689BB201229A40FB680A431A6075
:10F3C00000BF1437BD465DF8047B704780B485B03C
:10F3D00000AF78607B681B0C03F1804303F58E233C
:10F3E000FB60FB6819687B689BB2012202FA03F399
:10F3F000DA43FB680A401A6000BF1437BD465DF867
:10F40000047B704780B485B000AF786039607B685A
:10F410001B69FB60FB6823F47053FB60FA683B6870
:10F420001343FB607B68FA681A6100BF1437BD465E
:10F430005DF8047B704780B500AFFDF77BF800BF37
:10F4400080BD80B582B000AF0346FB7197F90730ED
:10F4500013F1800F01D1012305E097F90730184619
:10F46000FDF79AF8002318460837BD4680BD80B4E2
:10F4700083B000AF78600B46FB70FB78002B06D0A2
:10F480007B681B6A43F040027B681A6205E07B6878
:10F490001B6A23F040027B681A6200BF0C37BD462E
:10F4A0005DF8047B704780B483B000AF78600B4692
:10F4B000FB70FB78002B0AD07B6893F82130DBB21D
:10F4C00063F07F03DAB27B6883F8212009E07B6870
:10F4D00093F82130DBB203F07F03DAB27B6883F864
:10F4E000212000BF0C37BD465DF8047B704780B417
:10F4F00085B000AFF8600B467A60FB72FB7AFA6861
:10F500001B01134403F584731968FB7A7A680A4374
:10F51000F9681B010B4403F584731A6000BF1437AC
:10F52000BD465DF8047B704780B485B000AFF860DD
:10F530000B467A60FB72FB7AFA6810331B011344A6
:10F540007A681A6000BF1437BD465DF8047B7047C7
:10F5500080B483B000AF78600B46FB70FB787A68AC
:10F560001B01134403F584731A68FB7842F001020F
:10F5700079681B010B4403F584731A6000BF0C37D4
:10F58000BD465DF8047B704780B500AF00213C208C
:10F59000FDF720F83C20FFF754FF00BF80BD80B589
:10F5A00000AF00213D20FDF715F83D20FFF749FF92
:10F5B00000BF80BD80B500AF00213E20FDF70AF8F6
:10F5C0003E20FFF73EFF00BF80BD80B500AFFDF7D6
:10F5D0002BF8FDF755F8FDF77FF8FDF797F8FFF7E3
:10F5E000D3FFFFF7DCFFFFF7E5FFFDF7A9F8FDF715
:10F5F000BFF8FDF7CFF800BF80BD80B500AFFFF7C3
:10F60000E4FF00BF80BD80B485B000AF78607B6848
:10F610001B0C03F1804303F58E23FB60FB68196824
:10F620007B689BB201229A40FB680A431A6000BFC4
:10F630001437BD465DF8047B704780B485B000AFD9
:10F64000F860B9601346FB71FB68BA6853F8223062
:10F6500023F4E062FB791B0203F4E06342EA030156
:10F66000FB68BA6843F8221000BF1437BD465DF846
:10F67000047B704780B485B000AFF860B960134672
:10F68000FB71FB68BA6853F8223023F47022FB79CF
:10F690001B0403F4702342EA0301FB68BA6843F8D1
:10F6A000221000BF1437BD465DF8047B704780B55B
:10F6B00000AFFDF7CBF800BF80BD80B582B000AFD2
:10F6C0000346FB7197F9073013F1800F01D1012335
:10F6D00005E097F907301846FDF7FAFC00231846B5
:10F6E0000837BD4680BD80B483B000AF7860396014
:10F6F0007B681A693B6822FA03F303F0010318469A
:10F700000C37BD465DF8047B704780B485B000AF10
:10F71000F860B9601346FB71FB68BA6853F8223091
:10F7200023F47022FB791B0403F4702342EA0301E3
:10F73000FB68BA6843F8221000BF1437BD465DF875
:10F74000047B704780B483B000AF78607B68D3F8E7
:10F75000A03018460C37BD465DF8047B704780B476
:10F7600083B000AF786039607B683A68C3F8A02046
:10F7700000BF0C37BD465DF8047B704708B5FDF748
:10F780002DFFBDE80840F7F79FB8B5EEC00AF1EECF
:10F7900010FA48BFB1EE400A7047B5EEC00AF1EE6C
:10F7A00010FAF0EE400A41BFF1EE400A00214FF09E
:10F7B000FF30B0EE600A5CBF00210120F2F778B99B
:10F7C00000F07EBB00F096BBC368826923F0200383
:10F7D00010B5C360836A9A4204460ED000F0B4F8B4
:10F7E000E36823F4405323F0100343F01003E36075
:10F7F000A36AA3612369E3622360E36823F480437F
:10F8000023F04003E36010BDCB6823F4002270B501
:10F810000C46CA609906054602D52046FFF7D4FF7C
:10F82000D4E902365A1C10DAB0050ED4C3F1FF2316
:10F8300003F57F03FE33A360236846F490365A1C19
:10F84000E66022601D70E8B270BD41F28A0232406B
:10F85000022A07D0002346F08006A360E6604FF03E
:10F86000FF30F1E74AF210033340B3F5004F0AD1FD
:10F8700000212046FDF710FEE368990602D52046D8
:10F88000FFF7A2FFE66846F4903316F4706FE3606A
:10F890000ED1606900F053FB00B372051ED504F170
:10F8A0002403236123600123E36146F49233E36080
:10F8B00013F4106F2168266926D0E36A99422CBFA1
:10F8C000C6EB0101C6EB0301B9B9731CE362236007
:10F8D000E36923635A1EA2603570B4E74FF4807069
:10F8E000FDF7CAFDE26820614FF48073E36146F4DE
:10F8F00094331A432060E260DAE722463046FDF78F
:10F9000021FD0028E1D0AAE74A1CEDB222600D706B
:10F91000E26A216891422CBFC6EB0101C6EB0201ED
:10F92000E26922635B0503D40A2D01D08A4209DC17
:10F930000023E6622660A36022463046FDF702FD02
:10F9400000288CD128467FE738B501680569C36A6D
:10F950000446C06820F40022E26000F08202022A1D
:10F9600002D04FF0FF3038BD10F48030FBD0994208
:10F9700038BF19468D4208D1E368E562002023F4C0
:10F9800080332560A060E360EDE72246491B2846EE
:10F99000FDF7D8FC0028EFD0E3E7A8B14FF0805383
:10F9A00040F80C3C50F8042C72B11368B3F1805F3E
:10F9B0000AD150F8083C516803330B4440F8083C26
:10F9C000936840F8043CEDE7704738B555EC104BB0
:10F9D00010EE100A00220023294600F0EDF910B1C4
:10F9E00005F100431D4645EC104B38BD38B50546C2
:10F9F0000C4615F8010B70B1A368013B002BA36006
:10FA000004DB23685A1C22601870F2E72146FFF7D6
:10FA1000FBFE431CEDD138BD40EA01039B0770B5E6
:10FA20000DD104460B46032A1946204607D906681D
:10FA30000D68AE4204F1040403F1040304D002444F
:10FA4000904203D1002008E0043AECE710F8013BB3
:10FA500011F8014BA342F3D0181B70BD70B5C468F8
:10FA6000A50708D0B2F5007F11D0B2F5806F04D0A1
:10FA7000B2F5807F0BD0012008E000F124010123C2
:10FA8000224301610160C361C260002070BD5E1E3F
:10FA90006FF07F45AE42F3D3EDE70028B8BF404298
:10FAA000704710B5421C8307044616D1234654F80C
:10FAB000041BA1F1013020EA010010F0803FF5D0D5
:10FAC00011F0FF0F11D011F47F4F0CD011F47F0F04
:10FAD00014BF23460333981A04E010F8013B002BAF
:10FAE000E1D1801A10BD0233F5E70133F3E770B5B9
:10FAF0000D4606461046144600F02DF82B78722B62
:10FB000017D0772B18D0612B23D1082348F202029B
:10FB100015F8011F2B2912D0622915D01B07E260AE
:10FB2000666104D5022200212046FDF7B5FC20467F
:10FB300070BD00230122EBE704230222E8E742F034
:10FB4000030243F00203E3E742F0040243F001033F
:10FB5000DEE70024EBE7F0B5C468A10789B00546ED
:10FB600022D0220718D4D0E90467FDF7DBFD384620
:10FB700000F0D9F9230502D53046FFF70EFFA40D9A
:10FB8000A40514F1A54F07D1296A2022684600F088
:10FB9000E8F9684600F00BF83C2200212846FFF700
:10FBA00011FE002009B0F0BD4FF0FF30FAE710B5AC
:10FBB0000446FFF776FF01462046BDE8104000F0FE
:10FBC000C4B9C36870B513F00306044611D09B0690
:10FBD00011D5856AFFF7F8FDE36823F44053E3602D
:10FBE0002046FFF7B1FE0022064629462046FDF7D3
:10FBF00053FC304670BD816905680D4401696D1A7A
:10FC0000EAE75FF0000C30B51C0022D112006FD083
:10FC1000914206D305460846002100F06FF80446DD
:10FC2000284600F06BF80A462146BDE830401CF03B
:10FC3000404F08BF704703D54942404261F100017F
:10FC40005FEA8C0C38BF70475B42524263F100039D
:10FC5000704742D41C0C04BF1B040CF1100C13F0B1
:10FC60007F4F04BF1B020CF1080C13F0704F04BF50
:10FC70001B010CF1040C13F0404F04BF0CF1020CFB
:10FC80005FEA83035CBF0CF1010C5B00CCF1200E3A
:10FC900022FA0EF4234302FA0CF200FA0CF520FAD1
:10FCA0000EF001FA0CF4204321FA0EF114461A4624
:10FCB00000F024F8A4FB0023AA1A71EB03033CBF55
:10FCC0001B190138CCF1200E22FA0CF203FA0EF4C3
:10FCD000224323FA0CF30021A7E7821A71EB0303F6
:10FCE0003CBF02460B464FF0000141F100009CE78B
:10FCF00000200021BDE8304000F03DB80423B1EB06
:10FD0000122F09D2090241EA10610002013B08BF2B
:10FD10007047B1EB122FF5D30018494134BF91421F
:10FD2000891A4041494134BF9142891A40414941B1
:10FD300034BF9142891A4041494134BF9142891AE6
:10FD40004041494134BF9142891A4041494134BF41
:10FD50009142891A4041494134BF9142891A404138
:10FD6000494134BF9142891A4041A3F1010313F084
:10FD70000F0FD2D170477047CB0243EA505040F288
:10FD80001E43A3EB115340F00040FF2B20FA03F079
:10FD900011D913F4E06F01D14042704711F0804057
:10FDA00009D04B0013F5001F04D86FF0004000EBA2
:10FDB000D17070470020704730B50D461C4655EA9B
:10FDC000040301460BD4630013F5001F1DD8A542A0
:10FDD00019D31AD190422CBF0020012030BD6800F9
:10FDE00010F5001F11D8630013F5001F0DD80B4349
:10FDF00013431843F2D0A54205D806D1914294BFCF
:10FE000000200120EAE70120E8E70020E6E730B51E
:10FE10000C46194654EA01030BD44B0013F5001F9E
:10FE20001CD88C421CD319D190428CBF00200120D9
:10FE300030BD650015F5001F10D84B0013F5001FED
:10FE40000CD88C420CD801D1904209D218431043EF
:10FE500050EA05030CBF01200020E9E70020E7E796
:10FE60000120E5E730B50C46194654EA01034FEA94
:10FE700044050AD415F5001F1ED88C421ED81BD18C
:10FE8000904234BF0020012030BD15F5001F13D86B
:10FE90004B0013F5001F0FD88C420FD304D19042B2
:10FEA0008CBF00200120EFE71843104350EA050300
:10FEB0000CBF01200020E7E70020E5E70120E3E791
:10FEC00040EA0103DB0703460CD40346043A22BF91
:10FED00051F804CB43F804CBB2F10402F7D2043258
:10FEE00008BF7047013A24BF11F801CB03F801CBDA
:10FEF000F8D87047034613F0030F0ED101F0FF014D
:10FF000041EA012141EA0141043A24BF43F8041BBC
:10FF1000B2F10402F9D202F10402013A24BF03F85B
:10FF2000011BFAE7704703B469460220ABBE02B07A
:10FF3000704703B469460C20ABBE02B0704703B4EF
:10FF400069460920ABBE02B0704703B469460E2073
:10FF5000ABBE02B0704703B469460A20ABBE02B024
:10FF600070470FB469460D20ABBE04B070470FB4A4
:10FF700069460520ABBE04B07047FFFFFFFFFFFFDF
:10FF8000000000000000F03FDA90A4A2AFA4EE3F12
:10FF900087A4FBDC1858ED3F9C5285DD9B19EC3F94
:10FFA000ADD35A999FE8EA3F90F0A38291C4E93F0C
:10FFB000DBA02A42E5ACE83F8701EB7314A1E73FE1
:10FFC000CD3B7F669EA0E63F295448DD07ABE53F69
:10FFD000272A36D5DABFE43F2234124CA6DEE33FAF
:10FFE00015B7310AFE06E33F3862756E7A38E23F94
:10FFF0007B517D3CB872E13F0F89F96C58B5E03F09
:020000021000EC
:10000000000000000000E03F433A5C5573657273E6
:100010005C41646D696E5C446F63756D656E74738D
:100020005C4D43555870726573736F4944455F3139
:10003000312E302E315F323536335C323238655CEA
:100040004D4B3634465835313278787831325F50FE
:10005000726F6A6563745C647269766572732F6629
:10006000736C5F61646331362E683A343839203AF4
:10007000206368616E6E656C47726F7570203C20FE
:100080002875696E7433325F742946534C5F464558
:1000900041545552455F41444331365F434F4E56BC
:1000A000455253494F4E5F434F4E54524F4C5F435E
:1000B0004F554E5400FFFFFF0600000000000000F7
:1000C000040000000700000005000000030000001D
:1000D0000100000002000000100000000D00000000
:1000E0000C000000120000000E0000000A000000DA
:1000F00008000000090000000F00000013000000CD
:10010000170000000B0000001400000011000000A8
:100110001600000015000000202122232425262798
:10012000008100FF00020400030001100302000030
:100130000302010006000400060500200605040075
:100140002E66736C5F73642E633A333238203A2024
:100150006361726400FFFFFF2E66736C5F73642E31
:10016000633A333335203A206361726400FFFFFF46
:100170002E66736C5F73642E633A333432203A20F8
:100180006361726400FFFFFF2E66736C5F73642E01
:10019000633A343332203A206361726400FFFFFF18
:1001A0002E66736C5F73642E633A343538203A20C0
:1001B000636F6E74656E74002E66736C5F73642E6D
:1001C000633A353233203A206361726400FFFFFFE7
:1001D0002E66736C5F73642E633A353536203A2091
:1001E0006361726400FFFFFF2E66736C5F73642EA1
:1001F000633A363031203A206361726400FFFFFFBA
:100200002E66736C5F73642E633A363239203A205F
:1002100063617264000000002E66736C5F73642E6D
:10022000633A363330203A2073746174757300FF7B
:100230002E66736C5F73642E633A363630203A2034
:1002400063617264000000002E66736C5F73642E3D
:10025000633A363631203A2072617753637200FF79
:100260002E66736C5F73642E633A373138203A2000
:100270006361726400FFFFFF2E66736C5F73642E10
:10028000633A373739203A206361726400FFFFFF19
:100290002E66736C5F73642E633A383932203A20CD
:1002A0006361726400FFFFFF2E66736C5F73642EE0
:1002B000633A393330203A206361726400000000F1
:1002C0002E66736C5F73642E633A393331203A20A3
:1002D00072617743736400FF2E66736C5F73642EE4
:1002E000633A31303331203A206361726400FFFF9A
:1002F0002E66736C5F73642E633A31303631203A68
:1003000020636172640000002E66736C5F73642E5C
:10031000633A31303632203A2072617743696400A3
:100320002E66736C5F73642E633A31303836203A30
:10033000206361726400FFFF2E66736C5F73642E2E
:10034000633A31313130203A206361726400FFFF3B
:100350002E66736C5F73642E633A31313635203A02
:10036000206361726400FFFF2E66736C5F73642EFE
:10037000633A31323034203A206361726400FFFF07
:100380002E66736C5F73642E633A31333137203AD3
:1003900020636172640000002E66736C5F73642ECC
:1003A000633A31333138203A2073726300FFFFFF24
:1003B0002E66736C5F73642E633A31333336203AA2
:1003C000206361726400FFFF2E66736C5F73642E9E
:1003D000633A31343035203A206361726400FFFFA4
:1003E0002E66736C5F73642E633A31343336203A71
:1003F00020636172640000002E66736C5F73642E6C
:10040000633A31343337203A20627566666572008C
:100410002E66736C5F73642E633A31343338203A3E
:1004200020626C6F636B436F756E74002E66736C25
:100430005F73642E633A31343339203A20626C6F33
:10044000636B53697A65203D3D2046534C5F5344AE
:100450004D4D435F44454641554C545F424C4F43DC
:100460004B5F53495A4500FF2E66736C5F73642ED1
:10047000633A31343835203A2063617264000000F9
:100480002E66736C5F73642E633A31343836203ACB
:1004900020627566666572002E66736C5F73642EEB
:1004A000633A31343837203A20626C6F636B436FA4
:1004B000756E74002E66736C5F73642E633A31340C
:1004C0003838203A20626C6F636B53697A65203D3F
:1004D0003D2046534C5F53444D4D435F4445464198
:1004E000554C545F424C4F434B5F53495A4500FFB4
:1004F0002E66736C5F73642E633A31363239203A5C
:10050000206361726400FFFF2E66736C5F73642E5C
:10051000633A31363337203A206361726400000059
:100520002E66736C5F73642E633A31363338203A2B
:1005300020627566666572002E66736C5F73642E4A
:10054000633A31363339203A20626C6F636B436F04
:10055000756E74002E66736C5F73642E633A313669
:100560003430203A2028626C6F636B436F756E7471
:10057000202B207374617274426C6F636B29203C72
:100580003D20636172642D3E626C6F636B436F75D7
:100590006E7400FF2E66736C5F73642E633A31369F
:1005A0003933203A20636172640000002E66736C58
:1005B0005F73642E633A31363934203A20627566AF
:1005C000666572002E66736C5F73642E633A313613
:1005D0003935203A20626C6F636B436F756E74001F
:1005E0002E66736C5F73642E633A31363936203A67
:1005F0002028626C6F636B436F756E74202B2073C1
:1006000074617274426C6F636B29203C3D2063619E
:1006100072642D3E626C6F636B436F756E7400FF86
:100620002E66736C5F73642E633A31383037203A2C
:10063000206361726400FFFF2E66736C5F73642E2B
:10064000633A31393130203A20636172640000002E
:100650002E66736C5F73642E633A31393131203A00
:1006600020636172642D3E6973486F7374526561D3
:100670006479203D3D207472756500FF2E66736CB1
:100680005F73642E633A31393931203A20636172E5
:10069000640000002E66736C5F73642E633A313918
:1006A0003932203A20636172642D3E757372506155
:1006B00072616D2E636420213D204E554C4C00FF2D
:1006C0002E66736C5F73646D6D635F686F73742EF9
:1006D000633A313736203A20686F737420213D2009
:1006E0004E554C4C000000002E66736C5F73646DB9
:1006F0006D635F686F73742E633A313737203A2029
:10070000686F73742D3E686F73744576656E7420E0
:10071000213D204E554C4C0000B0034000B00B4032
:100720001B003C101B0030102E66736C5F6164630D
:1007300031362E633A3533203A20696E7374616E18
:100740006365203C2041525241595F53495A452824
:10075000735F616463313642617365732900FFFF23
:100760002E66736C5F61646331362E633A363620D1
:100770003A204E554C4C20213D20636F6E666967D0
:1007800000FFFFFF2E66736C5F61646331362E637A
:100790003A343535203A206368616E6E656C477275
:1007A0006F7570203C204144435F5343315F434F9A
:1007B000554E54002E66736C5F61646331362E6350
:1007C0003A343536203A204E554C4C20213D20639A
:1007D0006F6E66696700FFFF2E66736C5F6164630E
:1007E00031362E633A343835203A206368616E6EB4
:1007F000656C47726F7570203C204144435F5343E2
:10080000315F434F554E54002E66736C5F636C6FBF
:10081000636B2E633A323138203A20305520213D27
:1008200020675F7874616C3046726571000000006B
:100830002E66736C5F636C6F636B2E633A32323378
:10084000203A20305520213D20675F7874616C3359
:10085000324672657100FFFF2E66736C5F636C6FCA
:10086000636B2E633A333539203A20675F787461C1
:100870006C304672657100FF2E66736C5F636C6F3F
:10088000636B2E633A333836203A20675F787461A1
:100890006C333246726571002E66736C5F636C6FE9
:1008A000636B2E633A373631203A206D6367706C84
:1008B0006C30636C6B00FFFF2E66736C5F636C6F54
:1008C000636B2E633A31303137203A20636F6E66A6
:1008D000696700FF2E66736C5F636C6F636B2E63DA
:1008E0003A31383937203A20636F6E66696700FF06
:1008F0002E66736C5F636C6F636B2E633A323137B5
:1009000038203A20636F6E66696700FF8002DC0260
:100910000005B80580079508000A710B2E66736CF8
:100920005F636F6D6D6F6E2E633A323433203A2001
:10093000305520213D2064656C61795F757300003E
:100940002E66736C5F636F6D6D6F6E2E633A32341B
:1009500035203A20636F756E74203C3D2055494E1A
:100960005433325F4D41580000C00C4000D00C4061
:100970000C002C100D002C102E66736C5F646163EC
:100980002E633A3532203A20696E7374616E636566
:10099000203C2041525241595F53495A4528735FC8
:1009A00064616342617365732900FFFF2E66736C97
:1009B0005F6461632E633A3730203A204E554C4CC9
:1009C00020213D20636F6E66696700FF2E66736CA1
:1009D0005F6461632E633A323132203A20696E647B
:1009E0006578203C204441435F4441544C5F434F71
:1009F000554E54002E66736C5F6461632E633A3209
:100A00003330203A20696E646578203C20444143AD
:100A10005F4441544C5F434F554E54002E66736CF7
:100A20005F647370692E633A32313935203A204E53
:100A3000554C4C20213D20675F6473706948616E9E
:100A4000646C655B305D00FF2E66736C5F64737071
:100A5000692E633A32323033203A204E554C4C20C6
:100A6000213D20675F6473706948616E646C655BEB
:100A7000315D00FF2E66736C5F647370692E633A9C
:100A800032323131203A204E554C4C20213D2067E6
:100A90005F6473706948616E646C655B325D00FF12
:100AA0002E66736C5F65646D612E633A3133313548
:100AB000203A2068616E646C6520213D204E554CC3
:100AC0004C00FFFF0090044000A0044000B0044030
:100AD00000C0044000D0044000F00F4040F00F4040
:100AE00080F00F40C0F00F4000F10F402E66736C95
:100AF0005F6770696F2E633A3637203A20696E73EC
:100B000074616E6365203C2041525241595F5349E4
:100B10005A4528735F6770696F4261736573290076
:100B20002E66736C5F6770696F2E633A31303020C8
:100B30003A204E554C4C20213D20636F6E6669670C
:100B400000FFFFFF1400160018001A001C001E0012
:100B5000220028001C002000240028002C00300067
:100B60003800440030003800400048005000580071
:100B70006800800050006000700080009000A000BD
:100B8000C000F000A000C000E00000012001400112
:100B90008001E00140018001C001000240028002AA
:100BA0000003C003800200038003000480040005EA
:100BB0000006800700050006000700080009000A7B
:100BC000000C000F06003410070034100600281037
:100BD000006006400070064000600E402E66736C98
:100BE0005F6932632E633A313539203A20696E737A
:100BF00074616E6365203C2041525241595F5349F4
:100C00005A4528735F69326342617365732900FF37
:100C10002E66736C5F6932632E633A353636203A3E
:100C2000204E554C4C20213D206D617374657243FC
:100C30006F6E6669670000002E66736C5F693263D1
:100C40002E633A353637203A20305520213D207327
:100C50007263436C6F636B5F487A00FF2E66736C40
:100C60005F7069742E633A3535203A20696E73746B
:100C7000616E6365203C2041525241595F53495A8D
:100C80004528735F70697442617365732900FFFFC3
:100C90002E66736C5F7069742E633A3730203A2089
:100CA0004E554C4C20213D20636F6E66696700FFF6
:100CB0002E66736C5F736468632E633A3232382039
:100CC0003A20696E7374616E6365203C2041525214
:100CD00041595F53495A4528735F736468634261A1
:100CE000736529002E66736C5F736468632E633AC4
:100CF000333331203A20636F6D6D616E6420213D86
:100D0000204E554C4C00FFFF2E66736C5F73646879
:100D1000632E633A383130203A20636F6E6669671C
:100D200020213D204E554C4C000000002E66736C77
:100D30005F736468632E633A383132203A20636F00
:100D40006E6669672D3E646D614D6F646520213D5F
:100D5000206B534448435F446D614D6F646541644B
:100D60006D6131002E66736C5F736468632E633A45
:100D7000383134203A2028636F6E6669672D3E77DC
:100D80007269746557617465726D61726B4C6576DA
:100D9000656C203E3D2031554C29202626202863B5
:100DA0006F6E6669672D3E77726974655761746509
:100DB000726D61726B4C6576656C203C3D20313202
:100DC00038554C29000000002E66736C5F73646810
:100DD000632E633A383135203A2028636F6E666996
:100DE000672D3E7265616457617465726D61726BE7
:100DF0004C6576656C203E3D2031554C29202626D9
:100E00002028636F6E6669672D3E72656164576165
:100E10007465726D61726B4C6576656C203C3D202B
:100E2000313238554C2900FF2E66736C5F7364684D
:100E3000632E633A393433203A20737263436C6F04
:100E4000636B5F487A20213D203055002E66736C1D
:100E50005F736468632E633A393434203A20286221
:100E60007573436C6F636B5F487A20213D2030556A
:100E7000292026262028627573436C6F636B5F48B8
:100E80007A203C3D20737263436C6F636B5F487ADA
:100E90002900FFFF2E66736C5F736468632E633AEC
:100EA00031303833203A20636F6E66696720213D08
:100EB000204E554C4C0000002E66736C5F736468C6
:100EC000632E633A31303834203A20636F6E66699E
:100ED000672D3E64617461426C6F636B53697A6520
:100EE000203C3D2028534448435F424C4B415454DE
:100EF000525F424C4B53495A455F4D41534B203E44
:100F00003E20534448435F424C4B415454525F424D
:100F10004C4B53495A455F534849465429000000F9
:100F20002E66736C5F736468632E633A31303835B4
:100F3000203A20636F6E6669672D3E64617461427A
:100F40006C6F636B436F756E74203C3D2028534477
:100F500048435F424C4B415454525F424C4B434ECA
:100F6000545F4D41534B203E3E20534448435F4223
:100F70004C4B415454525F424C4B434E545F534888
:100F80004946542900FFFFFF2E66736C5F73646847
:100F9000632E633A31333836203A207472616E73AF
:100FA00066657220213D204E554C4C002E66736CB8
:100FB0005F736468632E633A31363037203A2073AA
:100FC0005F7364686348616E646C655B305D2021AB
:100FD0003D204E554C4C00FF070000010000000072
:100FE000600306FF03000000000024010024F40059
:100FF0000504A000000001030100000100FFFFFF45
:10100000000101030100000000FFFFFF0100FFFFDE
:101010000100FFFF01000000E09304000000000059
:1010200001000000E09304000000000000FFFFFF4B
:101030000101FFFF2E73646D6D635F636F6E666900
:10104000672E633A3734203A206361726400FFFFF1
:10105000030000002A2A2A206173736572742066D7
:1010600061696C6564203A20002A2A2A205F437354
:1010700079735F616C6C6F63206661696C65640A8B
:081080000072007700FFFFFF82
:1010880020590020805900200000000000000000C6
:1010980000000000000000001E000000000000002A
:1010A8000000000000000000000000000000000038
:1010B8000000000000000000000000000000000028
:1010C8000000000000000000000000000000000018
:1010D800000000000000000000000000000000FF09
:1010E800FF000000000000000000000000000000F9
:1010F800FFFFFF000000000000000000FFFFFF00EE
:10110800000000000000000000FFFF0000000000D9
:101118000000000000000000000000000000FF00C8
:1011280000FF00FF000000FF00000000000000FFBB
:10113800000000FF00000000000000FF000000FFAA
:101148000000000000000000FF0000000000000098
:101158000000000000000000000000000000FF0088
:10116800000000FF000000FF000000000000000079
:10117800000000FF00000000000000FF0000FFFF6B
:1011880000000000000000FF000000000000000058
:1011980000000000000000000000000000FFFFFF4A
:1011A800000000FF00FF00FF00000000000000003A
:1011B80000FFFF0000000000000000FFFF0000FF2C
:1011C80000000000000000FFFFFFFF00000000001B
:1011D8000000000000000000000000000000FF0008
:1011E800000000FF00FF00FF0000000000000000FA
:1011F800FF00000000000000000000FF000000FFEA
:1012080000000000000000FF000000FF00000000D8
:101218000000000000000000000000000000FF00C7
:1012280000000000FF00FF0000000000000000FFB9
:10123800FFFFFFFF000000FF00000000FFFFFF00AE
:10124800000000FF00000000FFFFFF00000000009A
:101258000000000000000000000000000000000086
:101268000000000000000000000000000000000076
:101278000000000000000000000000000000000066
:101288000000000000000000000000000000000056
:10129800000000000000000000000000FFFFFFFF4A
:1012A800FFFFFFFFFFFFFFFFFFFFFFFFFFFFFFFF46
:1012B800FFFFFFFFFFFFFFFFFFFFFFFFFFFFFFFF36
:1012C800FFFFFFFFFFFFFFFFFFFFFFFFFFFFFFFF26
:1012D800FFFFFFFFFFFFFFFFFFFFFFFFFFFFFFFF16
:1012E800FFFFFFFFFFFFFFFFFFFFFFFFFFFFFFFF06
:1012F800FFFFFFFFFFFFFFFFFFFFFFFFFFFFFFFFF6
:10130800FFFFFFFFFFFFFFFFFFFFFFFFFFFFFFFFE5
:10131800FFFFFFFFFFFFFFFFFFFFFFFFFFFFFFFFD5
:10132800FFFFFFFFFFFFFFFFFFFFFFFFFFFFFFFFC5
:10133800FFFFFFFFFFFFFFFFFFFFFFFFFFFFFFFFB5
:10134800FFFFFFFFFFFFFFFFFFFFFFFFFFFFFFFFA5
:10135800FFFFFFFFFFFFFFFFFFFFFFFFFFFFFFFF95
:10136800FFFFFFFFFFFFFFFFFFFFFFFFFFFFFFFF85
:10137800FFFFFFFFFFFFFFFFFFFF0000FFFFFFFF73
:10138800FFFFFFFFFFFFFFFFFFFFFFFFFFFFFFFF65
:10139800FFFFFFFFFFFFFF0000FFFFFFFFFFFFFF53
:1013A800FFFFFFFFFFFFFFFFFFFFFFFFFFFFFFFF45
:1013B800FFFFFFFFFFFFFFFFFF00FFFFFFFFFFFF34
:1013C800FFFFFFFFFFFFFFFFFFFFFFFFFFFFFFFF25
:1013D800FFFFFFFFFFFFFFFFFF00FFFFFFFFFFFF14
:1013E800FFFFFFFFFFFFFFFFFFFFFFFFFFFFFFFF05
:1013F800FFFFFFFFFFFFFFFFFF00FFFFFF00FFFFF3
:10140800FFFFFFFFFFFFFFFFFFFFFFFFFFFFFF00E3
:10141800FFFFFFFFFFFFFFFFFF00FFFFFFFFFFFFD3
:10142800FFFFFFFFFFFFFFFFFFFFFFFFFFFFFFFFC4
:10143800FFFFFFFFFFFFFFFFFFFFFFFF0000FFFFB2
:10144800FFFFFFFFFFFFFFFFFFFFFFFFFFFFFFFFA4
:10145800FFFFFFFFFFFFFFFFFFFFFFFFFFFFFFFF94
:10146800FFFFFFFFFFFFFFFFFFFFFFFFFFFFFFFF84
:10147800FFFFFFFFFFFFFFFFFFFFFFFFFF00FFFF73
:10148800FFFFFFFFFFFFFF0000FF00FFFFFF00005F
:10149800FFFFFF00FF0000FFFFFFFFFFFFFFFFFF51
:1014A800FFFFFFFFFFFFFFFFFFFFFFFFFFFFFFFF44
:1014B800FFFFFFFFFFFFFFFFFFFFFFFFFF00FFFF33
:1014C800FFFFFFFFFFFFFF00FF00FF00FFFFFF0020
:1014D800FFFFFF0000FFFF00FFFFFFFFFFFFFFFF11
:1014E800FFFFFFFFFFFFFFFFFFFFFFFFFFFFFFFF04
:1014F800FFFFFFFFFFFFFFFFFFFFFFFFFF00FFFFF3
:10150800FFFFFFFFFFFFFF00FF00FF00FFFFFF00DF
:10151800FFFFFF00FFFFFF00FFFFFFFFFFFFFFFFD1
:10152800FFFFFFFFFFFFFFFFFFFFFFFFFFFFFFFFC3
:10153800FFFFFFFFFFFFFFFFFFFFFFFFFF00FFFFB2
:10154800FFFFFFFFFFFFFF00FFFFFF00FFFFFF00A0
:10155800FFFFFF00FFFFFF00FFFFFFFFFFFFFFFF91
:10156800FFFFFFFFFFFFFFFFFFFFFFFFFFFFFFFF83
:10157800FFFFFFFFFFFFFFFFFF00FFFF000000FF6F
:10158800FFFFFFFFFFFFFF00FFFFFF00FFFF00005F
:1015980000FFFF00FFFFFF00FF00FFFFFFFFFFFF4F
:1015A800FFFFFFFFFFFFFFFFFFFFFFFFFFFFFFFF43
:1015B800FFFFFFFFFFFFFFFFFF00FFFFFFFFFFFF32
:1015C800FFFFFFFFFFFFFFFFFFFFFFFFFFFFFFFF23
:1015D800FFFFFFFFFFFFFFFFFF00FFFFFFFFFFFF12
:1015E800FFFFFFFFFFFFFFFFFFFFFFFFFFFFFFFF03
:1015F800FFFFFFFFFFFFFFFFFFFF0000FFFFFFFFF1
:10160800FFFFFFFFFFFFFFFFFFFFFFFFFFFFFFFFE2
:10161800FFFFFFFFFFFFFF0000FFFFFFFFFFFFFFD0
:10162800FFFFFFFFFFFFFFFFFFFFFFFFFFFFFFFFC2
:10163800FFFFFFFFFFFFFFFFFFFFFFFFFFFFFFFFB2
:10164800FFFFFFFFFFFFFFFFFFFFFFFFFFFFFFFFA2
:10165800FFFFFFFFFFFFFFFFFFFFFFFFFFFFFFFF92
:10166800FFFFFFFFFFFFFFFFFFFFFFFFFFFFFFFF82
:10167800FFFFFFFFFFFFFFFFFFFFFFFFFFFFFFFF72
:10168800FFFFFFFFFFFFFFFFFFFFFFFFFFFFFFFF62
:10169800FFFFFFFFFFFFFFFFFFFFFFFFFFFFFFFF52
:1016A800FFFFFFFFFFFFFFFFFFFFFFFFFFFFFFFF42
:1016B800FFFFFFFFFFFFFFFFFFFFFFFFFFFFFFFF32
:1016C800FFFFFFFFFFFFFFFFFFFFFFFFFFFFFFFF22
:1016D800FFFFFFFFFFFFFFFFFFFFFFFFFFFFFFFF12
:1016E800FFFFFFFFFF00FFFFFFFFFFFFFFFFFFFF01
:1016F800FFFFFFFFFFFFFFFFFFFFFFFFFFFFFFFFF2
:10170800FFFFFFFFFFFFFFFFFFFFFFFFFFFFFFFFE1
:10171800FFFFFFFFFFFFFFFFFFFFFFFFFFFF0000CF
:1017280000FFFFFF00FFFFFFFFFF000000FFFFFFBC
:10173800000000FFFF00FFFFFF00FFFF000000FFA9
:10174800FF00FF0000FFFFFFFFFFFFFFFFFFFFFF9E
:10175800FFFFFFFFFFFFFFFFFFFFFFFFFF00FFFF90
:10176800FFFFFFFFFFFFFFFFFF00FFFFFFFFFFFF80
:10177800FFFFFF00FF00FFFFFF00FF00FFFFFF006C
:10178800FF0000FFFF00FFFFFFFFFFFFFFFFFFFF5E
:10179800FFFFFFFFFFFFFFFFFFFFFFFFFFFF00004F
:1017A80000FFFFFFFFFFFFFFFFFF000000FFFFFF3D
:1017B80000000000FF00FFFFFF00FF000000000026
:1017C800FF00FFFFFFFFFFFFFFFFFFFFFFFFFFFF20
:1017D800FFFFFFFFFFFFFFFFFFFFFFFFFFFFFFFF11
:1017E800FF00FFFFFFFFFFFFFFFFFFFFFF00FF00FE
:1017F800FFFFFF00FFFF00FF00FFFF00FFFFFFFFED
:10180800FF00FFFFFFFFFFFFFFFFFFFFFFFFFFFFDF
:10181800FFFFFFFFFFFFFFFFFFFFFFFFFF000000CD
:1018280000FFFFFFFFFFFFFFFF00000000FFFFFFBB
:1018380000000000FFFFFF00FFFFFFFF000000FFA8
:10184800FF00FFFFFFFFFFFFFFFFFFFFFFFFFFFF9F
:10185800FFFFFFFFFFFFFFFFFFFFFFFFFFFFFFFF90
:10186800FFFFFFFFFFFFFFFFFFFFFFFFFFFFFFFF80
:10187800FFFFFFFFFFFFFFFFFFFFFFFFFFFFFFFF70
:10188800FFFFFFFFFFFFFFFFFFFFFFFFFFFFFFFF60
:10189800FFFFFFFFFFFFFFFFFFFFFFFF000000004C
:1018A8000000000000000000000000000000000030
:1018B8000000000000000000000000000000000020
:1018C8000000000000000000000000000000000010
:1018D800000000000000000000000000000000FF01
:1018E800FF000000000000000000000000000000F1
:1018F800FFFFFF000000000000000000FFFFFF00E6
:10190800000000000000000000FFFF0000000000D1
:101918000000000000000000000000000000FF00C0
:1019280000FF00FF000000FF00000000000000FFB3
:10193800000000FF00000000000000FF000000FFA2
:101948000000000000000000FF0000000000000090
:101958000000000000000000000000000000FF0080
:10196800000000FF000000FF000000000000000071
:10197800000000FF00000000000000FF0000FFFF63
:1019880000000000000000FF000000000000000050
:1019980000000000000000000000000000FFFFFF42
:1019A800000000FF00FF00FF000000000000000032
:1019B80000FFFF0000000000000000FFFF0000FF24
:1019C80000000000000000FFFFFFFF000000000013
:1019D8000000000000000000000000000000FF0000
:1019E800000000FF00FF00FF0000000000000000F2
:1019F800FF00000000000000000000FF000000FFE2
:101A080000000000000000FF000000FF00000000D0
:101A18000000000000000000000000000000FF00BF
:101A280000000000FF00FF0000000000000000FFB1
:101A3800FFFFFFFF000000FF00000000FFFFFF00A6
:101A4800000000FF00000000FFFFFF000000000092
:101A5800000000000000000000000000000000007E
:101A6800000000000000000000000000000000006E
:101A7800000000000000000000000000000000005E
:101A8800000000000000000000000000000000004E
:101A9800000000000000000000000000FFFFFFFF42
:101AA800FFFFFFFFFFFFFFFFFFFFFFFFFFFFFFFF3E
:101AB800FFFFFFFFFFFFFFFFFFFFFFFFFFFFFFFF2E
:101AC800FFFFFFFFFFFFFFFFFFFFFFFFFFFFFFFF1E
:101AD800FFFFFFFFFFFFFFFFFFFFFFFFFFFFFFFF0E
:101AE800FFFFFFFFFFFFFFFFFFFFFFFFFFFFFFFFFE
:101AF800FFFFFFFFFFFFFFFFFFFFFFFFFFFFFFFFEE
:101B0800FFFFFFFFFFFFFFFFFFFFFFFFFFFFFFFFDD
:101B1800FFFFFFFFFFFFFFFFFFFFFFFFFFFFFFFFCD
:101B2800FFFFFFFFFFFFFFFFFFFFFFFFFFFFFFFFBD
:101B3800FFFFFFFFFFFFFFFFFFFFFFFFFFFFFFFFAD
:101B4800FFFFFFFFFFFFFFFFFFFFFFFFFFFFFFFF9D
:101B5800FFFFFFFFFFFFFFFFFFFFFFFFFFFFFFFF8D
:101B6800FFFFFFFFFFFFFFFFFFFFFFFFFFFFFFFF7D
:101B7800FFFFFFFFFFFFFFFFFFFF0000FFFFFFFF6B
:101B8800FFFFFFFFFFFFFFFFFFFFFFFFFFFFFFFF5D
:101B9800FFFFFFFFFFFFFF0000FFFFFFFFFFFFFF4B
:101BA800FFFFFFFFFFFFFFFFFFFFFFFFFFFFFFFF3D
:101BB800FFFFFFFFFFFFFFFFFF00FFFFFFFFFFFF2C
:101BC800FFFFFFFFFFFFFFFFFFFFFFFFFFFFFFFF1D
:101BD800FFFFFFFFFFFFFFFFFF00FFFFFFFFFFFF0C
:101BE800FFFFFFFFFFFFFFFFFFFFFFFFFFFFFFFFFD
:101BF800FFFFFFFFFFFFFFFFFF00FF0000000000E7
